Component: ARM Compiler 5.06 update 1 (build 61) Tool: armlink [4d35a8]

==============================================================================

Section Cross References

    main.o(i.main) refers to delay.o(i.delay_init) for delay_init
    main.o(i.main) refers to usart1.o(i.usart1_Configuration) for usart1_Configuration
    main.o(i.main) refers to os_core.o(i.OSInit) for OSInit
    main.o(i.main) refers to os_task.o(i.OSTaskCreate) for OSTaskCreate
    main.o(i.main) refers to os_core.o(i.OSStart) for OSStart
    main.o(i.main) refers to stm32_config.o(.bss) for START_TASK_STK
    main.o(i.main) refers to main.o(i.start_task) for start_task
    main.o(i.start_task) refers to printf3.o(i.__0printf$3) for __2printf
    main.o(i.start_task) refers to delay.o(i.delay_ms) for delay_ms
    main.o(i.start_task) refers to stm32f107.o(i.System_Setup) for System_Setup
    main.o(i.start_task) refers to netconf.o(i.LwIP_Init) for LwIP_Init
    main.o(i.start_task) refers to os_core.o(i.OSStatInit) for OSStatInit
    main.o(i.start_task) refers to os_cpu_a.o(.text) for OS_CPU_SR_Save
    main.o(i.start_task) refers to os_task.o(i.OSTaskCreate) for OSTaskCreate
    main.o(i.start_task) refers to os_task.o(i.OSTaskSuspend) for OSTaskSuspend
    main.o(i.start_task) refers to stm32_config.o(.bss) for LED1_TASK_STK
    main.o(i.start_task) refers to main_server.o(i.main_Server_task) for main_Server_task
    main.o(i.start_task) refers to main_cilent.o(i.main_Client_task) for main_Client_task
    main_server.o(i.main_Server_task) refers to memseta.o(.text) for __aeabi_memclr4
    main_server.o(i.main_Server_task) refers to tcpserver.o(i.tcp_echoserver_init) for tcp_echoserver_init
    main_server.o(i.main_Server_task) refers to tcpserver.o(i.TCP_Server_Recv) for TCP_Server_Recv
    main_server.o(i.main_Server_task) refers to printf3.o(i.__0printf$3) for __2printf
    main_server.o(i.main_Server_task) refers to tcpserver.o(i.TCP_Server_Send) for TCP_Server_Send
    main_server.o(i.main_Server_task) refers to delay.o(i.delay_ms) for delay_ms
    main_cilent.o(i.main_Client_task) refers to memseta.o(.text) for __aeabi_memclr4
    main_cilent.o(i.main_Client_task) refers to printf3.o(i.__0printf$3) for __2printf
    main_cilent.o(i.main_Client_task) refers to tcpclient.o(i.tcp_echoclient_connect) for tcp_echoclient_connect
    main_cilent.o(i.main_Client_task) refers to delay.o(i.delay_ms) for delay_ms
    main_cilent.o(i.main_Client_task) refers to tcpclient.o(i.TCP_Client_Recv) for TCP_Client_Recv
    main_cilent.o(i.main_Client_task) refers to tcpclient.o(i.TCP_Client_Send) for TCP_Client_Send
    main_cilent.o(i.main_Client_task) refers to tcpclient.o(i.tcp_client_close) for tcp_client_close
    main_cilent.o(i.main_Client_task) refers to tcpclient.o(.data) for TcpClient_Link
    netconf.o(i.Display_Periodic_Handle) refers to printf3.o(i.__0sprintf$3) for __2sprintf
    netconf.o(i.Display_Periodic_Handle) refers to netconf.o(.data) for DisplayTimer
    netconf.o(i.Display_Periodic_Handle) refers to netconf.o(.bss) for netif
    netconf.o(i.LwIP_Init) refers to mem.o(i.mem_init) for mem_init
    netconf.o(i.LwIP_Init) refers to memp.o(i.memp_init) for memp_init
    netconf.o(i.LwIP_Init) refers to inet.o(i.htonl) for htonl
    netconf.o(i.LwIP_Init) refers to ethernetif.o(i.Set_MAC_Address) for Set_MAC_Address
    netconf.o(i.LwIP_Init) refers to netif.o(i.netif_add) for netif_add
    netconf.o(i.LwIP_Init) refers to netif.o(i.netif_set_default) for netif_set_default
    netconf.o(i.LwIP_Init) refers to netif.o(i.netif_set_up) for netif_set_up
    netconf.o(i.LwIP_Init) refers to etharp.o(i.ethernet_input) for ethernet_input
    netconf.o(i.LwIP_Init) refers to ethernetif.o(i.ethernetif_init) for ethernetif_init
    netconf.o(i.LwIP_Init) refers to netconf.o(.bss) for netif
    netconf.o(i.LwIP_Periodic_Handle) refers to tcp.o(i.tcp_tmr) for tcp_tmr
    netconf.o(i.LwIP_Periodic_Handle) refers to etharp.o(i.etharp_tmr) for etharp_tmr
    netconf.o(i.LwIP_Periodic_Handle) refers to netconf.o(.data) for TCPTimer
    netconf.o(i.LwIP_Pkt_Handle) refers to ethernetif.o(i.ethernetif_input) for ethernetif_input
    netconf.o(i.LwIP_Pkt_Handle) refers to netconf.o(.bss) for netif
    stm32_eth.o(i.ETH_DMAPTPRxDescChainInit) refers to stm32_eth.o(.data) for DMARxDescToGet
    stm32_eth.o(i.ETH_DMAPTPTxDescChainInit) refers to stm32_eth.o(.data) for DMATxDescToSet
    stm32_eth.o(i.ETH_DMARxDescChainInit) refers to stm32_eth.o(.data) for DMARxDescToGet
    stm32_eth.o(i.ETH_DMARxDescRingInit) refers to stm32_eth.o(.data) for DMARxDescToGet
    stm32_eth.o(i.ETH_DMATxDescChainInit) refers to stm32_eth.o(.data) for DMATxDescToSet
    stm32_eth.o(i.ETH_DMATxDescRingInit) refers to stm32_eth.o(.data) for DMATxDescToSet
    stm32_eth.o(i.ETH_DeInit) refers to stm32f10x_rcc.o(i.RCC_AHBPeriphResetCmd) for RCC_AHBPeriphResetCmd
    stm32_eth.o(i.ETH_DropRxPkt) refers to stm32_eth.o(.data) for DMARxDescToGet
    stm32_eth.o(i.ETH_GetRxPktSize) refers to stm32_eth.o(i.ETH_GetDMARxDescFrameLength) for ETH_GetDMARxDescFrameLength
    stm32_eth.o(i.ETH_GetRxPktSize) refers to stm32_eth.o(.data) for DMARxDescToGet
    stm32_eth.o(i.ETH_HandlePTPRxPkt) refers to stm32_eth.o(.data) for DMARxDescToGet
    stm32_eth.o(i.ETH_HandlePTPTxPkt) refers to stm32_eth.o(.data) for DMATxDescToSet
    stm32_eth.o(i.ETH_HandleRxPkt) refers to stm32_eth.o(.data) for DMARxDescToGet
    stm32_eth.o(i.ETH_HandleTxPkt) refers to stm32_eth.o(.data) for DMATxDescToSet
    stm32_eth.o(i.ETH_Init) refers to stm32f10x_rcc.o(i.RCC_GetClocksFreq) for RCC_GetClocksFreq
    stm32_eth.o(i.ETH_Init) refers to stm32_eth.o(i.ETH_WritePHYRegister) for ETH_WritePHYRegister
    stm32_eth.o(i.ETH_Init) refers to stm32_eth.o(i.ETH_Delay) for ETH_Delay
    stm32_eth.o(i.ETH_Init) refers to stm32_eth.o(i.ETH_ReadPHYRegister) for ETH_ReadPHYRegister
    stm32_eth.o(i.ETH_PHYLoopBackCmd) refers to stm32_eth.o(i.ETH_ReadPHYRegister) for ETH_ReadPHYRegister
    stm32_eth.o(i.ETH_PHYLoopBackCmd) refers to stm32_eth.o(i.ETH_WritePHYRegister) for ETH_WritePHYRegister
    stm32_eth.o(i.ETH_Start) refers to stm32_eth.o(i.ETH_MACTransmissionCmd) for ETH_MACTransmissionCmd
    stm32_eth.o(i.ETH_Start) refers to stm32_eth.o(i.ETH_FlushTransmitFIFO) for ETH_FlushTransmitFIFO
    stm32_eth.o(i.ETH_Start) refers to stm32_eth.o(i.ETH_MACReceptionCmd) for ETH_MACReceptionCmd
    stm32_eth.o(i.ETH_Start) refers to stm32_eth.o(i.ETH_DMATransmissionCmd) for ETH_DMATransmissionCmd
    stm32_eth.o(i.ETH_Start) refers to stm32_eth.o(i.ETH_DMAReceptionCmd) for ETH_DMAReceptionCmd
    stm32f107.o(i.Ethernet_Configuration) refers to stm32f10x_gpio.o(i.GPIO_ETH_MediaInterfaceConfig) for GPIO_ETH_MediaInterfaceConfig
    stm32f107.o(i.Ethernet_Configuration) refers to stm32f10x_rcc.o(i.RCC_PLL3Config) for RCC_PLL3Config
    stm32f107.o(i.Ethernet_Configuration) refers to stm32f10x_rcc.o(i.RCC_PLL3Cmd) for RCC_PLL3Cmd
    stm32f107.o(i.Ethernet_Configuration) refers to stm32f10x_rcc.o(i.RCC_GetFlagStatus) for RCC_GetFlagStatus
    stm32f107.o(i.Ethernet_Configuration) refers to stm32f10x_rcc.o(i.RCC_MCOConfig) for RCC_MCOConfig
    stm32f107.o(i.Ethernet_Configuration) refers to stm32_eth.o(i.ETH_DeInit) for ETH_DeInit
    stm32f107.o(i.Ethernet_Configuration) refers to stm32_eth.o(i.ETH_SoftwareReset) for ETH_SoftwareReset
    stm32f107.o(i.Ethernet_Configuration) refers to stm32_eth.o(i.ETH_GetSoftwareResetStatus) for ETH_GetSoftwareResetStatus
    stm32f107.o(i.Ethernet_Configuration) refers to stm32_eth.o(i.ETH_StructInit) for ETH_StructInit
    stm32f107.o(i.Ethernet_Configuration) refers to stm32_eth.o(i.ETH_Init) for ETH_Init
    stm32f107.o(i.Ethernet_Configuration) refers to stm32_eth.o(i.ETH_DMAITConfig) for ETH_DMAITConfig
    stm32f107.o(i.GPIO_Configuration) refers to stm32f10x_gpio.o(i.GPIO_Init) for GPIO_Init
    stm32f107.o(i.NVIC_Configuration) refers to misc.o(i.NVIC_SetVectorTable) for NVIC_SetVectorTable
    stm32f107.o(i.NVIC_Configuration) refers to misc.o(i.NVIC_PriorityGroupConfig) for NVIC_PriorityGroupConfig
    stm32f107.o(i.NVIC_Configuration) refers to misc.o(i.NVIC_Init) for NVIC_Init
    stm32f107.o(i.System_Setup) refers to stm32f10x_rcc.o(i.RCC_APB1PeriphClockCmd) for RCC_APB1PeriphClockCmd
    stm32f107.o(i.System_Setup) refers to stm32f10x_rcc.o(i.RCC_AHBPeriphClockCmd) for RCC_AHBPeriphClockCmd
    stm32f107.o(i.System_Setup) refers to stm32f10x_rcc.o(i.RCC_APB2PeriphClockCmd) for RCC_APB2PeriphClockCmd
    stm32f107.o(i.System_Setup) refers to stm32f107.o(i.NVIC_Configuration) for NVIC_Configuration
    stm32f107.o(i.System_Setup) refers to stm32f107.o(i.GPIO_Configuration) for GPIO_Configuration
    stm32f107.o(i.System_Setup) refers to stm32f107.o(i.Ethernet_Configuration) for Ethernet_Configuration
    stm32f107.o(i.System_Setup) refers to stm32f10x_rcc.o(i.RCC_GetClocksFreq) for RCC_GetClocksFreq
    stm32f107.o(i.System_Setup) refers to stm32f107.o(i.NVIC_SetPriority) for NVIC_SetPriority
    tcpclient.o(i.TCP_Client_Recv) refers to tcpclient.o(.data) for TcpClient_len
    tcpclient.o(i.TCP_Client_Recv) refers to tcpclient.o(.bss) for TcpClient_buff
    tcpclient.o(i.TCP_Client_Send) refers to tcp_out.o(i.tcp_write) for tcp_write
    tcpclient.o(i.TCP_Client_Send) refers to tcp_out.o(i.tcp_output) for tcp_output
    tcpclient.o(i.TCP_Client_Send) refers to tcpclient.o(.data) for Socket_Client
    tcpclient.o(i.tcp_client_close) refers to tcpclient.o(i.tcp_echoclient_connection_close) for tcp_echoclient_connection_close
    tcpclient.o(i.tcp_client_close) refers to tcpclient.o(.data) for rjes
    tcpclient.o(i.tcp_client_error) refers to tcpclient.o(i.tcp_echoclient_connection_close) for tcp_echoclient_connection_close
    tcpclient.o(i.tcp_client_error) refers to printf3.o(i.__0printf$3) for __2printf
    tcpclient.o(i.tcp_client_error) refers to tcpclient.o(.data) for Socket_Client
    tcpclient.o(i.tcp_client_error) refers to tcpclient.o(.constdata) for __FUNCTION__
    tcpclient.o(i.tcp_client_sent) refers to printf3.o(i.__0printf$3) for __2printf
    tcpclient.o(i.tcp_client_sent) refers to tcpclient.o(.constdata) for __FUNCTION__
    tcpclient.o(i.tcp_echoclient_connect) refers to tcp.o(i.tcp_new) for tcp_new
    tcpclient.o(i.tcp_echoclient_connect) refers to inet.o(i.htonl) for htonl
    tcpclient.o(i.tcp_echoclient_connect) refers to printf3.o(i.__0printf$3) for __2printf
    tcpclient.o(i.tcp_echoclient_connect) refers to tcp.o(i.tcp_connect) for tcp_connect
    tcpclient.o(i.tcp_echoclient_connect) refers to tcpclient.o(.data) for echoclient_pcb
    tcpclient.o(i.tcp_echoclient_connect) refers to tcpclient.o(.constdata) for __FUNCTION__
    tcpclient.o(i.tcp_echoclient_connect) refers to tcpclient.o(i.tcp_echoclient_connected) for tcp_echoclient_connected
    tcpclient.o(i.tcp_echoclient_connected) refers to mem.o(i.mem_malloc) for mem_malloc
    tcpclient.o(i.tcp_echoclient_connected) refers to tcp.o(i.tcp_arg) for tcp_arg
    tcpclient.o(i.tcp_echoclient_connected) refers to tcp.o(i.tcp_recv) for tcp_recv
    tcpclient.o(i.tcp_echoclient_connected) refers to tcp.o(i.tcp_err) for tcp_err
    tcpclient.o(i.tcp_echoclient_connected) refers to tcp.o(i.tcp_sent) for tcp_sent
    tcpclient.o(i.tcp_echoclient_connected) refers to tcp.o(i.tcp_poll) for tcp_poll
    tcpclient.o(i.tcp_echoclient_connected) refers to tcpclient.o(i.tcp_echoclient_connection_close) for tcp_echoclient_connection_close
    tcpclient.o(i.tcp_echoclient_connected) refers to tcpclient.o(.data) for TcpClient_Link
    tcpclient.o(i.tcp_echoclient_connected) refers to tcpclient.o(i.tcp_echoclient_recv) for tcp_echoclient_recv
    tcpclient.o(i.tcp_echoclient_connected) refers to tcpclient.o(i.tcp_client_error) for tcp_client_error
    tcpclient.o(i.tcp_echoclient_connected) refers to tcpclient.o(i.tcp_client_sent) for tcp_client_sent
    tcpclient.o(i.tcp_echoclient_connected) refers to tcpclient.o(i.tcp_echoclient_poll) for tcp_echoclient_poll
    tcpclient.o(i.tcp_echoclient_connection_close) refers to tcp.o(i.tcp_arg) for tcp_arg
    tcpclient.o(i.tcp_echoclient_connection_close) refers to tcp.o(i.tcp_recv) for tcp_recv
    tcpclient.o(i.tcp_echoclient_connection_close) refers to tcp.o(i.tcp_sent) for tcp_sent
    tcpclient.o(i.tcp_echoclient_connection_close) refers to tcp.o(i.tcp_err) for tcp_err
    tcpclient.o(i.tcp_echoclient_connection_close) refers to tcp.o(i.tcp_poll) for tcp_poll
    tcpclient.o(i.tcp_echoclient_connection_close) refers to mem.o(i.mem_free) for mem_free
    tcpclient.o(i.tcp_echoclient_connection_close) refers to tcp.o(i.tcp_close) for tcp_close
    tcpclient.o(i.tcp_echoclient_poll) refers to printf3.o(i.__0printf$3) for __2printf
    tcpclient.o(i.tcp_echoclient_poll) refers to tcpclient.o(i.tcp_echoclient_connection_close) for tcp_echoclient_connection_close
    tcpclient.o(i.tcp_echoclient_poll) refers to tcp.o(i.tcp_abandon) for tcp_abandon
    tcpclient.o(i.tcp_echoclient_poll) refers to tcpclient.o(.constdata) for __FUNCTION__
    tcpclient.o(i.tcp_echoclient_recv) refers to tcpclient.o(i.tcp_echoclient_connection_close) for tcp_echoclient_connection_close
    tcpclient.o(i.tcp_echoclient_recv) refers to pbuf.o(i.pbuf_free) for pbuf_free
    tcpclient.o(i.tcp_echoclient_recv) refers to tcp.o(i.tcp_recved) for tcp_recved
    tcpclient.o(i.tcp_echoclient_recv) refers to tcpclient.o(.data) for TcpClient_Link
    tcpclient.o(i.tcp_echoclient_recv) refers to tcpclient.o(.bss) for TcpClient_buff
    tcpserver.o(i.TCP_Server_Recv) refers to tcpserver.o(.data) for TcpServer_len
    tcpserver.o(i.TCP_Server_Recv) refers to tcpserver.o(.bss) for TcpServer_buff
    tcpserver.o(i.TCP_Server_Send) refers to tcp_out.o(i.tcp_write) for tcp_write
    tcpserver.o(i.TCP_Server_Send) refers to tcp_out.o(i.tcp_output) for tcp_output
    tcpserver.o(i.TCP_Server_Send) refers to tcpserver.o(.data) for Socket_Server
    tcpserver.o(i.tcp_echoserver_accept) refers to printf3.o(i.__0printf$3) for __2printf
    tcpserver.o(i.tcp_echoserver_accept) refers to tcp.o(i.tcp_setprio) for tcp_setprio
    tcpserver.o(i.tcp_echoserver_accept) refers to mem.o(i.mem_malloc) for mem_malloc
    tcpserver.o(i.tcp_echoserver_accept) refers to tcp.o(i.tcp_arg) for tcp_arg
    tcpserver.o(i.tcp_echoserver_accept) refers to tcp.o(i.tcp_recv) for tcp_recv
    tcpserver.o(i.tcp_echoserver_accept) refers to tcp.o(i.tcp_err) for tcp_err
    tcpserver.o(i.tcp_echoserver_accept) refers to tcp.o(i.tcp_poll) for tcp_poll
    tcpserver.o(i.tcp_echoserver_accept) refers to tcpserver.o(.constdata) for __FUNCTION__
    tcpserver.o(i.tcp_echoserver_accept) refers to tcpserver.o(i.tcp_echoserver_recv) for tcp_echoserver_recv
    tcpserver.o(i.tcp_echoserver_accept) refers to tcpserver.o(i.tcp_echoserver_error) for tcp_echoserver_error
    tcpserver.o(i.tcp_echoserver_accept) refers to tcpserver.o(i.tcp_echoserver_poll) for tcp_echoserver_poll
    tcpserver.o(i.tcp_echoserver_accept) refers to tcpserver.o(.data) for Socket_Server
    tcpserver.o(i.tcp_echoserver_connection_close) refers to tcp.o(i.tcp_arg) for tcp_arg
    tcpserver.o(i.tcp_echoserver_connection_close) refers to tcp.o(i.tcp_sent) for tcp_sent
    tcpserver.o(i.tcp_echoserver_connection_close) refers to tcp.o(i.tcp_recv) for tcp_recv
    tcpserver.o(i.tcp_echoserver_connection_close) refers to tcp.o(i.tcp_err) for tcp_err
    tcpserver.o(i.tcp_echoserver_connection_close) refers to tcp.o(i.tcp_poll) for tcp_poll
    tcpserver.o(i.tcp_echoserver_connection_close) refers to mem.o(i.mem_free) for mem_free
    tcpserver.o(i.tcp_echoserver_connection_close) refers to tcp.o(i.tcp_close) for tcp_close
    tcpserver.o(i.tcp_echoserver_error) refers to tcpserver.o(i.tcp_echoserver_connection_close) for tcp_echoserver_connection_close
    tcpserver.o(i.tcp_echoserver_error) refers to mem.o(i.mem_free) for mem_free
    tcpserver.o(i.tcp_echoserver_error) refers to tcpserver.o(.data) for Socket_Server
    tcpserver.o(i.tcp_echoserver_init) refers to tcp.o(i.tcp_new) for tcp_new
    tcpserver.o(i.tcp_echoserver_init) refers to tcp.o(i.tcp_bind) for tcp_bind
    tcpserver.o(i.tcp_echoserver_init) refers to tcp.o(i.tcp_listen_with_backlog) for tcp_listen_with_backlog
    tcpserver.o(i.tcp_echoserver_init) refers to tcp.o(i.tcp_accept) for tcp_accept
    tcpserver.o(i.tcp_echoserver_init) refers to tcpserver.o(.data) for tcp_echoserver_pcb
    tcpserver.o(i.tcp_echoserver_init) refers to ip_addr.o(.constdata) for ip_addr_any
    tcpserver.o(i.tcp_echoserver_init) refers to tcpserver.o(i.tcp_echoserver_accept) for tcp_echoserver_accept
    tcpserver.o(i.tcp_echoserver_poll) refers to printf3.o(i.__0printf$3) for __2printf
    tcpserver.o(i.tcp_echoserver_poll) refers to tcpserver.o(i.tcp_echoserver_send) for tcp_echoserver_send
    tcpserver.o(i.tcp_echoserver_poll) refers to tcpserver.o(i.tcp_echoserver_connection_close) for tcp_echoserver_connection_close
    tcpserver.o(i.tcp_echoserver_poll) refers to tcp.o(i.tcp_abandon) for tcp_abandon
    tcpserver.o(i.tcp_echoserver_poll) refers to tcpserver.o(.constdata) for __FUNCTION__
    tcpserver.o(i.tcp_echoserver_recv) refers to printf3.o(i.__0printf$3) for __2printf
    tcpserver.o(i.tcp_echoserver_recv) refers to tcpserver.o(i.tcp_echoserver_connection_close) for tcp_echoserver_connection_close
    tcpserver.o(i.tcp_echoserver_recv) refers to tcp.o(i.tcp_sent) for tcp_sent
    tcpserver.o(i.tcp_echoserver_recv) refers to tcpserver.o(i.tcp_echoserver_send) for tcp_echoserver_send
    tcpserver.o(i.tcp_echoserver_recv) refers to pbuf.o(i.pbuf_free) for pbuf_free
    tcpserver.o(i.tcp_echoserver_recv) refers to pbuf.o(i.pbuf_chain) for pbuf_chain
    tcpserver.o(i.tcp_echoserver_recv) refers to tcp.o(i.tcp_recved) for tcp_recved
    tcpserver.o(i.tcp_echoserver_recv) refers to tcpserver.o(.constdata) for __FUNCTION__
    tcpserver.o(i.tcp_echoserver_recv) refers to tcpserver.o(i.tcp_echoserver_sent) for tcp_echoserver_sent
    tcpserver.o(i.tcp_echoserver_recv) refers to tcpserver.o(.data) for TcpServer_len
    tcpserver.o(i.tcp_echoserver_recv) refers to tcpserver.o(.bss) for TcpServer_buff
    tcpserver.o(i.tcp_echoserver_send) refers to pbuf.o(i.pbuf_ref) for pbuf_ref
    tcpserver.o(i.tcp_echoserver_send) refers to pbuf.o(i.pbuf_free) for pbuf_free
    tcpserver.o(i.tcp_echoserver_send) refers to tcp.o(i.tcp_recved) for tcp_recved
    tcpserver.o(i.tcp_echoserver_sent) refers to tcpserver.o(i.tcp_echoserver_send) for tcp_echoserver_send
    tcpserver.o(i.tcp_echoserver_sent) refers to tcpserver.o(i.tcp_echoserver_connection_close) for tcp_echoserver_connection_close
    printf.o(i.fgetc) refers to stm32f10x_usart.o(i.USART_GetFlagStatus) for USART_GetFlagStatus
    printf.o(i.fgetc) refers to stm32f10x_usart.o(i.USART_ReceiveData) for USART_ReceiveData
    printf.o(i.fputc) refers to stm32f10x_usart.o(i.USART_GetFlagStatus) for USART_GetFlagStatus
    printf.o(i.fputc) refers to stm32f10x_usart.o(i.USART_SendData) for USART_SendData
    usart1.o(i.USART1_IRQHandler) refers to stm32f10x_usart.o(i.USART_GetITStatus) for USART_GetITStatus
    usart1.o(i.USART1_IRQHandler) refers to stm32f10x_usart.o(i.USART_ReceiveData) for USART_ReceiveData
    usart1.o(i.USART1_IRQHandler) refers to stm32f10x_usart.o(i.USART_ClearITPendingBit) for USART_ClearITPendingBit
    usart1.o(i.USART1_IRQHandler) refers to stm32f10x_usart.o(i.USART_GetFlagStatus) for USART_GetFlagStatus
    usart1.o(i.USART1_IRQHandler) refers to stm32f10x_usart.o(i.USART_ClearFlag) for USART_ClearFlag
    usart1.o(i.USART1_IRQHandler) refers to usart1.o(.data) for RX_SIZ
    usart1.o(i.USART1_IRQHandler) refers to usart1.o(.bss) for RX_BUFF
    usart1.o(i.usart1_Configuration) refers to stm32f10x_rcc.o(i.RCC_APB2PeriphClockCmd) for RCC_APB2PeriphClockCmd
    usart1.o(i.usart1_Configuration) refers to stm32f10x_gpio.o(i.GPIO_PinRemapConfig) for GPIO_PinRemapConfig
    usart1.o(i.usart1_Configuration) refers to stm32f10x_gpio.o(i.GPIO_Init) for GPIO_Init
    usart1.o(i.usart1_Configuration) refers to stm32f10x_usart.o(i.USART_Init) for USART_Init
    usart1.o(i.usart1_Configuration) refers to misc.o(i.NVIC_Init) for NVIC_Init
    usart1.o(i.usart1_Configuration) refers to stm32f10x_usart.o(i.USART_ITConfig) for USART_ITConfig
    usart1.o(i.usart1_Configuration) refers to stm32f10x_usart.o(i.USART_Cmd) for USART_Cmd
    usart1.o(i.usart1_Configuration) refers to stm32f10x_usart.o(i.USART_ClearFlag) for USART_ClearFlag
    usart1.o(i.usart1_Configuration) refers to usart1.o(.data) for RX_SIZ
    usart1.o(i.usart1_FreeBuff) refers to delay.o(i.delay_ms) for delay_ms
    usart1.o(i.usart1_FreeBuff) refers to usart1.o(.data) for RX_SIZ
    usart1.o(i.usart1_FreeBuff) refers to usart1.o(.bss) for RX_BUFF
    usart1.o(i.usart1_Receive) refers to delay.o(i.delay_ms) for delay_ms
    usart1.o(i.usart1_Receive) refers to usart1.o(.data) for RX_SIZ
    usart1.o(i.usart1_Receive) refers to usart1.o(.bss) for RX_BUFF
    usart1.o(i.usart1_Send) refers to stm32f10x_usart.o(i.USART_GetFlagStatus) for USART_GetFlagStatus
    usart1.o(i.usart1_Send) refers to stm32f10x_usart.o(i.USART_SendData) for USART_SendData
    usart1.o(i.usart1_Send) refers to stm32f10x_usart.o(i.USART_ClearITPendingBit) for USART_ClearITPendingBit
    delay.o(i.SysTick_Handler) refers to os_core.o(i.OSIntEnter) for OSIntEnter
    delay.o(i.SysTick_Handler) refers to os_core.o(i.OSTimeTick) for OSTimeTick
    delay.o(i.SysTick_Handler) refers to os_core.o(i.OSIntExit) for OSIntExit
    delay.o(i.delay_init) refers to misc.o(i.SysTick_CLKSourceConfig) for SysTick_CLKSourceConfig
    delay.o(i.delay_init) refers to system_stm32f10x.o(.data) for SystemCoreClock
    delay.o(i.delay_init) refers to delay.o(.data) for fac_us
    delay.o(i.delay_ms) refers to os_time.o(i.OSTimeDly) for OSTimeDly
    delay.o(i.delay_ms) refers to delay.o(i.delay_us) for delay_us
    delay.o(i.delay_ms) refers to os_core.o(.data) for OSRunning
    delay.o(i.delay_ms) refers to delay.o(.data) for fac_ms
    delay.o(i.delay_s) refers to delay.o(i.delay_ms) for delay_ms
    delay.o(i.delay_us) refers to delay.o(.data) for fac_us
    stm32f10x_it.o(i.BusFault_Handler) refers to printf3.o(i.__0printf$3) for __2printf
    stm32f10x_it.o(i.ETH_IRQHandler) refers to os_core.o(i.OSIntEnter) for OSIntEnter
    stm32f10x_it.o(i.ETH_IRQHandler) refers to netconf.o(i.LwIP_Pkt_Handle) for LwIP_Pkt_Handle
    stm32f10x_it.o(i.ETH_IRQHandler) refers to stm32_eth.o(i.ETH_GetRxPktSize) for ETH_GetRxPktSize
    stm32f10x_it.o(i.ETH_IRQHandler) refers to stm32_eth.o(i.ETH_DMAClearITPendingBit) for ETH_DMAClearITPendingBit
    stm32f10x_it.o(i.ETH_IRQHandler) refers to os_core.o(i.OSIntExit) for OSIntExit
    stm32f10x_it.o(i.HardFault_Handler) refers to printf3.o(i.__0printf$3) for __2printf
    stm32f10x_it.o(i.MemManage_Handler) refers to printf3.o(i.__0printf$3) for __2printf
    stm32f10x_it.o(i.UsageFault_Handler) refers to printf3.o(i.__0printf$3) for __2printf
    stm32_config.o(i.SoftReset) refers to delay.o(i.delay_s) for delay_s
    os_core.o(i.OSInit) refers to os_cpu_c.o(i.OSInitHookBegin) for OSInitHookBegin
    os_core.o(i.OSInit) refers to os_core.o(i.OS_InitMisc) for OS_InitMisc
    os_core.o(i.OSInit) refers to os_core.o(i.OS_InitRdyList) for OS_InitRdyList
    os_core.o(i.OSInit) refers to os_core.o(i.OS_InitTCBList) for OS_InitTCBList
    os_core.o(i.OSInit) refers to os_core.o(i.OS_InitEventList) for OS_InitEventList
    os_core.o(i.OSInit) refers to os_flag.o(i.OS_FlagInit) for OS_FlagInit
    os_core.o(i.OSInit) refers to os_q.o(i.OS_QInit) for OS_QInit
    os_core.o(i.OSInit) refers to os_core.o(i.OS_InitTaskIdle) for OS_InitTaskIdle
    os_core.o(i.OSInit) refers to os_core.o(i.OS_InitTaskStat) for OS_InitTaskStat
    os_core.o(i.OSInit) refers to os_cpu_c.o(i.OSInitHookEnd) for OSInitHookEnd
    os_core.o(i.OSIntEnter) refers to os_core.o(.data) for OSRunning
    os_core.o(i.OSIntExit) refers to os_cpu_a.o(.text) for OS_CPU_SR_Save
    os_core.o(i.OSIntExit) refers to os_core.o(i.OS_SchedNew) for OS_SchedNew
    os_core.o(i.OSIntExit) refers to os_core.o(.data) for OSRunning
    os_core.o(i.OSIntExit) refers to os_core.o(.bss) for OSTCBPrioTbl
    os_core.o(i.OSSchedLock) refers to os_cpu_a.o(.text) for OS_CPU_SR_Save
    os_core.o(i.OSSchedLock) refers to os_core.o(.data) for OSRunning
    os_core.o(i.OSSchedUnlock) refers to os_cpu_a.o(.text) for OS_CPU_SR_Save
    os_core.o(i.OSSchedUnlock) refers to os_core.o(i.OS_Sched) for OS_Sched
    os_core.o(i.OSSchedUnlock) refers to os_core.o(.data) for OSRunning
    os_core.o(i.OSStart) refers to os_core.o(i.OS_SchedNew) for OS_SchedNew
    os_core.o(i.OSStart) refers to os_cpu_a.o(.text) for OSStartHighRdy
    os_core.o(i.OSStart) refers to os_core.o(.data) for OSRunning
    os_core.o(i.OSStart) refers to os_core.o(.bss) for OSTCBPrioTbl
    os_core.o(i.OSStatInit) refers to os_time.o(i.OSTimeDly) for OSTimeDly
    os_core.o(i.OSStatInit) refers to os_cpu_a.o(.text) for OS_CPU_SR_Save
    os_core.o(i.OSStatInit) refers to os_core.o(.data) for OSIdleCtr
    os_core.o(i.OSTimeTick) refers to os_cpu_c.o(i.OSTimeTickHook) for OSTimeTickHook
    os_core.o(i.OSTimeTick) refers to os_cpu_a.o(.text) for OS_CPU_SR_Save
    os_core.o(i.OSTimeTick) refers to os_core.o(.data) for OSTime
    os_core.o(i.OS_EventTaskRdy) refers to os_core.o(i.OS_EventTaskRemove) for OS_EventTaskRemove
    os_core.o(i.OS_EventTaskRdy) refers to os_core.o(.constdata) for OSUnMapTbl
    os_core.o(i.OS_EventTaskRdy) refers to os_core.o(.bss) for OSTCBPrioTbl
    os_core.o(i.OS_EventTaskRdy) refers to os_core.o(.data) for OSRdyGrp
    os_core.o(i.OS_EventTaskWait) refers to os_core.o(.data) for OSTCBCur
    os_core.o(i.OS_InitEventList) refers to os_core.o(i.OS_MemClr) for OS_MemClr
    os_core.o(i.OS_InitEventList) refers to os_core.o(.bss) for OSEventTbl
    os_core.o(i.OS_InitEventList) refers to os_core.o(.data) for OSEventFreeList
    os_core.o(i.OS_InitMisc) refers to os_core.o(.data) for OSTime
    os_core.o(i.OS_InitRdyList) refers to os_core.o(.data) for OSRdyGrp
    os_core.o(i.OS_InitTCBList) refers to os_core.o(i.OS_MemClr) for OS_MemClr
    os_core.o(i.OS_InitTCBList) refers to os_core.o(.bss) for OSTCBTbl
    os_core.o(i.OS_InitTCBList) refers to os_core.o(.data) for OSTCBList
    os_core.o(i.OS_InitTaskIdle) refers to os_task.o(i.OSTaskCreateExt) for OSTaskCreateExt
    os_core.o(i.OS_InitTaskIdle) refers to os_task.o(i.OSTaskNameSet) for OSTaskNameSet
    os_core.o(i.OS_InitTaskIdle) refers to os_core.o(.bss) for OSTaskIdleStk
    os_core.o(i.OS_InitTaskIdle) refers to os_core.o(i.OS_TaskIdle) for OS_TaskIdle
    os_core.o(i.OS_InitTaskStat) refers to os_task.o(i.OSTaskCreateExt) for OSTaskCreateExt
    os_core.o(i.OS_InitTaskStat) refers to os_task.o(i.OSTaskNameSet) for OSTaskNameSet
    os_core.o(i.OS_InitTaskStat) refers to os_core.o(.bss) for OSTaskStatStk
    os_core.o(i.OS_InitTaskStat) refers to os_core.o(i.OS_TaskStat) for OS_TaskStat
    os_core.o(i.OS_Sched) refers to os_cpu_a.o(.text) for OS_CPU_SR_Save
    os_core.o(i.OS_Sched) refers to os_core.o(i.OS_SchedNew) for OS_SchedNew
    os_core.o(i.OS_Sched) refers to os_core.o(.data) for OSIntNesting
    os_core.o(i.OS_Sched) refers to os_core.o(.bss) for OSTCBPrioTbl
    os_core.o(i.OS_SchedNew) refers to os_core.o(.constdata) for OSUnMapTbl
    os_core.o(i.OS_SchedNew) refers to os_core.o(.data) for OSRdyGrp
    os_core.o(i.OS_TCBInit) refers to os_cpu_a.o(.text) for OS_CPU_SR_Save
    os_core.o(i.OS_TCBInit) refers to os_cpu_c.o(i.OSTCBInitHook) for OSTCBInitHook
    os_core.o(i.OS_TCBInit) refers to os_cpu_c.o(i.OSTaskCreateHook) for OSTaskCreateHook
    os_core.o(i.OS_TCBInit) refers to os_core.o(.data) for OSTCBFreeList
    os_core.o(i.OS_TCBInit) refers to os_core.o(.bss) for OSTCBPrioTbl
    os_core.o(i.OS_TaskIdle) refers to os_cpu_a.o(.text) for OS_CPU_SR_Save
    os_core.o(i.OS_TaskIdle) refers to os_cpu_c.o(i.OSTaskIdleHook) for OSTaskIdleHook
    os_core.o(i.OS_TaskIdle) refers to os_core.o(.data) for OSIdleCtr
    os_core.o(i.OS_TaskStat) refers to os_time.o(i.OSTimeDly) for OSTimeDly
    os_core.o(i.OS_TaskStat) refers to os_task.o(i.OSTaskSuspend) for OSTaskSuspend
    os_core.o(i.OS_TaskStat) refers to os_cpu_a.o(.text) for OS_CPU_SR_Save
    os_core.o(i.OS_TaskStat) refers to os_cpu_c.o(i.OSTaskStatHook) for OSTaskStatHook
    os_core.o(i.OS_TaskStat) refers to os_core.o(i.OS_TaskStatStkChk) for OS_TaskStatStkChk
    os_core.o(i.OS_TaskStat) refers to os_core.o(.data) for OSStatRdy
    os_core.o(i.OS_TaskStatStkChk) refers to os_task.o(i.OSTaskStkChk) for OSTaskStkChk
    os_core.o(i.OS_TaskStatStkChk) refers to os_core.o(.bss) for OSTCBPrioTbl
    os_flag.o(i.OSFlagAccept) refers to os_cpu_a.o(.text) for OS_CPU_SR_Save
    os_flag.o(i.OSFlagCreate) refers to os_cpu_a.o(.text) for OS_CPU_SR_Save
    os_flag.o(i.OSFlagCreate) refers to os_core.o(.data) for OSIntNesting
    os_flag.o(i.OSFlagDel) refers to os_cpu_a.o(.text) for OS_CPU_SR_Save
    os_flag.o(i.OSFlagDel) refers to os_flag.o(i.OS_FlagTaskRdy) for OS_FlagTaskRdy
    os_flag.o(i.OSFlagDel) refers to os_core.o(i.OS_Sched) for OS_Sched
    os_flag.o(i.OSFlagDel) refers to os_core.o(.data) for OSIntNesting
    os_flag.o(i.OSFlagNameGet) refers to os_cpu_a.o(.text) for OS_CPU_SR_Save
    os_flag.o(i.OSFlagNameGet) refers to os_core.o(i.OS_StrLen) for OS_StrLen
    os_flag.o(i.OSFlagNameGet) refers to os_core.o(.data) for OSIntNesting
    os_flag.o(i.OSFlagNameSet) refers to os_cpu_a.o(.text) for OS_CPU_SR_Save
    os_flag.o(i.OSFlagNameSet) refers to os_core.o(.data) for OSIntNesting
    os_flag.o(i.OSFlagPend) refers to os_cpu_a.o(.text) for OS_CPU_SR_Save
    os_flag.o(i.OSFlagPend) refers to os_flag.o(i.OS_FlagBlock) for OS_FlagBlock
    os_flag.o(i.OSFlagPend) refers to os_core.o(i.OS_Sched) for OS_Sched
    os_flag.o(i.OSFlagPend) refers to os_flag.o(i.OS_FlagUnlink) for OS_FlagUnlink
    os_flag.o(i.OSFlagPend) refers to os_core.o(.data) for OSIntNesting
    os_flag.o(i.OSFlagPendGetFlagsRdy) refers to os_cpu_a.o(.text) for OS_CPU_SR_Save
    os_flag.o(i.OSFlagPendGetFlagsRdy) refers to os_core.o(.data) for OSTCBCur
    os_flag.o(i.OSFlagPost) refers to os_cpu_a.o(.text) for OS_CPU_SR_Save
    os_flag.o(i.OSFlagPost) refers to os_flag.o(i.OS_FlagTaskRdy) for OS_FlagTaskRdy
    os_flag.o(i.OSFlagPost) refers to os_core.o(i.OS_Sched) for OS_Sched
    os_flag.o(i.OSFlagQuery) refers to os_cpu_a.o(.text) for OS_CPU_SR_Save
    os_flag.o(i.OS_FlagBlock) refers to os_core.o(.data) for OSTCBCur
    os_flag.o(i.OS_FlagInit) refers to os_core.o(i.OS_MemClr) for OS_MemClr
    os_flag.o(i.OS_FlagInit) refers to os_core.o(.bss) for OSFlagTbl
    os_flag.o(i.OS_FlagInit) refers to os_core.o(.data) for OSFlagFreeList
    os_flag.o(i.OS_FlagTaskRdy) refers to os_flag.o(i.OS_FlagUnlink) for OS_FlagUnlink
    os_flag.o(i.OS_FlagTaskRdy) refers to os_core.o(.data) for OSRdyGrp
    os_mbox.o(i.OSMboxAccept) refers to os_cpu_a.o(.text) for OS_CPU_SR_Save
    os_mbox.o(i.OSMboxCreate) refers to os_cpu_a.o(.text) for OS_CPU_SR_Save
    os_mbox.o(i.OSMboxCreate) refers to os_core.o(i.OS_EventWaitListInit) for OS_EventWaitListInit
    os_mbox.o(i.OSMboxCreate) refers to os_core.o(.data) for OSIntNesting
    os_mbox.o(i.OSMboxDel) refers to os_cpu_a.o(.text) for OS_CPU_SR_Save
    os_mbox.o(i.OSMboxDel) refers to os_core.o(i.OS_EventTaskRdy) for OS_EventTaskRdy
    os_mbox.o(i.OSMboxDel) refers to os_core.o(i.OS_Sched) for OS_Sched
    os_mbox.o(i.OSMboxDel) refers to os_core.o(.data) for OSIntNesting
    os_mbox.o(i.OSMboxPend) refers to os_cpu_a.o(.text) for OS_CPU_SR_Save
    os_mbox.o(i.OSMboxPend) refers to os_core.o(i.OS_EventTaskWait) for OS_EventTaskWait
    os_mbox.o(i.OSMboxPend) refers to os_core.o(i.OS_Sched) for OS_Sched
    os_mbox.o(i.OSMboxPend) refers to os_core.o(i.OS_EventTaskRemove) for OS_EventTaskRemove
    os_mbox.o(i.OSMboxPend) refers to os_core.o(.data) for OSIntNesting
    os_mbox.o(i.OSMboxPendAbort) refers to os_cpu_a.o(.text) for OS_CPU_SR_Save
    os_mbox.o(i.OSMboxPendAbort) refers to os_core.o(i.OS_EventTaskRdy) for OS_EventTaskRdy
    os_mbox.o(i.OSMboxPendAbort) refers to os_core.o(i.OS_Sched) for OS_Sched
    os_mbox.o(i.OSMboxPost) refers to os_cpu_a.o(.text) for OS_CPU_SR_Save
    os_mbox.o(i.OSMboxPost) refers to os_core.o(i.OS_EventTaskRdy) for OS_EventTaskRdy
    os_mbox.o(i.OSMboxPost) refers to os_core.o(i.OS_Sched) for OS_Sched
    os_mbox.o(i.OSMboxPostOpt) refers to os_cpu_a.o(.text) for OS_CPU_SR_Save
    os_mbox.o(i.OSMboxPostOpt) refers to os_core.o(i.OS_EventTaskRdy) for OS_EventTaskRdy
    os_mbox.o(i.OSMboxPostOpt) refers to os_core.o(i.OS_Sched) for OS_Sched
    os_mbox.o(i.OSMboxQuery) refers to os_cpu_a.o(.text) for OS_CPU_SR_Save
    os_mutex.o(i.OSMutexAccept) refers to os_cpu_a.o(.text) for OS_CPU_SR_Save
    os_mutex.o(i.OSMutexAccept) refers to os_core.o(.data) for OSIntNesting
    os_mutex.o(i.OSMutexCreate) refers to os_cpu_a.o(.text) for OS_CPU_SR_Save
    os_mutex.o(i.OSMutexCreate) refers to os_core.o(i.OS_EventWaitListInit) for OS_EventWaitListInit
    os_mutex.o(i.OSMutexCreate) refers to os_core.o(.data) for OSIntNesting
    os_mutex.o(i.OSMutexCreate) refers to os_core.o(.bss) for OSTCBPrioTbl
    os_mutex.o(i.OSMutexDel) refers to os_cpu_a.o(.text) for OS_CPU_SR_Save
    os_mutex.o(i.OSMutexDel) refers to os_mutex.o(i.OSMutex_RdyAtPrio) for OSMutex_RdyAtPrio
    os_mutex.o(i.OSMutexDel) refers to os_core.o(i.OS_EventTaskRdy) for OS_EventTaskRdy
    os_mutex.o(i.OSMutexDel) refers to os_core.o(i.OS_Sched) for OS_Sched
    os_mutex.o(i.OSMutexDel) refers to os_core.o(.data) for OSIntNesting
    os_mutex.o(i.OSMutexDel) refers to os_core.o(.bss) for OSTCBPrioTbl
    os_mutex.o(i.OSMutexPend) refers to os_cpu_a.o(.text) for OS_CPU_SR_Save
    os_mutex.o(i.OSMutexPend) refers to os_core.o(i.OS_EventTaskWait) for OS_EventTaskWait
    os_mutex.o(i.OSMutexPend) refers to os_core.o(i.OS_Sched) for OS_Sched
    os_mutex.o(i.OSMutexPend) refers to os_core.o(i.OS_EventTaskRemove) for OS_EventTaskRemove
    os_mutex.o(i.OSMutexPend) refers to os_core.o(.data) for OSIntNesting
    os_mutex.o(i.OSMutexPend) refers to os_core.o(.bss) for OSTCBPrioTbl
    os_mutex.o(i.OSMutexPost) refers to os_cpu_a.o(.text) for OS_CPU_SR_Save
    os_mutex.o(i.OSMutexPost) refers to os_mutex.o(i.OSMutex_RdyAtPrio) for OSMutex_RdyAtPrio
    os_mutex.o(i.OSMutexPost) refers to os_core.o(i.OS_EventTaskRdy) for OS_EventTaskRdy
    os_mutex.o(i.OSMutexPost) refers to os_core.o(i.OS_Sched) for OS_Sched
    os_mutex.o(i.OSMutexPost) refers to os_core.o(.data) for OSIntNesting
    os_mutex.o(i.OSMutexPost) refers to os_core.o(.bss) for OSTCBPrioTbl
    os_mutex.o(i.OSMutexQuery) refers to os_cpu_a.o(.text) for OS_CPU_SR_Save
    os_mutex.o(i.OSMutexQuery) refers to os_core.o(.data) for OSIntNesting
    os_mutex.o(i.OSMutex_RdyAtPrio) refers to os_core.o(.data) for OSRdyTbl
    os_mutex.o(i.OSMutex_RdyAtPrio) refers to os_core.o(.bss) for OSTCBPrioTbl
    os_q.o(i.OSQAccept) refers to os_cpu_a.o(.text) for OS_CPU_SR_Save
    os_q.o(i.OSQCreate) refers to os_cpu_a.o(.text) for OS_CPU_SR_Save
    os_q.o(i.OSQCreate) refers to os_core.o(i.OS_EventWaitListInit) for OS_EventWaitListInit
    os_q.o(i.OSQCreate) refers to os_core.o(.data) for OSIntNesting
    os_q.o(i.OSQDel) refers to os_cpu_a.o(.text) for OS_CPU_SR_Save
    os_q.o(i.OSQDel) refers to os_core.o(i.OS_EventTaskRdy) for OS_EventTaskRdy
    os_q.o(i.OSQDel) refers to os_core.o(i.OS_Sched) for OS_Sched
    os_q.o(i.OSQDel) refers to os_core.o(.data) for OSIntNesting
    os_q.o(i.OSQFlush) refers to os_cpu_a.o(.text) for OS_CPU_SR_Save
    os_q.o(i.OSQPend) refers to os_cpu_a.o(.text) for OS_CPU_SR_Save
    os_q.o(i.OSQPend) refers to os_core.o(i.OS_EventTaskWait) for OS_EventTaskWait
    os_q.o(i.OSQPend) refers to os_core.o(i.OS_Sched) for OS_Sched
    os_q.o(i.OSQPend) refers to os_core.o(i.OS_EventTaskRemove) for OS_EventTaskRemove
    os_q.o(i.OSQPend) refers to os_core.o(.data) for OSIntNesting
    os_q.o(i.OSQPendAbort) refers to os_cpu_a.o(.text) for OS_CPU_SR_Save
    os_q.o(i.OSQPendAbort) refers to os_core.o(i.OS_EventTaskRdy) for OS_EventTaskRdy
    os_q.o(i.OSQPendAbort) refers to os_core.o(i.OS_Sched) for OS_Sched
    os_q.o(i.OSQPost) refers to os_cpu_a.o(.text) for OS_CPU_SR_Save
    os_q.o(i.OSQPost) refers to os_core.o(i.OS_EventTaskRdy) for OS_EventTaskRdy
    os_q.o(i.OSQPost) refers to os_core.o(i.OS_Sched) for OS_Sched
    os_q.o(i.OSQPostFront) refers to os_cpu_a.o(.text) for OS_CPU_SR_Save
    os_q.o(i.OSQPostFront) refers to os_core.o(i.OS_EventTaskRdy) for OS_EventTaskRdy
    os_q.o(i.OSQPostFront) refers to os_core.o(i.OS_Sched) for OS_Sched
    os_q.o(i.OSQPostOpt) refers to os_cpu_a.o(.text) for OS_CPU_SR_Save
    os_q.o(i.OSQPostOpt) refers to os_core.o(i.OS_EventTaskRdy) for OS_EventTaskRdy
    os_q.o(i.OSQPostOpt) refers to os_core.o(i.OS_Sched) for OS_Sched
    os_q.o(i.OSQQuery) refers to os_cpu_a.o(.text) for OS_CPU_SR_Save
    os_q.o(i.OS_QInit) refers to os_core.o(i.OS_MemClr) for OS_MemClr
    os_q.o(i.OS_QInit) refers to os_core.o(.bss) for OSQTbl
    os_q.o(i.OS_QInit) refers to os_core.o(.data) for OSQFreeList
    os_sem.o(i.OSSemAccept) refers to os_cpu_a.o(.text) for OS_CPU_SR_Save
    os_sem.o(i.OSSemCreate) refers to os_cpu_a.o(.text) for OS_CPU_SR_Save
    os_sem.o(i.OSSemCreate) refers to os_core.o(i.OS_EventWaitListInit) for OS_EventWaitListInit
    os_sem.o(i.OSSemCreate) refers to os_core.o(.data) for OSIntNesting
    os_sem.o(i.OSSemDel) refers to os_cpu_a.o(.text) for OS_CPU_SR_Save
    os_sem.o(i.OSSemDel) refers to os_core.o(i.OS_EventTaskRdy) for OS_EventTaskRdy
    os_sem.o(i.OSSemDel) refers to os_core.o(i.OS_Sched) for OS_Sched
    os_sem.o(i.OSSemDel) refers to os_core.o(.data) for OSIntNesting
    os_sem.o(i.OSSemPend) refers to os_cpu_a.o(.text) for OS_CPU_SR_Save
    os_sem.o(i.OSSemPend) refers to os_core.o(i.OS_EventTaskWait) for OS_EventTaskWait
    os_sem.o(i.OSSemPend) refers to os_core.o(i.OS_Sched) for OS_Sched
    os_sem.o(i.OSSemPend) refers to os_core.o(i.OS_EventTaskRemove) for OS_EventTaskRemove
    os_sem.o(i.OSSemPend) refers to os_core.o(.data) for OSIntNesting
    os_sem.o(i.OSSemPendAbort) refers to os_cpu_a.o(.text) for OS_CPU_SR_Save
    os_sem.o(i.OSSemPendAbort) refers to os_core.o(i.OS_EventTaskRdy) for OS_EventTaskRdy
    os_sem.o(i.OSSemPendAbort) refers to os_core.o(i.OS_Sched) for OS_Sched
    os_sem.o(i.OSSemPost) refers to os_cpu_a.o(.text) for OS_CPU_SR_Save
    os_sem.o(i.OSSemPost) refers to os_core.o(i.OS_EventTaskRdy) for OS_EventTaskRdy
    os_sem.o(i.OSSemPost) refers to os_core.o(i.OS_Sched) for OS_Sched
    os_sem.o(i.OSSemQuery) refers to os_cpu_a.o(.text) for OS_CPU_SR_Save
    os_sem.o(i.OSSemSet) refers to os_cpu_a.o(.text) for OS_CPU_SR_Save
    os_task.o(i.OSTaskChangePrio) refers to os_cpu_a.o(.text) for OS_CPU_SR_Save
    os_task.o(i.OSTaskChangePrio) refers to os_core.o(i.OS_Sched) for OS_Sched
    os_task.o(i.OSTaskChangePrio) refers to os_core.o(.bss) for OSTCBPrioTbl
    os_task.o(i.OSTaskChangePrio) refers to os_core.o(.data) for OSTCBCur
    os_task.o(i.OSTaskCreate) refers to os_cpu_a.o(.text) for OS_CPU_SR_Save
    os_task.o(i.OSTaskCreate) refers to os_cpu_c.o(i.OSTaskStkInit) for OSTaskStkInit
    os_task.o(i.OSTaskCreate) refers to os_core.o(i.OS_TCBInit) for OS_TCBInit
    os_task.o(i.OSTaskCreate) refers to os_core.o(i.OS_Sched) for OS_Sched
    os_task.o(i.OSTaskCreate) refers to os_core.o(.data) for OSIntNesting
    os_task.o(i.OSTaskCreate) refers to os_core.o(.bss) for OSTCBPrioTbl
    os_task.o(i.OSTaskCreateExt) refers to os_cpu_a.o(.text) for OS_CPU_SR_Save
    os_task.o(i.OSTaskCreateExt) refers to os_task.o(i.OS_TaskStkClr) for OS_TaskStkClr
    os_task.o(i.OSTaskCreateExt) refers to os_cpu_c.o(i.OSTaskStkInit) for OSTaskStkInit
    os_task.o(i.OSTaskCreateExt) refers to os_core.o(i.OS_TCBInit) for OS_TCBInit
    os_task.o(i.OSTaskCreateExt) refers to os_core.o(i.OS_Sched) for OS_Sched
    os_task.o(i.OSTaskCreateExt) refers to os_core.o(.data) for OSIntNesting
    os_task.o(i.OSTaskCreateExt) refers to os_core.o(.bss) for OSTCBPrioTbl
    os_task.o(i.OSTaskDel) refers to os_cpu_a.o(.text) for OS_CPU_SR_Save
    os_task.o(i.OSTaskDel) refers to os_core.o(i.OS_EventTaskRemove) for OS_EventTaskRemove
    os_task.o(i.OSTaskDel) refers to os_flag.o(i.OS_FlagUnlink) for OS_FlagUnlink
    os_task.o(i.OSTaskDel) refers to os_core.o(i.OS_Dummy) for OS_Dummy
    os_task.o(i.OSTaskDel) refers to os_cpu_c.o(i.OSTaskDelHook) for OSTaskDelHook
    os_task.o(i.OSTaskDel) refers to os_core.o(i.OS_Sched) for OS_Sched
    os_task.o(i.OSTaskDel) refers to os_core.o(.data) for OSIntNesting
    os_task.o(i.OSTaskDel) refers to os_core.o(.bss) for OSTCBPrioTbl
    os_task.o(i.OSTaskDelReq) refers to os_cpu_a.o(.text) for OS_CPU_SR_Save
    os_task.o(i.OSTaskDelReq) refers to os_core.o(.data) for OSTCBCur
    os_task.o(i.OSTaskDelReq) refers to os_core.o(.bss) for OSTCBPrioTbl
    os_task.o(i.OSTaskNameGet) refers to os_cpu_a.o(.text) for OS_CPU_SR_Save
    os_task.o(i.OSTaskNameGet) refers to os_core.o(i.OS_StrLen) for OS_StrLen
    os_task.o(i.OSTaskNameGet) refers to os_core.o(.data) for OSIntNesting
    os_task.o(i.OSTaskNameGet) refers to os_core.o(.bss) for OSTCBPrioTbl
    os_task.o(i.OSTaskNameSet) refers to os_cpu_a.o(.text) for OS_CPU_SR_Save
    os_task.o(i.OSTaskNameSet) refers to os_core.o(.data) for OSIntNesting
    os_task.o(i.OSTaskNameSet) refers to os_core.o(.bss) for OSTCBPrioTbl
    os_task.o(i.OSTaskQuery) refers to os_cpu_a.o(.text) for OS_CPU_SR_Save
    os_task.o(i.OSTaskQuery) refers to os_core.o(i.OS_MemCopy) for OS_MemCopy
    os_task.o(i.OSTaskQuery) refers to os_core.o(.data) for OSTCBCur
    os_task.o(i.OSTaskQuery) refers to os_core.o(.bss) for OSTCBPrioTbl
    os_task.o(i.OSTaskRegGet) refers to os_cpu_a.o(.text) for OS_CPU_SR_Save
    os_task.o(i.OSTaskRegGet) refers to os_core.o(.data) for OSTCBCur
    os_task.o(i.OSTaskRegGet) refers to os_core.o(.bss) for OSTCBPrioTbl
    os_task.o(i.OSTaskRegSet) refers to os_cpu_a.o(.text) for OS_CPU_SR_Save
    os_task.o(i.OSTaskRegSet) refers to os_core.o(.data) for OSTCBCur
    os_task.o(i.OSTaskRegSet) refers to os_core.o(.bss) for OSTCBPrioTbl
    os_task.o(i.OSTaskResume) refers to os_cpu_a.o(.text) for OS_CPU_SR_Save
    os_task.o(i.OSTaskResume) refers to os_core.o(i.OS_Sched) for OS_Sched
    os_task.o(i.OSTaskResume) refers to os_core.o(.bss) for OSTCBPrioTbl
    os_task.o(i.OSTaskResume) refers to os_core.o(.data) for OSRdyGrp
    os_task.o(i.OSTaskStkChk) refers to os_cpu_a.o(.text) for OS_CPU_SR_Save
    os_task.o(i.OSTaskStkChk) refers to os_core.o(.data) for OSTCBCur
    os_task.o(i.OSTaskStkChk) refers to os_core.o(.bss) for OSTCBPrioTbl
    os_task.o(i.OSTaskSuspend) refers to os_cpu_a.o(.text) for OS_CPU_SR_Save
    os_task.o(i.OSTaskSuspend) refers to os_core.o(i.OS_Sched) for OS_Sched
    os_task.o(i.OSTaskSuspend) refers to os_core.o(.data) for OSTCBCur
    os_task.o(i.OSTaskSuspend) refers to os_core.o(.bss) for OSTCBPrioTbl
    os_task.o(i.OS_TaskReturn) refers to os_cpu_c.o(i.OSTaskReturnHook) for OSTaskReturnHook
    os_task.o(i.OS_TaskReturn) refers to os_task.o(i.OSTaskDel) for OSTaskDel
    os_task.o(i.OS_TaskReturn) refers to os_core.o(.data) for OSTCBCur
    os_time.o(i.OSTimeDly) refers to os_cpu_a.o(.text) for OS_CPU_SR_Save
    os_time.o(i.OSTimeDly) refers to os_core.o(i.OS_Sched) for OS_Sched
    os_time.o(i.OSTimeDly) refers to os_core.o(.data) for OSIntNesting
    os_time.o(i.OSTimeDlyHMSM) refers to os_time.o(i.OSTimeDly) for OSTimeDly
    os_time.o(i.OSTimeDlyHMSM) refers to os_core.o(.data) for OSIntNesting
    os_time.o(i.OSTimeDlyResume) refers to os_cpu_a.o(.text) for OS_CPU_SR_Save
    os_time.o(i.OSTimeDlyResume) refers to os_core.o(i.OS_Sched) for OS_Sched
    os_time.o(i.OSTimeDlyResume) refers to os_core.o(.bss) for OSTCBPrioTbl
    os_time.o(i.OSTimeDlyResume) refers to os_core.o(.data) for OSRdyGrp
    os_time.o(i.OSTimeGet) refers to os_cpu_a.o(.text) for OS_CPU_SR_Save
    os_time.o(i.OSTimeGet) refers to os_core.o(.data) for OSTime
    os_time.o(i.OSTimeSet) refers to os_cpu_a.o(.text) for OS_CPU_SR_Save
    os_time.o(i.OSTimeSet) refers to os_core.o(.data) for OSTime
    os_cpu_a.o(.text) refers to os_core.o(.data) for OSRunning
    os_cpu_a.o(.text) refers to os_cpu_c.o(i.OSTaskSwHook) for OSTaskSwHook
    ethernetif.o(i.ETH_GetCurrentTxBuffer) refers to stm32_eth.o(.data) for DMATxDescToSet
    ethernetif.o(i.ETH_RxPkt_ChainMode) refers to stm32_eth.o(.data) for DMARxDescToGet
    ethernetif.o(i.ETH_TxPkt_ChainMode) refers to stm32_eth.o(.data) for DMATxDescToSet
    ethernetif.o(i.Set_MAC_Address) refers to stm32_eth.o(i.ETH_MACAddressConfig) for ETH_MACAddressConfig
    ethernetif.o(i.Set_MAC_Address) refers to ethernetif.o(.data) for MACaddr
    ethernetif.o(i.ethernetif_init) refers to mem.o(i.mem_malloc) for mem_malloc
    ethernetif.o(i.ethernetif_init) refers to ethernetif.o(i.low_level_init) for low_level_init
    ethernetif.o(i.ethernetif_init) refers to etharp.o(i.etharp_output) for etharp_output
    ethernetif.o(i.ethernetif_init) refers to ethernetif.o(i.low_level_output) for low_level_output
    ethernetif.o(i.ethernetif_input) refers to ethernetif.o(i.low_level_input) for low_level_input
    ethernetif.o(i.ethernetif_input) refers to pbuf.o(i.pbuf_free) for pbuf_free
    ethernetif.o(i.low_level_init) refers to stm32_eth.o(i.ETH_DMATxDescChainInit) for ETH_DMATxDescChainInit
    ethernetif.o(i.low_level_init) refers to stm32_eth.o(i.ETH_DMARxDescChainInit) for ETH_DMARxDescChainInit
    ethernetif.o(i.low_level_init) refers to stm32_eth.o(i.ETH_DMARxDescReceiveITConfig) for ETH_DMARxDescReceiveITConfig
    ethernetif.o(i.low_level_init) refers to stm32_eth.o(i.ETH_DMATxDescChecksumInsertionConfig) for ETH_DMATxDescChecksumInsertionConfig
    ethernetif.o(i.low_level_init) refers to stm32_eth.o(i.ETH_Start) for ETH_Start
    ethernetif.o(i.low_level_init) refers to ethernetif.o(.data) for MACaddr
    ethernetif.o(i.low_level_init) refers to ethernetif.o(.bss) for Tx_Buff
    ethernetif.o(i.low_level_input) refers to ethernetif.o(i.ETH_RxPkt_ChainMode) for ETH_RxPkt_ChainMode
    ethernetif.o(i.low_level_input) refers to pbuf.o(i.pbuf_alloc) for pbuf_alloc
    ethernetif.o(i.low_level_input) refers to memcpya.o(.text) for __aeabi_memcpy
    ethernetif.o(i.low_level_output) refers to ethernetif.o(i.ETH_GetCurrentTxBuffer) for ETH_GetCurrentTxBuffer
    ethernetif.o(i.low_level_output) refers to memcpya.o(.text) for __aeabi_memcpy
    ethernetif.o(i.low_level_output) refers to ethernetif.o(i.ETH_TxPkt_ChainMode) for ETH_TxPkt_ChainMode
    ethernetif.o(.data) refers to ethernetif.o(.bss) for DMATxDscrTab
    init.o(i.lwip_init) refers to mem.o(i.mem_init) for mem_init
    init.o(i.lwip_init) refers to memp.o(i.memp_init) for memp_init
    mem.o(i.mem_calloc) refers to mem.o(i.mem_malloc) for mem_malloc
    mem.o(i.mem_calloc) refers to memseta.o(.text) for __aeabi_memclr
    mem.o(i.mem_free) refers to mem.o(i.plug_holes) for plug_holes
    mem.o(i.mem_free) refers to mem.o(.data) for ram
    mem.o(i.mem_init) refers to mem.o(.bss) for ram_heap
    mem.o(i.mem_init) refers to mem.o(.data) for ram
    mem.o(i.mem_malloc) refers to mem.o(.data) for lfree
    mem.o(i.mem_realloc) refers to mem.o(.data) for ram
    mem.o(i.plug_holes) refers to mem.o(.data) for ram
    memp.o(i.memp_free) refers to memp.o(.bss) for memp_tab
    memp.o(i.memp_init) refers to memp.o(.bss) for memp_memory
    memp.o(i.memp_init) refers to memp.o(.constdata) for memp_sizes
    memp.o(i.memp_malloc) refers to memp.o(.bss) for memp_tab
    netif.o(i.netif_add) refers to netif.o(i.netif_set_addr) for netif_set_addr
    netif.o(i.netif_add) refers to netif.o(.data) for netifnum
    netif.o(i.netif_find) refers to netif.o(.data) for netif_list
    netif.o(i.netif_remove) refers to netif.o(i.netif_set_default) for netif_set_default
    netif.o(i.netif_remove) refers to netif.o(.data) for netif_list
    netif.o(i.netif_set_addr) refers to netif.o(i.netif_set_ipaddr) for netif_set_ipaddr
    netif.o(i.netif_set_addr) refers to netif.o(i.netif_set_netmask) for netif_set_netmask
    netif.o(i.netif_set_addr) refers to netif.o(i.netif_set_gw) for netif_set_gw
    netif.o(i.netif_set_default) refers to netif.o(.data) for netif_default
    netif.o(i.netif_set_ipaddr) refers to tcp.o(i.tcp_abandon) for tcp_abandon
    netif.o(i.netif_set_ipaddr) refers to tcp.o(.data) for tcp_active_pcbs
    netif.o(i.netif_set_up) refers to etharp.o(i.etharp_request) for etharp_request
    pbuf.o(i.pbuf_alloc) refers to memp.o(i.memp_malloc) for memp_malloc
    pbuf.o(i.pbuf_alloc) refers to pbuf.o(i.pbuf_free) for pbuf_free
    pbuf.o(i.pbuf_alloc) refers to mem.o(i.mem_malloc) for mem_malloc
    pbuf.o(i.pbuf_chain) refers to pbuf.o(i.pbuf_cat) for pbuf_cat
    pbuf.o(i.pbuf_chain) refers to pbuf.o(i.pbuf_ref) for pbuf_ref
    pbuf.o(i.pbuf_coalesce) refers to pbuf.o(i.pbuf_alloc) for pbuf_alloc
    pbuf.o(i.pbuf_coalesce) refers to pbuf.o(i.pbuf_copy) for pbuf_copy
    pbuf.o(i.pbuf_coalesce) refers to pbuf.o(i.pbuf_free) for pbuf_free
    pbuf.o(i.pbuf_copy) refers to memcpya.o(.text) for __aeabi_memcpy
    pbuf.o(i.pbuf_copy_partial) refers to memcpya.o(.text) for __aeabi_memcpy
    pbuf.o(i.pbuf_dechain) refers to pbuf.o(i.pbuf_free) for pbuf_free
    pbuf.o(i.pbuf_free) refers to memp.o(i.memp_free) for memp_free
    pbuf.o(i.pbuf_free) refers to mem.o(i.mem_free) for mem_free
    pbuf.o(i.pbuf_realloc) refers to mem.o(i.mem_realloc) for mem_realloc
    pbuf.o(i.pbuf_realloc) refers to pbuf.o(i.pbuf_free) for pbuf_free
    pbuf.o(i.pbuf_take) refers to memcpya.o(.text) for __aeabi_memcpy
    tcp.o(i.tcp_abandon) refers to tcp.o(i.tcp_pcb_remove) for tcp_pcb_remove
    tcp.o(i.tcp_abandon) refers to memp.o(i.memp_free) for memp_free
    tcp.o(i.tcp_abandon) refers to tcp.o(i.tcp_segs_free) for tcp_segs_free
    tcp.o(i.tcp_abandon) refers to tcp_out.o(i.tcp_rst) for tcp_rst
    tcp.o(i.tcp_abandon) refers to tcp.o(.data) for tcp_tw_pcbs
    tcp.o(i.tcp_alloc) refers to memp.o(i.memp_malloc) for memp_malloc
    tcp.o(i.tcp_alloc) refers to tcp.o(i.tcp_kill_timewait) for tcp_kill_timewait
    tcp.o(i.tcp_alloc) refers to tcp.o(i.tcp_kill_prio) for tcp_kill_prio
    tcp.o(i.tcp_alloc) refers to memseta.o(.text) for __aeabi_memclr4
    tcp.o(i.tcp_alloc) refers to tcp.o(i.tcp_next_iss) for tcp_next_iss
    tcp.o(i.tcp_alloc) refers to tcp.o(.data) for tcp_ticks
    tcp.o(i.tcp_alloc) refers to tcp.o(i.tcp_recv_null) for tcp_recv_null
    tcp.o(i.tcp_bind) refers to tcp.o(i.tcp_new_port) for tcp_new_port
    tcp.o(i.tcp_bind) refers to tcp.o(.data) for tcp_listen_pcbs
    tcp.o(i.tcp_close) refers to printf3.o(i.__0printf$3) for __2printf
    tcp.o(i.tcp_close) refers to memp.o(i.memp_free) for memp_free
    tcp.o(i.tcp_close) refers to tcp.o(i.tcp_pcb_remove) for tcp_pcb_remove
    tcp.o(i.tcp_close) refers to tcp_out.o(i.tcp_send_ctrl) for tcp_send_ctrl
    tcp.o(i.tcp_close) refers to tcp_out.o(i.tcp_output) for tcp_output
    tcp.o(i.tcp_close) refers to tcp.o(.constdata) for __FUNCTION__
    tcp.o(i.tcp_close) refers to tcp.o(.data) for tcp_bound_pcbs
    tcp.o(i.tcp_connect) refers to tcp.o(i.tcp_new_port) for tcp_new_port
    tcp.o(i.tcp_connect) refers to tcp.o(i.tcp_next_iss) for tcp_next_iss
    tcp.o(i.tcp_connect) refers to tcp.o(i.tcp_eff_send_mss) for tcp_eff_send_mss
    tcp.o(i.tcp_connect) refers to tcp_out.o(i.tcp_enqueue) for tcp_enqueue
    tcp.o(i.tcp_connect) refers to tcp_out.o(i.tcp_output) for tcp_output
    tcp.o(i.tcp_connect) refers to tcp.o(.data) for tcp_bound_pcbs
    tcp.o(i.tcp_eff_send_mss) refers to ip.o(i.ip_route) for ip_route
    tcp.o(i.tcp_fasttmr) refers to pbuf.o(i.pbuf_free) for pbuf_free
    tcp.o(i.tcp_fasttmr) refers to tcp_out.o(i.tcp_output) for tcp_output
    tcp.o(i.tcp_fasttmr) refers to tcp.o(.data) for tcp_active_pcbs
    tcp.o(i.tcp_kill_prio) refers to tcp.o(i.tcp_abandon) for tcp_abandon
    tcp.o(i.tcp_kill_prio) refers to tcp.o(.data) for tcp_active_pcbs
    tcp.o(i.tcp_kill_timewait) refers to tcp.o(i.tcp_abandon) for tcp_abandon
    tcp.o(i.tcp_kill_timewait) refers to tcp.o(.data) for tcp_tw_pcbs
    tcp.o(i.tcp_listen_with_backlog) refers to memp.o(i.memp_malloc) for memp_malloc
    tcp.o(i.tcp_listen_with_backlog) refers to memp.o(i.memp_free) for memp_free
    tcp.o(i.tcp_listen_with_backlog) refers to tcp.o(.data) for tcp_bound_pcbs
    tcp.o(i.tcp_listen_with_backlog) refers to tcp.o(i.tcp_accept_null) for tcp_accept_null
    tcp.o(i.tcp_new) refers to tcp.o(i.tcp_alloc) for tcp_alloc
    tcp.o(i.tcp_new_port) refers to tcp.o(.data) for port
    tcp.o(i.tcp_next_iss) refers to tcp.o(.data) for iss
    tcp.o(i.tcp_pcb_purge) refers to pbuf.o(i.pbuf_free) for pbuf_free
    tcp.o(i.tcp_pcb_purge) refers to tcp.o(i.tcp_segs_free) for tcp_segs_free
    tcp.o(i.tcp_pcb_purge) refers to tcp.o(.data) for tcp_listen_pcbs
    tcp.o(i.tcp_pcb_remove) refers to tcp.o(i.tcp_pcb_purge) for tcp_pcb_purge
    tcp.o(i.tcp_pcb_remove) refers to tcp_out.o(i.tcp_output) for tcp_output
    tcp.o(i.tcp_pcb_remove) refers to tcp.o(.data) for tcp_tmp_pcb
    tcp.o(i.tcp_recv_null) refers to pbuf.o(i.pbuf_free) for pbuf_free
    tcp.o(i.tcp_recv_null) refers to tcp.o(i.tcp_close) for tcp_close
    tcp.o(i.tcp_recved) refers to tcp.o(i.tcp_update_rcv_ann_wnd) for tcp_update_rcv_ann_wnd
    tcp.o(i.tcp_recved) refers to tcp_out.o(i.tcp_output) for tcp_output
    tcp.o(i.tcp_seg_free) refers to pbuf.o(i.pbuf_free) for pbuf_free
    tcp.o(i.tcp_seg_free) refers to memp.o(i.memp_free) for memp_free
    tcp.o(i.tcp_segs_free) refers to tcp.o(i.tcp_seg_free) for tcp_seg_free
    tcp.o(i.tcp_slowtmr) refers to tcp_out.o(i.tcp_zero_window_probe) for tcp_zero_window_probe
    tcp.o(i.tcp_slowtmr) refers to tcp_out.o(i.tcp_rexmit_rto) for tcp_rexmit_rto
    tcp.o(i.tcp_slowtmr) refers to tcp.o(i.tcp_abandon) for tcp_abandon
    tcp.o(i.tcp_slowtmr) refers to tcp_out.o(i.tcp_keepalive) for tcp_keepalive
    tcp.o(i.tcp_slowtmr) refers to tcp.o(i.tcp_pcb_purge) for tcp_pcb_purge
    tcp.o(i.tcp_slowtmr) refers to memp.o(i.memp_free) for memp_free
    tcp.o(i.tcp_slowtmr) refers to tcp_out.o(i.tcp_output) for tcp_output
    tcp.o(i.tcp_slowtmr) refers to tcp.o(.data) for tcp_ticks
    tcp.o(i.tcp_slowtmr) refers to tcp.o(.constdata) for tcp_persist_backoff
    tcp.o(i.tcp_tmr) refers to tcp.o(i.tcp_fasttmr) for tcp_fasttmr
    tcp.o(i.tcp_tmr) refers to tcp.o(i.tcp_slowtmr) for tcp_slowtmr
    tcp.o(i.tcp_tmr) refers to tcp.o(.data) for tcp_timer
    tcp_in.o(i.tcp_input) refers to inet.o(i.ntohs) for ntohs
    tcp_in.o(i.tcp_input) refers to pbuf.o(i.pbuf_header) for pbuf_header
    tcp_in.o(i.tcp_input) refers to pbuf.o(i.pbuf_free) for pbuf_free
    tcp_in.o(i.tcp_input) refers to ip_addr.o(i.ip_addr_isbroadcast) for ip_addr_isbroadcast
    tcp_in.o(i.tcp_input) refers to inet.o(i.ntohl) for ntohl
    tcp_in.o(i.tcp_input) refers to tcp_in.o(i.tcp_timewait_input) for tcp_timewait_input
    tcp_in.o(i.tcp_input) refers to tcp_in.o(i.tcp_listen_input) for tcp_listen_input
    tcp_in.o(i.tcp_input) refers to tcp_in.o(i.tcp_process) for tcp_process
    tcp_in.o(i.tcp_input) refers to tcp.o(i.tcp_pcb_remove) for tcp_pcb_remove
    tcp_in.o(i.tcp_input) refers to memp.o(i.memp_free) for memp_free
    tcp_in.o(i.tcp_input) refers to tcp_in.o(.data) for iphdr
    tcp_in.o(i.tcp_input) refers to tcp.o(.data) for tcp_active_pcbs
    tcp_in.o(i.tcp_input) refers to tcp_in.o(.bss) for inseg
    tcp_in.o(i.tcp_input) refers to tcp_out.o(i.tcp_output) for tcp_output
    tcp_in.o(i.tcp_input) refers to tcp_out.o(i.tcp_rst) for tcp_rst
    tcp_in.o(i.tcp_listen_input) refers to tcp_out.o(i.tcp_rst) for tcp_rst
    tcp_in.o(i.tcp_listen_input) refers to tcp.o(i.tcp_alloc) for tcp_alloc
    tcp_in.o(i.tcp_listen_input) refers to tcp_in.o(i.tcp_parseopt) for tcp_parseopt
    tcp_in.o(i.tcp_listen_input) refers to tcp.o(i.tcp_eff_send_mss) for tcp_eff_send_mss
    tcp_in.o(i.tcp_listen_input) refers to tcp_out.o(i.tcp_enqueue) for tcp_enqueue
    tcp_in.o(i.tcp_listen_input) refers to tcp.o(i.tcp_abandon) for tcp_abandon
    tcp_in.o(i.tcp_listen_input) refers to tcp_out.o(i.tcp_output) for tcp_output
    tcp_in.o(i.tcp_listen_input) refers to tcp_in.o(.data) for flags
    tcp_in.o(i.tcp_listen_input) refers to tcp.o(.data) for tcp_active_pcbs
    tcp_in.o(i.tcp_parseopt) refers to inet.o(i.ntohs) for ntohs
    tcp_in.o(i.tcp_parseopt) refers to tcp_in.o(.data) for tcphdr
    tcp_in.o(i.tcp_process) refers to tcp_out.o(i.tcp_output) for tcp_output
    tcp_in.o(i.tcp_process) refers to tcp_in.o(i.tcp_parseopt) for tcp_parseopt
    tcp_in.o(i.tcp_process) refers to inet.o(i.ntohl) for ntohl
    tcp_in.o(i.tcp_process) refers to tcp.o(i.tcp_eff_send_mss) for tcp_eff_send_mss
    tcp_in.o(i.tcp_process) refers to tcp.o(i.tcp_seg_free) for tcp_seg_free
    tcp_in.o(i.tcp_process) refers to tcp_out.o(i.tcp_rst) for tcp_rst
    tcp_in.o(i.tcp_process) refers to tcp.o(i.tcp_abandon) for tcp_abandon
    tcp_in.o(i.tcp_process) refers to tcp_in.o(i.tcp_receive) for tcp_receive
    tcp_in.o(i.tcp_process) refers to tcp_out.o(i.tcp_rexmit) for tcp_rexmit
    tcp_in.o(i.tcp_process) refers to tcp.o(i.tcp_pcb_purge) for tcp_pcb_purge
    tcp_in.o(i.tcp_process) refers to tcp_in.o(.data) for flags
    tcp_in.o(i.tcp_process) refers to tcp.o(.data) for tcp_ticks
    tcp_in.o(i.tcp_receive) refers to tcp_out.o(i.tcp_rexmit) for tcp_rexmit
    tcp_in.o(i.tcp_receive) refers to pbuf.o(i.pbuf_clen) for pbuf_clen
    tcp_in.o(i.tcp_receive) refers to tcp.o(i.tcp_seg_free) for tcp_seg_free
    tcp_in.o(i.tcp_receive) refers to inet.o(i.ntohl) for ntohl
    tcp_in.o(i.tcp_receive) refers to inet.o(i.ntohs) for ntohs
    tcp_in.o(i.tcp_receive) refers to tcp_in.o(.data) for flags
    tcp_in.o(i.tcp_receive) refers to tcp.o(.data) for tcp_ticks
    tcp_in.o(i.tcp_receive) refers to tcp_in.o(.bss) for inseg
    tcp_in.o(i.tcp_receive) refers to pbuf.o(i.pbuf_header) for pbuf_header
    tcp_in.o(i.tcp_receive) refers to tcp_out.o(i.tcp_output) for tcp_output
    tcp_in.o(i.tcp_receive) refers to inet.o(i.htons) for htons
    tcp_in.o(i.tcp_receive) refers to pbuf.o(i.pbuf_realloc) for pbuf_realloc
    tcp_in.o(i.tcp_receive) refers to tcp.o(i.tcp_update_rcv_ann_wnd) for tcp_update_rcv_ann_wnd
    tcp_in.o(i.tcp_timewait_input) refers to tcp_out.o(i.tcp_output) for tcp_output
    tcp_in.o(i.tcp_timewait_input) refers to tcp_in.o(.data) for seqno
    tcp_out.o(i.tcp_enqueue) refers to memp.o(i.memp_malloc) for memp_malloc
    tcp_out.o(i.tcp_enqueue) refers to pbuf.o(i.pbuf_alloc) for pbuf_alloc
    tcp_out.o(i.tcp_enqueue) refers to pbuf.o(i.pbuf_clen) for pbuf_clen
    tcp_out.o(i.tcp_enqueue) refers to memcpya.o(.text) for __aeabi_memcpy
    tcp_out.o(i.tcp_enqueue) refers to pbuf.o(i.pbuf_free) for pbuf_free
    tcp_out.o(i.tcp_enqueue) refers to pbuf.o(i.pbuf_cat) for pbuf_cat
    tcp_out.o(i.tcp_enqueue) refers to pbuf.o(i.pbuf_header) for pbuf_header
    tcp_out.o(i.tcp_enqueue) refers to inet.o(i.htons) for htons
    tcp_out.o(i.tcp_enqueue) refers to inet.o(i.htonl) for htonl
    tcp_out.o(i.tcp_enqueue) refers to inet.o(i.ntohs) for ntohs
    tcp_out.o(i.tcp_enqueue) refers to memp.o(i.memp_free) for memp_free
    tcp_out.o(i.tcp_enqueue) refers to tcp.o(i.tcp_segs_free) for tcp_segs_free
    tcp_out.o(i.tcp_keepalive) refers to pbuf.o(i.pbuf_alloc) for pbuf_alloc
    tcp_out.o(i.tcp_keepalive) refers to inet.o(i.htonl) for htonl
    tcp_out.o(i.tcp_keepalive) refers to tcp_out.o(i.tcp_output_set_header) for tcp_output_set_header
    tcp_out.o(i.tcp_keepalive) refers to ip.o(i.ip_output) for ip_output
    tcp_out.o(i.tcp_keepalive) refers to pbuf.o(i.pbuf_free) for pbuf_free
    tcp_out.o(i.tcp_output) refers to inet.o(i.ntohl) for ntohl
    tcp_out.o(i.tcp_output) refers to pbuf.o(i.pbuf_alloc) for pbuf_alloc
    tcp_out.o(i.tcp_output) refers to inet.o(i.htonl) for htonl
    tcp_out.o(i.tcp_output) refers to tcp_out.o(i.tcp_output_set_header) for tcp_output_set_header
    tcp_out.o(i.tcp_output) refers to ip.o(i.ip_output) for ip_output
    tcp_out.o(i.tcp_output) refers to pbuf.o(i.pbuf_free) for pbuf_free
    tcp_out.o(i.tcp_output) refers to inet.o(i.ntohs) for ntohs
    tcp_out.o(i.tcp_output) refers to inet.o(i.htons) for htons
    tcp_out.o(i.tcp_output) refers to tcp_out.o(i.tcp_output_segment) for tcp_output_segment
    tcp_out.o(i.tcp_output) refers to tcp.o(i.tcp_seg_free) for tcp_seg_free
    tcp_out.o(i.tcp_output) refers to tcp_in.o(.data) for tcp_input_pcb
    tcp_out.o(i.tcp_output_segment) refers to inet.o(i.htonl) for htonl
    tcp_out.o(i.tcp_output_segment) refers to inet.o(i.htons) for htons
    tcp_out.o(i.tcp_output_segment) refers to ip.o(i.ip_route) for ip_route
    tcp_out.o(i.tcp_output_segment) refers to inet.o(i.ntohl) for ntohl
    tcp_out.o(i.tcp_output_segment) refers to ip.o(i.ip_output) for ip_output
    tcp_out.o(i.tcp_output_segment) refers to tcp.o(.data) for tcp_ticks
    tcp_out.o(i.tcp_output_set_header) refers to inet.o(i.htons) for htons
    tcp_out.o(i.tcp_output_set_header) refers to inet.o(i.htonl) for htonl
    tcp_out.o(i.tcp_output_set_header) refers to inet.o(i.ntohs) for ntohs
    tcp_out.o(i.tcp_rexmit) refers to inet.o(i.ntohl) for ntohl
    tcp_out.o(i.tcp_rexmit) refers to tcp_out.o(i.tcp_output) for tcp_output
    tcp_out.o(i.tcp_rexmit_rto) refers to tcp_out.o(i.tcp_output) for tcp_output
    tcp_out.o(i.tcp_rst) refers to pbuf.o(i.pbuf_alloc) for pbuf_alloc
    tcp_out.o(i.tcp_rst) refers to inet.o(i.htons) for htons
    tcp_out.o(i.tcp_rst) refers to inet.o(i.htonl) for htonl
    tcp_out.o(i.tcp_rst) refers to inet.o(i.ntohs) for ntohs
    tcp_out.o(i.tcp_rst) refers to ip.o(i.ip_output) for ip_output
    tcp_out.o(i.tcp_rst) refers to pbuf.o(i.pbuf_free) for pbuf_free
    tcp_out.o(i.tcp_send_ctrl) refers to tcp_out.o(i.tcp_enqueue) for tcp_enqueue
    tcp_out.o(i.tcp_write) refers to tcp_out.o(i.tcp_enqueue) for tcp_enqueue
    tcp_out.o(i.tcp_zero_window_probe) refers to pbuf.o(i.pbuf_alloc) for pbuf_alloc
    tcp_out.o(i.tcp_zero_window_probe) refers to tcp_out.o(i.tcp_output_set_header) for tcp_output_set_header
    tcp_out.o(i.tcp_zero_window_probe) refers to ip.o(i.ip_output) for ip_output
    tcp_out.o(i.tcp_zero_window_probe) refers to pbuf.o(i.pbuf_free) for pbuf_free
    icmp.o(i.icmp_dest_unreach) refers to icmp.o(i.icmp_send_response) for icmp_send_response
    icmp.o(i.icmp_input) refers to inet.o(i.ntohs) for ntohs
    icmp.o(i.icmp_input) refers to pbuf.o(i.pbuf_header) for pbuf_header
    icmp.o(i.icmp_input) refers to inet.o(i.ntohl) for ntohl
    icmp.o(i.icmp_input) refers to ip_addr.o(i.ip_addr_isbroadcast) for ip_addr_isbroadcast
    icmp.o(i.icmp_input) refers to pbuf.o(i.pbuf_free) for pbuf_free
    icmp.o(i.icmp_input) refers to inet_chksum.o(i.inet_chksum_pbuf) for inet_chksum_pbuf
    icmp.o(i.icmp_input) refers to pbuf.o(i.pbuf_alloc) for pbuf_alloc
    icmp.o(i.icmp_input) refers to pbuf.o(i.pbuf_copy) for pbuf_copy
    icmp.o(i.icmp_input) refers to inet.o(i.htons) for htons
    icmp.o(i.icmp_input) refers to ip.o(i.ip_output_if) for ip_output_if
    icmp.o(i.icmp_send_response) refers to pbuf.o(i.pbuf_alloc) for pbuf_alloc
    icmp.o(i.icmp_send_response) refers to memcpya.o(.text) for __aeabi_memcpy
    icmp.o(i.icmp_send_response) refers to inet_chksum.o(i.inet_chksum) for inet_chksum
    icmp.o(i.icmp_send_response) refers to ip.o(i.ip_output) for ip_output
    icmp.o(i.icmp_send_response) refers to pbuf.o(i.pbuf_free) for pbuf_free
    icmp.o(i.icmp_time_exceeded) refers to icmp.o(i.icmp_send_response) for icmp_send_response
    inet.o(i.inet_addr) refers to inet.o(i.inet_aton) for inet_aton
    inet.o(i.inet_aton) refers to inet.o(i.htonl) for htonl
    inet.o(i.inet_ntoa) refers to inet.o(.bss) for str
    inet.o(i.ntohl) refers to inet.o(i.htonl) for htonl
    inet.o(i.ntohs) refers to inet.o(i.htons) for htons
    inet_chksum.o(i.inet_chksum) refers to inet_chksum.o(i.lwip_standard_chksum) for lwip_standard_chksum
    inet_chksum.o(i.inet_chksum_pbuf) refers to inet_chksum.o(i.lwip_standard_chksum) for lwip_standard_chksum
    inet_chksum.o(i.inet_chksum_pseudo) refers to inet_chksum.o(i.lwip_standard_chksum) for lwip_standard_chksum
    inet_chksum.o(i.inet_chksum_pseudo) refers to inet.o(i.htons) for htons
    inet_chksum.o(i.lwip_standard_chksum) refers to inet.o(i.htons) for htons
    ip.o(i.ip_current_header) refers to ip.o(.data) for current_header
    ip.o(i.ip_current_netif) refers to ip.o(.data) for current_netif
    ip.o(i.ip_input) refers to inet.o(i.ntohs) for ntohs
    ip.o(i.ip_input) refers to pbuf.o(i.pbuf_free) for pbuf_free
    ip.o(i.ip_input) refers to pbuf.o(i.pbuf_realloc) for pbuf_realloc
    ip.o(i.ip_input) refers to netif.o(i.netif_is_up) for netif_is_up
    ip.o(i.ip_input) refers to ip_addr.o(i.ip_addr_isbroadcast) for ip_addr_isbroadcast
    ip.o(i.ip_input) refers to inet.o(i.ntohl) for ntohl
    ip.o(i.ip_input) refers to inet.o(i.htons) for htons
    ip.o(i.ip_input) refers to ip_frag.o(i.ip_reass) for ip_reass
    ip.o(i.ip_input) refers to tcp_in.o(i.tcp_input) for tcp_input
    ip.o(i.ip_input) refers to icmp.o(i.icmp_input) for icmp_input
    ip.o(i.ip_input) refers to icmp.o(i.icmp_dest_unreach) for icmp_dest_unreach
    ip.o(i.ip_input) refers to netif.o(.data) for netif_list
    ip.o(i.ip_input) refers to ip.o(.data) for current_netif
    ip.o(i.ip_output) refers to ip.o(i.ip_route) for ip_route
    ip.o(i.ip_output) refers to ip.o(i.ip_output_if) for ip_output_if
    ip.o(i.ip_output_if) refers to pbuf.o(i.pbuf_header) for pbuf_header
    ip.o(i.ip_output_if) refers to inet.o(i.ntohs) for ntohs
    ip.o(i.ip_output_if) refers to inet.o(i.htons) for htons
    ip.o(i.ip_output_if) refers to ip_frag.o(i.ip_frag) for ip_frag
    ip.o(i.ip_output_if) refers to ip.o(.data) for ip_id
    ip.o(i.ip_route) refers to netif.o(i.netif_is_up) for netif_is_up
    ip.o(i.ip_route) refers to netif.o(.data) for netif_list
    ip_frag.o(i.ip_frag) refers to pbuf.o(i.pbuf_alloc) for pbuf_alloc
    ip_frag.o(i.ip_frag) refers to memcpya.o(.text) for __aeabi_memcpy
    ip_frag.o(i.ip_frag) refers to inet.o(i.ntohs) for ntohs
    ip_frag.o(i.ip_frag) refers to pbuf.o(i.pbuf_copy_partial) for pbuf_copy_partial
    ip_frag.o(i.ip_frag) refers to inet.o(i.htons) for htons
    ip_frag.o(i.ip_frag) refers to inet_chksum.o(i.inet_chksum) for inet_chksum
    ip_frag.o(i.ip_frag) refers to pbuf.o(i.pbuf_realloc) for pbuf_realloc
    ip_frag.o(i.ip_frag) refers to pbuf.o(i.pbuf_chain) for pbuf_chain
    ip_frag.o(i.ip_frag) refers to pbuf.o(i.pbuf_free) for pbuf_free
    ip_frag.o(i.ip_frag) refers to ip_frag.o(.bss) for buf
    ip_frag.o(i.ip_reass) refers to inet.o(i.ntohs) for ntohs
    ip_frag.o(i.ip_reass) refers to pbuf.o(i.pbuf_clen) for pbuf_clen
    ip_frag.o(i.ip_reass) refers to ip_frag.o(i.ip_reass_remove_oldest_datagram) for ip_reass_remove_oldest_datagram
    ip_frag.o(i.ip_reass) refers to ip_frag.o(i.ip_reass_enqueue_new_datagram) for ip_reass_enqueue_new_datagram
    ip_frag.o(i.ip_reass) refers to memcpya.o(.text) for __aeabi_memcpy
    ip_frag.o(i.ip_reass) refers to ip_frag.o(i.ip_reass_chain_frag_into_datagram_and_validate) for ip_reass_chain_frag_into_datagram_and_validate
    ip_frag.o(i.ip_reass) refers to inet.o(i.htons) for htons
    ip_frag.o(i.ip_reass) refers to inet_chksum.o(i.inet_chksum) for inet_chksum
    ip_frag.o(i.ip_reass) refers to pbuf.o(i.pbuf_header) for pbuf_header
    ip_frag.o(i.ip_reass) refers to pbuf.o(i.pbuf_cat) for pbuf_cat
    ip_frag.o(i.ip_reass) refers to ip_frag.o(i.ip_reass_dequeue_datagram) for ip_reass_dequeue_datagram
    ip_frag.o(i.ip_reass) refers to pbuf.o(i.pbuf_free) for pbuf_free
    ip_frag.o(i.ip_reass) refers to ip_frag.o(.data) for ip_reass_pbufcount
    ip_frag.o(i.ip_reass_chain_frag_into_datagram_and_validate) refers to inet.o(i.ntohs) for ntohs
    ip_frag.o(i.ip_reass_chain_frag_into_datagram_and_validate) refers to pbuf.o(i.pbuf_clen) for pbuf_clen
    ip_frag.o(i.ip_reass_chain_frag_into_datagram_and_validate) refers to pbuf.o(i.pbuf_free) for pbuf_free
    ip_frag.o(i.ip_reass_chain_frag_into_datagram_and_validate) refers to ip_frag.o(.data) for ip_reass_pbufcount
    ip_frag.o(i.ip_reass_dequeue_datagram) refers to memp.o(i.memp_free) for memp_free
    ip_frag.o(i.ip_reass_dequeue_datagram) refers to ip_frag.o(.data) for reassdatagrams
    ip_frag.o(i.ip_reass_enqueue_new_datagram) refers to memp.o(i.memp_malloc) for memp_malloc
    ip_frag.o(i.ip_reass_enqueue_new_datagram) refers to ip_frag.o(i.ip_reass_remove_oldest_datagram) for ip_reass_remove_oldest_datagram
    ip_frag.o(i.ip_reass_enqueue_new_datagram) refers to memseta.o(.text) for __aeabi_memclr4
    ip_frag.o(i.ip_reass_enqueue_new_datagram) refers to memcpya.o(.text) for __aeabi_memcpy
    ip_frag.o(i.ip_reass_enqueue_new_datagram) refers to ip_frag.o(.data) for reassdatagrams
    ip_frag.o(i.ip_reass_free_complete_datagram) refers to memcpya.o(.text) for __aeabi_memcpy
    ip_frag.o(i.ip_reass_free_complete_datagram) refers to icmp.o(i.icmp_time_exceeded) for icmp_time_exceeded
    ip_frag.o(i.ip_reass_free_complete_datagram) refers to pbuf.o(i.pbuf_clen) for pbuf_clen
    ip_frag.o(i.ip_reass_free_complete_datagram) refers to pbuf.o(i.pbuf_free) for pbuf_free
    ip_frag.o(i.ip_reass_free_complete_datagram) refers to ip_frag.o(i.ip_reass_dequeue_datagram) for ip_reass_dequeue_datagram
    ip_frag.o(i.ip_reass_free_complete_datagram) refers to ip_frag.o(.data) for ip_reass_pbufcount
    ip_frag.o(i.ip_reass_remove_oldest_datagram) refers to ip_frag.o(i.ip_reass_free_complete_datagram) for ip_reass_free_complete_datagram
    ip_frag.o(i.ip_reass_remove_oldest_datagram) refers to ip_frag.o(.data) for reassdatagrams
    ip_frag.o(i.ip_reass_tmr) refers to ip_frag.o(i.ip_reass_free_complete_datagram) for ip_reass_free_complete_datagram
    ip_frag.o(i.ip_reass_tmr) refers to ip_frag.o(.data) for reassdatagrams
    etharp.o(i.etharp_arp_input) refers to pbuf.o(i.pbuf_free) for pbuf_free
    etharp.o(i.etharp_arp_input) refers to inet.o(i.htons) for htons
    etharp.o(i.etharp_arp_input) refers to etharp.o(i.update_arp_entry) for update_arp_entry
    etharp.o(i.etharp_find_addr) refers to etharp.o(i.find_entry) for find_entry
    etharp.o(i.etharp_find_addr) refers to etharp.o(.bss) for arp_table
    etharp.o(i.etharp_ip_input) refers to etharp.o(i.update_arp_entry) for update_arp_entry
    etharp.o(i.etharp_output) refers to pbuf.o(i.pbuf_header) for pbuf_header
    etharp.o(i.etharp_output) refers to ip_addr.o(i.ip_addr_isbroadcast) for ip_addr_isbroadcast
    etharp.o(i.etharp_output) refers to inet.o(i.ntohl) for ntohl
    etharp.o(i.etharp_output) refers to etharp.o(i.etharp_query) for etharp_query
    etharp.o(i.etharp_output) refers to etharp.o(i.etharp_send_ip) for etharp_send_ip
    etharp.o(i.etharp_output) refers to etharp.o(.constdata) for ethbroadcast
    etharp.o(i.etharp_query) refers to ip_addr.o(i.ip_addr_isbroadcast) for ip_addr_isbroadcast
    etharp.o(i.etharp_query) refers to inet.o(i.ntohl) for ntohl
    etharp.o(i.etharp_query) refers to etharp.o(i.find_entry) for find_entry
    etharp.o(i.etharp_query) refers to etharp.o(i.etharp_request) for etharp_request
    etharp.o(i.etharp_query) refers to etharp.o(i.etharp_send_ip) for etharp_send_ip
    etharp.o(i.etharp_query) refers to pbuf.o(i.pbuf_alloc) for pbuf_alloc
    etharp.o(i.etharp_query) refers to pbuf.o(i.pbuf_copy) for pbuf_copy
    etharp.o(i.etharp_query) refers to pbuf.o(i.pbuf_free) for pbuf_free
    etharp.o(i.etharp_query) refers to pbuf.o(i.pbuf_ref) for pbuf_ref
    etharp.o(i.etharp_query) refers to memp.o(i.memp_malloc) for memp_malloc
    etharp.o(i.etharp_query) refers to etharp.o(.bss) for arp_table
    etharp.o(i.etharp_raw) refers to pbuf.o(i.pbuf_alloc) for pbuf_alloc
    etharp.o(i.etharp_raw) refers to inet.o(i.htons) for htons
    etharp.o(i.etharp_raw) refers to pbuf.o(i.pbuf_free) for pbuf_free
    etharp.o(i.etharp_request) refers to etharp.o(i.etharp_raw) for etharp_raw
    etharp.o(i.etharp_request) refers to etharp.o(.constdata) for ethzero
    etharp.o(i.etharp_send_ip) refers to inet.o(i.htons) for htons
    etharp.o(i.etharp_tmr) refers to etharp.o(i.free_etharp_q) for free_etharp_q
    etharp.o(i.etharp_tmr) refers to etharp.o(.bss) for arp_table
    etharp.o(i.ethernet_input) refers to inet.o(i.htons) for htons
    etharp.o(i.ethernet_input) refers to etharp.o(i.etharp_ip_input) for etharp_ip_input
    etharp.o(i.ethernet_input) refers to pbuf.o(i.pbuf_header) for pbuf_header
    etharp.o(i.ethernet_input) refers to pbuf.o(i.pbuf_free) for pbuf_free
    etharp.o(i.ethernet_input) refers to ip.o(i.ip_input) for ip_input
    etharp.o(i.ethernet_input) refers to etharp.o(i.etharp_arp_input) for etharp_arp_input
    etharp.o(i.find_entry) refers to etharp.o(i.free_etharp_q) for free_etharp_q
    etharp.o(i.find_entry) refers to etharp.o(.data) for etharp_cached_entry
    etharp.o(i.find_entry) refers to etharp.o(.bss) for arp_table
    etharp.o(i.free_etharp_q) refers to pbuf.o(i.pbuf_free) for pbuf_free
    etharp.o(i.free_etharp_q) refers to memp.o(i.memp_free) for memp_free
    etharp.o(i.update_arp_entry) refers to ip_addr.o(i.ip_addr_isbroadcast) for ip_addr_isbroadcast
    etharp.o(i.update_arp_entry) refers to inet.o(i.ntohl) for ntohl
    etharp.o(i.update_arp_entry) refers to etharp.o(i.find_entry) for find_entry
    etharp.o(i.update_arp_entry) refers to memp.o(i.memp_free) for memp_free
    etharp.o(i.update_arp_entry) refers to etharp.o(i.etharp_send_ip) for etharp_send_ip
    etharp.o(i.update_arp_entry) refers to pbuf.o(i.pbuf_free) for pbuf_free
    etharp.o(i.update_arp_entry) refers to etharp.o(.bss) for arp_table
    stm32f10x_gpio.o(i.GPIO_AFIODeInit) refers to stm32f10x_rcc.o(i.RCC_APB2PeriphResetCmd) for RCC_APB2PeriphResetCmd
    stm32f10x_gpio.o(i.GPIO_DeInit) refers to stm32f10x_rcc.o(i.RCC_APB2PeriphResetCmd) for RCC_APB2PeriphResetCmd
    stm32f10x_rcc.o(i.RCC_GetClocksFreq) refers to stm32f10x_rcc.o(.data) for APBAHBPrescTable
    stm32f10x_rcc.o(i.RCC_WaitForHSEStartUp) refers to stm32f10x_rcc.o(i.RCC_GetFlagStatus) for RCC_GetFlagStatus
    stm32f10x_usart.o(i.USART_DeInit) refers to stm32f10x_rcc.o(i.RCC_APB2PeriphResetCmd) for RCC_APB2PeriphResetCmd
    stm32f10x_usart.o(i.USART_DeInit) refers to stm32f10x_rcc.o(i.RCC_APB1PeriphResetCmd) for RCC_APB1PeriphResetCmd
    stm32f10x_usart.o(i.USART_Init) refers to stm32f10x_rcc.o(i.RCC_GetClocksFreq) for RCC_GetClocksFreq
    stm32f10x_spi.o(i.I2S_Init) refers to stm32f10x_rcc.o(i.RCC_GetClocksFreq) for RCC_GetClocksFreq
    stm32f10x_spi.o(i.SPI_I2S_DeInit) refers to stm32f10x_rcc.o(i.RCC_APB2PeriphResetCmd) for RCC_APB2PeriphResetCmd
    stm32f10x_spi.o(i.SPI_I2S_DeInit) refers to stm32f10x_rcc.o(i.RCC_APB1PeriphResetCmd) for RCC_APB1PeriphResetCmd
    stm32f10x_adc.o(i.ADC_DeInit) refers to stm32f10x_rcc.o(i.RCC_APB2PeriphResetCmd) for RCC_APB2PeriphResetCmd
    stm32f10x_tim.o(i.TIM_DeInit) refers to stm32f10x_rcc.o(i.RCC_APB2PeriphResetCmd) for RCC_APB2PeriphResetCmd
    stm32f10x_tim.o(i.TIM_DeInit) refers to stm32f10x_rcc.o(i.RCC_APB1PeriphResetCmd) for RCC_APB1PeriphResetCmd
    stm32f10x_tim.o(i.TIM_ETRClockMode1Config) refers to stm32f10x_tim.o(i.TIM_ETRConfig) for TIM_ETRConfig
    stm32f10x_tim.o(i.TIM_ETRClockMode2Config) refers to stm32f10x_tim.o(i.TIM_ETRConfig) for TIM_ETRConfig
    stm32f10x_tim.o(i.TIM_ICInit) refers to stm32f10x_tim.o(i.TI1_Config) for TI1_Config
    stm32f10x_tim.o(i.TIM_ICInit) refers to stm32f10x_tim.o(i.TIM_SetIC1Prescaler) for TIM_SetIC1Prescaler
    stm32f10x_tim.o(i.TIM_ICInit) refers to stm32f10x_tim.o(i.TI2_Config) for TI2_Config
    stm32f10x_tim.o(i.TIM_ICInit) refers to stm32f10x_tim.o(i.TIM_SetIC2Prescaler) for TIM_SetIC2Prescaler
    stm32f10x_tim.o(i.TIM_ICInit) refers to stm32f10x_tim.o(i.TI3_Config) for TI3_Config
    stm32f10x_tim.o(i.TIM_ICInit) refers to stm32f10x_tim.o(i.TIM_SetIC3Prescaler) for TIM_SetIC3Prescaler
    stm32f10x_tim.o(i.TIM_ICInit) refers to stm32f10x_tim.o(i.TI4_Config) for TI4_Config
    stm32f10x_tim.o(i.TIM_ICInit) refers to stm32f10x_tim.o(i.TIM_SetIC4Prescaler) for TIM_SetIC4Prescaler
    stm32f10x_tim.o(i.TIM_ITRxExternalClockConfig) refers to stm32f10x_tim.o(i.TIM_SelectInputTrigger) for TIM_SelectInputTrigger
    stm32f10x_tim.o(i.TIM_PWMIConfig) refers to stm32f10x_tim.o(i.TI1_Config) for TI1_Config
    stm32f10x_tim.o(i.TIM_PWMIConfig) refers to stm32f10x_tim.o(i.TIM_SetIC1Prescaler) for TIM_SetIC1Prescaler
    stm32f10x_tim.o(i.TIM_PWMIConfig) refers to stm32f10x_tim.o(i.TI2_Config) for TI2_Config
    stm32f10x_tim.o(i.TIM_PWMIConfig) refers to stm32f10x_tim.o(i.TIM_SetIC2Prescaler) for TIM_SetIC2Prescaler
    stm32f10x_tim.o(i.TIM_TIxExternalClockConfig) refers to stm32f10x_tim.o(i.TI2_Config) for TI2_Config
    stm32f10x_tim.o(i.TIM_TIxExternalClockConfig) refers to stm32f10x_tim.o(i.TI1_Config) for TI1_Config
    stm32f10x_tim.o(i.TIM_TIxExternalClockConfig) refers to stm32f10x_tim.o(i.TIM_SelectInputTrigger) for TIM_SelectInputTrigger
    stm32f10x_i2c.o(i.I2C_DeInit) refers to stm32f10x_rcc.o(i.RCC_APB1PeriphResetCmd) for RCC_APB1PeriphResetCmd
    stm32f10x_i2c.o(i.I2C_Init) refers to stm32f10x_rcc.o(i.RCC_GetClocksFreq) for RCC_GetClocksFreq
    startup_stm32f10x_cl.o(RESET) refers to startup_stm32f10x_cl.o(STACK) for __initial_sp
    startup_stm32f10x_cl.o(RESET) refers to startup_stm32f10x_cl.o(.text) for Reset_Handler
    startup_stm32f10x_cl.o(RESET) refers to stm32f10x_it.o(i.NMI_Handler) for NMI_Handler
    startup_stm32f10x_cl.o(RESET) refers to stm32f10x_it.o(i.HardFault_Handler) for HardFault_Handler
    startup_stm32f10x_cl.o(RESET) refers to stm32f10x_it.o(i.MemManage_Handler) for MemManage_Handler
    startup_stm32f10x_cl.o(RESET) refers to stm32f10x_it.o(i.BusFault_Handler) for BusFault_Handler
    startup_stm32f10x_cl.o(RESET) refers to stm32f10x_it.o(i.UsageFault_Handler) for UsageFault_Handler
    startup_stm32f10x_cl.o(RESET) refers to stm32f10x_it.o(i.SVC_Handler) for SVC_Handler
    startup_stm32f10x_cl.o(RESET) refers to stm32f10x_it.o(i.DebugMon_Handler) for DebugMon_Handler
    startup_stm32f10x_cl.o(RESET) refers to os_cpu_a.o(.text) for PendSV_Handler
    startup_stm32f10x_cl.o(RESET) refers to delay.o(i.SysTick_Handler) for SysTick_Handler
    startup_stm32f10x_cl.o(RESET) refers to usart1.o(i.USART1_IRQHandler) for USART1_IRQHandler
    startup_stm32f10x_cl.o(RESET) refers to stm32f10x_it.o(i.ETH_IRQHandler) for ETH_IRQHandler
    startup_stm32f10x_cl.o(.text) refers to system_stm32f10x.o(i.SystemInit) for SystemInit
    startup_stm32f10x_cl.o(.text) refers to entry.o(.ARM.Collect$$$$00000000) for __main
    system_stm32f10x.o(i.SetSysClock) refers to system_stm32f10x.o(i.SetSysClockTo72) for SetSysClockTo72
    system_stm32f10x.o(i.SystemCoreClockUpdate) refers to system_stm32f10x.o(.data) for SystemCoreClock
    system_stm32f10x.o(i.SystemInit) refers to system_stm32f10x.o(i.SetSysClock) for SetSysClock
    entry.o(.ARM.Collect$$$$00000000) refers (Special) to entry10a.o(.ARM.Collect$$$$0000000D) for __rt_final_cpp
    entry.o(.ARM.Collect$$$$00000000) refers (Special) to entry11a.o(.ARM.Collect$$$$0000000F) for __rt_final_exit
    entry.o(.ARM.Collect$$$$00000000) refers (Special) to entry7b.o(.ARM.Collect$$$$00000008) for _main_clock
    entry.o(.ARM.Collect$$$$00000000) refers (Special) to entry8b.o(.ARM.Collect$$$$0000000A) for _main_cpp_init
    entry.o(.ARM.Collect$$$$00000000) refers (Special) to entry9a.o(.ARM.Collect$$$$0000000B) for _main_init
    entry.o(.ARM.Collect$$$$00000000) refers (Special) to entry5.o(.ARM.Collect$$$$00000004) for _main_scatterload
    entry.o(.ARM.Collect$$$$00000000) refers (Special) to entry2.o(.ARM.Collect$$$$00000001) for _main_stk
    printfb.o(i.__0fprintf$bare) refers to printfb.o(i._printf_core) for _printf_core
    printfb.o(i.__0fprintf$bare) refers to printf.o(i.fputc) for fputc
    printfb.o(i.__0printf$bare) refers to printfb.o(i._printf_core) for _printf_core
    printfb.o(i.__0printf$bare) refers to printf.o(i.fputc) for fputc
    printfb.o(i.__0printf$bare) refers to printf.o(.data) for __stdout
    printfb.o(i.__0snprintf$bare) refers to printfb.o(i._printf_core) for _printf_core
    printfb.o(i.__0snprintf$bare) refers to printfb.o(i._snputc) for _snputc
    printfb.o(i.__0sprintf$bare) refers to printfb.o(i._printf_core) for _printf_core
    printfb.o(i.__0sprintf$bare) refers to printfb.o(i._sputc) for _sputc
    printfb.o(i.__0vfprintf$bare) refers to printfb.o(i._printf_core) for _printf_core
    printfb.o(i.__0vfprintf$bare) refers to printf.o(i.fputc) for fputc
    printfb.o(i.__0vprintf$bare) refers to printfb.o(i._printf_core) for _printf_core
    printfb.o(i.__0vprintf$bare) refers to printf.o(i.fputc) for fputc
    printfb.o(i.__0vprintf$bare) refers to printf.o(.data) for __stdout
    printfb.o(i.__0vsnprintf$bare) refers to printfb.o(i._printf_core) for _printf_core
    printfb.o(i.__0vsnprintf$bare) refers to printfb.o(i._snputc) for _snputc
    printfb.o(i.__0vsprintf$bare) refers to printfb.o(i._printf_core) for _printf_core
    printfb.o(i.__0vsprintf$bare) refers to printfb.o(i._sputc) for _sputc
    printf0.o(i.__0fprintf$0) refers to printf0.o(i._printf_core) for _printf_core
    printf0.o(i.__0fprintf$0) refers to printf.o(i.fputc) for fputc
    printf0.o(i.__0printf$0) refers to printf0.o(i._printf_core) for _printf_core
    printf0.o(i.__0printf$0) refers to printf.o(i.fputc) for fputc
    printf0.o(i.__0printf$0) refers to printf.o(.data) for __stdout
    printf0.o(i.__0snprintf$0) refers to printf0.o(i._printf_core) for _printf_core
    printf0.o(i.__0snprintf$0) refers to printf0.o(i._snputc) for _snputc
    printf0.o(i.__0sprintf$0) refers to printf0.o(i._printf_core) for _printf_core
    printf0.o(i.__0sprintf$0) refers to printf0.o(i._sputc) for _sputc
    printf0.o(i.__0vfprintf$0) refers to printf0.o(i._printf_core) for _printf_core
    printf0.o(i.__0vfprintf$0) refers to printf.o(i.fputc) for fputc
    printf0.o(i.__0vprintf$0) refers to printf0.o(i._printf_core) for _printf_core
    printf0.o(i.__0vprintf$0) refers to printf.o(i.fputc) for fputc
    printf0.o(i.__0vprintf$0) refers to printf.o(.data) for __stdout
    printf0.o(i.__0vsnprintf$0) refers to printf0.o(i._printf_core) for _printf_core
    printf0.o(i.__0vsnprintf$0) refers to printf0.o(i._snputc) for _snputc
    printf0.o(i.__0vsprintf$0) refers to printf0.o(i._printf_core) for _printf_core
    printf0.o(i.__0vsprintf$0) refers to printf0.o(i._sputc) for _sputc
    printf1.o(i.__0fprintf$1) refers to printf1.o(i._printf_core) for _printf_core
    printf1.o(i.__0fprintf$1) refers to printf.o(i.fputc) for fputc
    printf1.o(i.__0printf$1) refers to printf1.o(i._printf_core) for _printf_core
    printf1.o(i.__0printf$1) refers to printf.o(i.fputc) for fputc
    printf1.o(i.__0printf$1) refers to printf.o(.data) for __stdout
    printf1.o(i.__0snprintf$1) refers to printf1.o(i._printf_core) for _printf_core
    printf1.o(i.__0snprintf$1) refers to printf1.o(i._snputc) for _snputc
    printf1.o(i.__0sprintf$1) refers to printf1.o(i._printf_core) for _printf_core
    printf1.o(i.__0sprintf$1) refers to printf1.o(i._sputc) for _sputc
    printf1.o(i.__0vfprintf$1) refers to printf1.o(i._printf_core) for _printf_core
    printf1.o(i.__0vfprintf$1) refers to printf.o(i.fputc) for fputc
    printf1.o(i.__0vprintf$1) refers to printf1.o(i._printf_core) for _printf_core
    printf1.o(i.__0vprintf$1) refers to printf.o(i.fputc) for fputc
    printf1.o(i.__0vprintf$1) refers to printf.o(.data) for __stdout
    printf1.o(i.__0vsnprintf$1) refers to printf1.o(i._printf_core) for _printf_core
    printf1.o(i.__0vsnprintf$1) refers to printf1.o(i._snputc) for _snputc
    printf1.o(i.__0vsprintf$1) refers to printf1.o(i._printf_core) for _printf_core
    printf1.o(i.__0vsprintf$1) refers to printf1.o(i._sputc) for _sputc
    printf1.o(i._printf_core) refers to uidiv.o(.text) for __aeabi_uidivmod
    printf2.o(i.__0fprintf$2) refers to printf2.o(i._printf_core) for _printf_core
    printf2.o(i.__0fprintf$2) refers to printf.o(i.fputc) for fputc
    printf2.o(i.__0printf$2) refers to printf2.o(i._printf_core) for _printf_core
    printf2.o(i.__0printf$2) refers to printf.o(i.fputc) for fputc
    printf2.o(i.__0printf$2) refers to printf.o(.data) for __stdout
    printf2.o(i.__0snprintf$2) refers to printf2.o(i._printf_core) for _printf_core
    printf2.o(i.__0snprintf$2) refers to printf2.o(i._snputc) for _snputc
    printf2.o(i.__0sprintf$2) refers to printf2.o(i._printf_core) for _printf_core
    printf2.o(i.__0sprintf$2) refers to printf2.o(i._sputc) for _sputc
    printf2.o(i.__0vfprintf$2) refers to printf2.o(i._printf_core) for _printf_core
    printf2.o(i.__0vfprintf$2) refers to printf.o(i.fputc) for fputc
    printf2.o(i.__0vprintf$2) refers to printf2.o(i._printf_core) for _printf_core
    printf2.o(i.__0vprintf$2) refers to printf.o(i.fputc) for fputc
    printf2.o(i.__0vprintf$2) refers to printf.o(.data) for __stdout
    printf2.o(i.__0vsnprintf$2) refers to printf2.o(i._printf_core) for _printf_core
    printf2.o(i.__0vsnprintf$2) refers to printf2.o(i._snputc) for _snputc
    printf2.o(i.__0vsprintf$2) refers to printf2.o(i._printf_core) for _printf_core
    printf2.o(i.__0vsprintf$2) refers to printf2.o(i._sputc) for _sputc
    printf3.o(i.__0fprintf$3) refers to printf3.o(i._printf_core) for _printf_core
    printf3.o(i.__0fprintf$3) refers to printf.o(i.fputc) for fputc
    printf3.o(i.__0printf$3) refers to printf3.o(i._printf_core) for _printf_core
    printf3.o(i.__0printf$3) refers to printf.o(i.fputc) for fputc
    printf3.o(i.__0printf$3) refers to printf.o(.data) for __stdout
    printf3.o(i.__0snprintf$3) refers to printf3.o(i._printf_core) for _printf_core
    printf3.o(i.__0snprintf$3) refers to printf3.o(i._snputc) for _snputc
    printf3.o(i.__0sprintf$3) refers to printf3.o(i._printf_core) for _printf_core
    printf3.o(i.__0sprintf$3) refers to printf3.o(i._sputc) for _sputc
    printf3.o(i.__0vfprintf$3) refers to printf3.o(i._printf_core) for _printf_core
    printf3.o(i.__0vfprintf$3) refers to printf.o(i.fputc) for fputc
    printf3.o(i.__0vprintf$3) refers to printf3.o(i._printf_core) for _printf_core
    printf3.o(i.__0vprintf$3) refers to printf.o(i.fputc) for fputc
    printf3.o(i.__0vprintf$3) refers to printf.o(.data) for __stdout
    printf3.o(i.__0vsnprintf$3) refers to printf3.o(i._printf_core) for _printf_core
    printf3.o(i.__0vsnprintf$3) refers to printf3.o(i._snputc) for _snputc
    printf3.o(i.__0vsprintf$3) refers to printf3.o(i._printf_core) for _printf_core
    printf3.o(i.__0vsprintf$3) refers to printf3.o(i._sputc) for _sputc
    printf3.o(i._printf_core) refers to uidiv.o(.text) for __aeabi_uidivmod
    printf4.o(i.__0fprintf$4) refers to printf4.o(i._printf_core) for _printf_core
    printf4.o(i.__0fprintf$4) refers to printf.o(i.fputc) for fputc
    printf4.o(i.__0printf$4) refers to printf4.o(i._printf_core) for _printf_core
    printf4.o(i.__0printf$4) refers to printf.o(i.fputc) for fputc
    printf4.o(i.__0printf$4) refers to printf.o(.data) for __stdout
    printf4.o(i.__0snprintf$4) refers to printf4.o(i._printf_core) for _printf_core
    printf4.o(i.__0snprintf$4) refers to printf4.o(i._snputc) for _snputc
    printf4.o(i.__0sprintf$4) refers to printf4.o(i._printf_core) for _printf_core
    printf4.o(i.__0sprintf$4) refers to printf4.o(i._sputc) for _sputc
    printf4.o(i.__0vfprintf$4) refers to printf4.o(i._printf_core) for _printf_core
    printf4.o(i.__0vfprintf$4) refers to printf.o(i.fputc) for fputc
    printf4.o(i.__0vprintf$4) refers to printf4.o(i._printf_core) for _printf_core
    printf4.o(i.__0vprintf$4) refers to printf.o(i.fputc) for fputc
    printf4.o(i.__0vprintf$4) refers to printf.o(.data) for __stdout
    printf4.o(i.__0vsnprintf$4) refers to printf4.o(i._printf_core) for _printf_core
    printf4.o(i.__0vsnprintf$4) refers to printf4.o(i._snputc) for _snputc
    printf4.o(i.__0vsprintf$4) refers to printf4.o(i._printf_core) for _printf_core
    printf4.o(i.__0vsprintf$4) refers to printf4.o(i._sputc) for _sputc
    printf4.o(i._printf_core) refers to uldiv.o(.text) for __aeabi_uldivmod
    printf5.o(i.__0fprintf$5) refers to printf5.o(i._printf_core) for _printf_core
    printf5.o(i.__0fprintf$5) refers to printf.o(i.fputc) for fputc
    printf5.o(i.__0printf$5) refers to printf5.o(i._printf_core) for _printf_core
    printf5.o(i.__0printf$5) refers to printf.o(i.fputc) for fputc
    printf5.o(i.__0printf$5) refers to printf.o(.data) for __stdout
    printf5.o(i.__0snprintf$5) refers to printf5.o(i._printf_core) for _printf_core
    printf5.o(i.__0snprintf$5) refers to printf5.o(i._snputc) for _snputc
    printf5.o(i.__0sprintf$5) refers to printf5.o(i._printf_core) for _printf_core
    printf5.o(i.__0sprintf$5) refers to printf5.o(i._sputc) for _sputc
    printf5.o(i.__0vfprintf$5) refers to printf5.o(i._printf_core) for _printf_core
    printf5.o(i.__0vfprintf$5) refers to printf.o(i.fputc) for fputc
    printf5.o(i.__0vprintf$5) refers to printf5.o(i._printf_core) for _printf_core
    printf5.o(i.__0vprintf$5) refers to printf.o(i.fputc) for fputc
    printf5.o(i.__0vprintf$5) refers to printf.o(.data) for __stdout
    printf5.o(i.__0vsnprintf$5) refers to printf5.o(i._printf_core) for _printf_core
    printf5.o(i.__0vsnprintf$5) refers to printf5.o(i._snputc) for _snputc
    printf5.o(i.__0vsprintf$5) refers to printf5.o(i._printf_core) for _printf_core
    printf5.o(i.__0vsprintf$5) refers to printf5.o(i._sputc) for _sputc
    printf5.o(i._printf_core) refers to uldiv.o(.text) for __aeabi_uldivmod
    printf6.o(i.__0fprintf$6) refers to printf6.o(i._printf_core) for _printf_core
    printf6.o(i.__0fprintf$6) refers to printf.o(i.fputc) for fputc
    printf6.o(i.__0printf$6) refers to printf6.o(i._printf_core) for _printf_core
    printf6.o(i.__0printf$6) refers to printf.o(i.fputc) for fputc
    printf6.o(i.__0printf$6) refers to printf.o(.data) for __stdout
    printf6.o(i.__0snprintf$6) refers to printf6.o(i._printf_core) for _printf_core
    printf6.o(i.__0snprintf$6) refers to printf6.o(i._snputc) for _snputc
    printf6.o(i.__0sprintf$6) refers to printf6.o(i._printf_core) for _printf_core
    printf6.o(i.__0sprintf$6) refers to printf6.o(i._sputc) for _sputc
    printf6.o(i.__0vfprintf$6) refers to printf6.o(i._printf_core) for _printf_core
    printf6.o(i.__0vfprintf$6) refers to printf.o(i.fputc) for fputc
    printf6.o(i.__0vprintf$6) refers to printf6.o(i._printf_core) for _printf_core
    printf6.o(i.__0vprintf$6) refers to printf.o(i.fputc) for fputc
    printf6.o(i.__0vprintf$6) refers to printf.o(.data) for __stdout
    printf6.o(i.__0vsnprintf$6) refers to printf6.o(i._printf_core) for _printf_core
    printf6.o(i.__0vsnprintf$6) refers to printf6.o(i._snputc) for _snputc
    printf6.o(i.__0vsprintf$6) refers to printf6.o(i._printf_core) for _printf_core
    printf6.o(i.__0vsprintf$6) refers to printf6.o(i._sputc) for _sputc
    printf6.o(i._printf_core) refers to printf6.o(i._printf_pre_padding) for _printf_pre_padding
    printf6.o(i._printf_core) refers to uidiv.o(.text) for __aeabi_uidivmod
    printf6.o(i._printf_core) refers to printf6.o(i._printf_post_padding) for _printf_post_padding
    printf7.o(i.__0fprintf$7) refers to printf7.o(i._printf_core) for _printf_core
    printf7.o(i.__0fprintf$7) refers to printf.o(i.fputc) for fputc
    printf7.o(i.__0printf$7) refers to printf7.o(i._printf_core) for _printf_core
    printf7.o(i.__0printf$7) refers to printf.o(i.fputc) for fputc
    printf7.o(i.__0printf$7) refers to printf.o(.data) for __stdout
    printf7.o(i.__0snprintf$7) refers to printf7.o(i._printf_core) for _printf_core
    printf7.o(i.__0snprintf$7) refers to printf7.o(i._snputc) for _snputc
    printf7.o(i.__0sprintf$7) refers to printf7.o(i._printf_core) for _printf_core
    printf7.o(i.__0sprintf$7) refers to printf7.o(i._sputc) for _sputc
    printf7.o(i.__0vfprintf$7) refers to printf7.o(i._printf_core) for _printf_core
    printf7.o(i.__0vfprintf$7) refers to printf.o(i.fputc) for fputc
    printf7.o(i.__0vprintf$7) refers to printf7.o(i._printf_core) for _printf_core
    printf7.o(i.__0vprintf$7) refers to printf.o(i.fputc) for fputc
    printf7.o(i.__0vprintf$7) refers to printf.o(.data) for __stdout
    printf7.o(i.__0vsnprintf$7) refers to printf7.o(i._printf_core) for _printf_core
    printf7.o(i.__0vsnprintf$7) refers to printf7.o(i._snputc) for _snputc
    printf7.o(i.__0vsprintf$7) refers to printf7.o(i._printf_core) for _printf_core
    printf7.o(i.__0vsprintf$7) refers to printf7.o(i._sputc) for _sputc
    printf7.o(i._printf_core) refers to printf7.o(i._printf_pre_padding) for _printf_pre_padding
    printf7.o(i._printf_core) refers to uldiv.o(.text) for __aeabi_uldivmod
    printf7.o(i._printf_core) refers to printf7.o(i._printf_post_padding) for _printf_post_padding
    printf8.o(i.__0fprintf$8) refers to printf8.o(i._printf_core) for _printf_core
    printf8.o(i.__0fprintf$8) refers to printf.o(i.fputc) for fputc
    printf8.o(i.__0printf$8) refers to printf8.o(i._printf_core) for _printf_core
    printf8.o(i.__0printf$8) refers to printf.o(i.fputc) for fputc
    printf8.o(i.__0printf$8) refers to printf.o(.data) for __stdout
    printf8.o(i.__0snprintf$8) refers to printf8.o(i._printf_core) for _printf_core
    printf8.o(i.__0snprintf$8) refers to printf8.o(i._snputc) for _snputc
    printf8.o(i.__0sprintf$8) refers to printf8.o(i._printf_core) for _printf_core
    printf8.o(i.__0sprintf$8) refers to printf8.o(i._sputc) for _sputc
    printf8.o(i.__0vfprintf$8) refers to printf8.o(i._printf_core) for _printf_core
    printf8.o(i.__0vfprintf$8) refers to printf.o(i.fputc) for fputc
    printf8.o(i.__0vprintf$8) refers to printf8.o(i._printf_core) for _printf_core
    printf8.o(i.__0vprintf$8) refers to printf.o(i.fputc) for fputc
    printf8.o(i.__0vprintf$8) refers to printf.o(.data) for __stdout
    printf8.o(i.__0vsnprintf$8) refers to printf8.o(i._printf_core) for _printf_core
    printf8.o(i.__0vsnprintf$8) refers to printf8.o(i._snputc) for _snputc
    printf8.o(i.__0vsprintf$8) refers to printf8.o(i._printf_core) for _printf_core
    printf8.o(i.__0vsprintf$8) refers to printf8.o(i._sputc) for _sputc
    printf8.o(i._printf_core) refers to printf8.o(i._printf_pre_padding) for _printf_pre_padding
    printf8.o(i._printf_core) refers to uldiv.o(.text) for __aeabi_uldivmod
    printf8.o(i._printf_core) refers to printf8.o(i._printf_post_padding) for _printf_post_padding
    printfa.o(i.__0fprintf) refers (Special) to iusefp.o(.text) for __I$use$fp
    printfa.o(i.__0fprintf) refers to printfa.o(i._printf_core) for _printf_core
    printfa.o(i.__0fprintf) refers to printf.o(i.fputc) for fputc
    printfa.o(i.__0printf) refers (Special) to iusefp.o(.text) for __I$use$fp
    printfa.o(i.__0printf) refers to printfa.o(i._printf_core) for _printf_core
    printfa.o(i.__0printf) refers to printf.o(i.fputc) for fputc
    printfa.o(i.__0printf) refers to printf.o(.data) for __stdout
    printfa.o(i.__0snprintf) refers (Special) to iusefp.o(.text) for __I$use$fp
    printfa.o(i.__0snprintf) refers to printfa.o(i._printf_core) for _printf_core
    printfa.o(i.__0snprintf) refers to printfa.o(i._snputc) for _snputc
    printfa.o(i.__0sprintf) refers (Special) to iusefp.o(.text) for __I$use$fp
    printfa.o(i.__0sprintf) refers to printfa.o(i._printf_core) for _printf_core
    printfa.o(i.__0sprintf) refers to printfa.o(i._sputc) for _sputc
    printfa.o(i.__0vfprintf) refers (Special) to iusefp.o(.text) for __I$use$fp
    printfa.o(i.__0vfprintf) refers to printfa.o(i._printf_core) for _printf_core
    printfa.o(i.__0vfprintf) refers to printf.o(i.fputc) for fputc
    printfa.o(i.__0vprintf) refers (Special) to iusefp.o(.text) for __I$use$fp
    printfa.o(i.__0vprintf) refers to printfa.o(i._printf_core) for _printf_core
    printfa.o(i.__0vprintf) refers to printf.o(i.fputc) for fputc
    printfa.o(i.__0vprintf) refers to printf.o(.data) for __stdout
    printfa.o(i.__0vsnprintf) refers (Special) to iusefp.o(.text) for __I$use$fp
    printfa.o(i.__0vsnprintf) refers to printfa.o(i._printf_core) for _printf_core
    printfa.o(i.__0vsnprintf) refers to printfa.o(i._snputc) for _snputc
    printfa.o(i.__0vsprintf) refers (Special) to iusefp.o(.text) for __I$use$fp
    printfa.o(i.__0vsprintf) refers to printfa.o(i._printf_core) for _printf_core
    printfa.o(i.__0vsprintf) refers to printfa.o(i._sputc) for _sputc
    printfa.o(i._fp_digits) refers (Special) to iusefp.o(.text) for __I$use$fp
    printfa.o(i._fp_digits) refers to dmul.o(.text) for __aeabi_dmul
    printfa.o(i._fp_digits) refers to ddiv.o(.text) for __aeabi_ddiv
    printfa.o(i._fp_digits) refers to cdrcmple.o(.text) for __aeabi_cdrcmple
    printfa.o(i._fp_digits) refers to dadd.o(.text) for __aeabi_dadd
    printfa.o(i._fp_digits) refers to dfixul.o(.text) for __aeabi_d2ulz
    printfa.o(i._fp_digits) refers to uldiv.o(.text) for __aeabi_uldivmod
    printfa.o(i._printf_core) refers (Special) to iusefp.o(.text) for __I$use$fp
    printfa.o(i._printf_core) refers to printfa.o(i._printf_pre_padding) for _printf_pre_padding
    printfa.o(i._printf_core) refers to uldiv.o(.text) for __aeabi_uldivmod
    printfa.o(i._printf_core) refers to printfa.o(i._printf_post_padding) for _printf_post_padding
    printfa.o(i._printf_core) refers to printfa.o(i._fp_digits) for _fp_digits
    printfa.o(i._printf_core) refers to uidiv.o(.text) for __aeabi_uidivmod
    printfa.o(i._printf_post_padding) refers (Special) to iusefp.o(.text) for __I$use$fp
    printfa.o(i._printf_pre_padding) refers (Special) to iusefp.o(.text) for __I$use$fp
    printfa.o(i._snputc) refers (Special) to iusefp.o(.text) for __I$use$fp
    printfa.o(i._sputc) refers (Special) to iusefp.o(.text) for __I$use$fp
    entry2.o(.ARM.Collect$$$$00000001) refers to entry2.o(.ARM.Collect$$$$00002712) for __lit__00000000
    entry2.o(.ARM.Collect$$$$00002712) refers to startup_stm32f10x_cl.o(STACK) for __initial_sp
    entry2.o(__vectab_stack_and_reset_area) refers to startup_stm32f10x_cl.o(STACK) for __initial_sp
    entry2.o(__vectab_stack_and_reset_area) refers to entry.o(.ARM.Collect$$$$00000000) for __main
    entry5.o(.ARM.Collect$$$$00000004) refers to init.o(.text) for __scatterload
    entry9a.o(.ARM.Collect$$$$0000000B) refers to main.o(i.main) for main
    entry9b.o(.ARM.Collect$$$$0000000C) refers to main.o(i.main) for main
    uldiv.o(.text) refers to llushr.o(.text) for __aeabi_llsr
    uldiv.o(.text) refers to llshl.o(.text) for __aeabi_llsl
    dadd.o(.text) refers to llshl.o(.text) for __aeabi_llsl
    dadd.o(.text) refers to llsshr.o(.text) for __aeabi_lasr
    dadd.o(.text) refers to depilogue.o(.text) for _double_epilogue
    dmul.o(.text) refers to depilogue.o(.text) for _double_epilogue
    ddiv.o(.text) refers to depilogue.o(.text) for _double_round
    dfixul.o(.text) refers to llushr.o(.text) for __aeabi_llsr
    dfixul.o(.text) refers to llshl.o(.text) for __aeabi_llsl
    init.o(.text) refers to entry5.o(.ARM.Collect$$$$00000004) for __main_after_scatterload
    depilogue.o(.text) refers to llshl.o(.text) for __aeabi_llsl
    depilogue.o(.text) refers to llushr.o(.text) for __aeabi_llsr


==============================================================================

Removing Unused input sections from the image.

    Removing netconf.o(i.Display_Periodic_Handle), (148 bytes).
    Removing netconf.o(i.LwIP_Periodic_Handle), (60 bytes).
    Removing netconf.o(.data), (26 bytes).
    Removing stm32_eth.o(i.ETH_BackPressureActivationCmd), (36 bytes).
    Removing stm32_eth.o(i.ETH_DMAClearFlag), (12 bytes).
    Removing stm32_eth.o(i.ETH_DMAPTPRxDescChainInit), (116 bytes).
    Removing stm32_eth.o(i.ETH_DMAPTPTxDescChainInit), (112 bytes).
    Removing stm32_eth.o(i.ETH_DMARxDescEndOfRingCmd), (22 bytes).
    Removing stm32_eth.o(i.ETH_DMARxDescRingInit), (96 bytes).
    Removing stm32_eth.o(i.ETH_DMARxDescSecondAddressChainedCmd), (22 bytes).
    Removing stm32_eth.o(i.ETH_DMATxDescBufferSizeConfig), (14 bytes).
    Removing stm32_eth.o(i.ETH_DMATxDescCRCCmd), (22 bytes).
    Removing stm32_eth.o(i.ETH_DMATxDescEndOfRingCmd), (22 bytes).
    Removing stm32_eth.o(i.ETH_DMATxDescFrameSegmentConfig), (8 bytes).
    Removing stm32_eth.o(i.ETH_DMATxDescRingInit), (80 bytes).
    Removing stm32_eth.o(i.ETH_DMATxDescSecondAddressChainedCmd), (22 bytes).
    Removing stm32_eth.o(i.ETH_DMATxDescShortFramePaddingCmd), (22 bytes).
    Removing stm32_eth.o(i.ETH_DMATxDescTimeStampCmd), (22 bytes).
    Removing stm32_eth.o(i.ETH_DMATxDescTransmitITConfig), (22 bytes).
    Removing stm32_eth.o(i.ETH_DropRxPkt), (88 bytes).
    Removing stm32_eth.o(i.ETH_EnablePTPTimeStampAddend), (20 bytes).
    Removing stm32_eth.o(i.ETH_EnablePTPTimeStampInterruptTrigger), (20 bytes).
    Removing stm32_eth.o(i.ETH_EnablePTPTimeStampUpdate), (20 bytes).
    Removing stm32_eth.o(i.ETH_GetBufferUnavailableMissedFrameCounter), (12 bytes).
    Removing stm32_eth.o(i.ETH_GetCurrentRxBufferAddress), (12 bytes).
    Removing stm32_eth.o(i.ETH_GetCurrentRxDescStartAddress), (12 bytes).
    Removing stm32_eth.o(i.ETH_GetCurrentTxBufferAddress), (12 bytes).
    Removing stm32_eth.o(i.ETH_GetCurrentTxDescStartAddress), (12 bytes).
    Removing stm32_eth.o(i.ETH_GetDMAFlagStatus), (24 bytes).
    Removing stm32_eth.o(i.ETH_GetDMAITStatus), (24 bytes).
    Removing stm32_eth.o(i.ETH_GetDMAOverflowStatus), (24 bytes).
    Removing stm32_eth.o(i.ETH_GetDMARxDescBufferSize), (20 bytes).
    Removing stm32_eth.o(i.ETH_GetDMARxDescFlagStatus), (18 bytes).
    Removing stm32_eth.o(i.ETH_GetDMATxDescCollisionCount), (10 bytes).
    Removing stm32_eth.o(i.ETH_GetDMATxDescFlagStatus), (18 bytes).
    Removing stm32_eth.o(i.ETH_GetFlowControlBusyStatus), (24 bytes).
    Removing stm32_eth.o(i.ETH_GetFlushTransmitFIFOStatus), (24 bytes).
    Removing stm32_eth.o(i.ETH_GetMACAddress), (40 bytes).
    Removing stm32_eth.o(i.ETH_GetMACFlagStatus), (24 bytes).
    Removing stm32_eth.o(i.ETH_GetMACITStatus), (24 bytes).
    Removing stm32_eth.o(i.ETH_GetMMCITStatus), (68 bytes).
    Removing stm32_eth.o(i.ETH_GetMMCRegister), (12 bytes).
    Removing stm32_eth.o(i.ETH_GetPMTFlagStatus), (24 bytes).
    Removing stm32_eth.o(i.ETH_GetPTPFlagStatus), (24 bytes).
    Removing stm32_eth.o(i.ETH_GetPTPRegister), (12 bytes).
    Removing stm32_eth.o(i.ETH_GetReceiveProcessState), (16 bytes).
    Removing stm32_eth.o(i.ETH_GetRxOverflowMissedFrameCounter), (16 bytes).
    Removing stm32_eth.o(i.ETH_GetTransmitProcessState), (16 bytes).
    Removing stm32_eth.o(i.ETH_GlobalUnicastWakeUpCmd), (36 bytes).
    Removing stm32_eth.o(i.ETH_HandlePTPRxPkt), (260 bytes).
    Removing stm32_eth.o(i.ETH_HandlePTPTxPkt), (320 bytes).
    Removing stm32_eth.o(i.ETH_HandleRxPkt), (204 bytes).
    Removing stm32_eth.o(i.ETH_HandleTxPkt), (184 bytes).
    Removing stm32_eth.o(i.ETH_InitializePTPTimeStamp), (20 bytes).
    Removing stm32_eth.o(i.ETH_InitiatePauseControlFrame), (20 bytes).
    Removing stm32_eth.o(i.ETH_MACAddressFilterConfig), (44 bytes).
    Removing stm32_eth.o(i.ETH_MACAddressMaskBytesFilterConfig), (36 bytes).
    Removing stm32_eth.o(i.ETH_MACAddressPerfectFilterCmd), (44 bytes).
    Removing stm32_eth.o(i.ETH_MACITConfig), (32 bytes).
    Removing stm32_eth.o(i.ETH_MMCCounterFreezeCmd), (44 bytes).
    Removing stm32_eth.o(i.ETH_MMCCounterRolloverCmd), (44 bytes).
    Removing stm32_eth.o(i.ETH_MMCCountersReset), (24 bytes).
    Removing stm32_eth.o(i.ETH_MMCITConfig), (84 bytes).
    Removing stm32_eth.o(i.ETH_MMCResetOnReadCmd), (44 bytes).
    Removing stm32_eth.o(i.ETH_MagicPacketDetectionCmd), (36 bytes).
    Removing stm32_eth.o(i.ETH_PHYLoopBackCmd), (52 bytes).
    Removing stm32_eth.o(i.ETH_PTPTimeStampCmd), (36 bytes).
    Removing stm32_eth.o(i.ETH_PTPUpdateMethodConfig), (36 bytes).
    Removing stm32_eth.o(i.ETH_PowerDownCmd), (36 bytes).
    Removing stm32_eth.o(i.ETH_ResetWakeUpFrameFilterRegisterPointer), (20 bytes).
    Removing stm32_eth.o(i.ETH_ResumeDMAReception), (12 bytes).
    Removing stm32_eth.o(i.ETH_ResumeDMATransmission), (12 bytes).
    Removing stm32_eth.o(i.ETH_SetDMARxDescOwnBit), (10 bytes).
    Removing stm32_eth.o(i.ETH_SetDMATxDescOwnBit), (10 bytes).
    Removing stm32_eth.o(i.ETH_SetPTPSubSecondIncrement), (12 bytes).
    Removing stm32_eth.o(i.ETH_SetPTPTargetTime), (16 bytes).
    Removing stm32_eth.o(i.ETH_SetPTPTimeStampAddend), (12 bytes).
    Removing stm32_eth.o(i.ETH_SetPTPTimeStampUpdate), (24 bytes).
    Removing stm32_eth.o(i.ETH_SetWakeUpFrameFilterRegister), (28 bytes).
    Removing stm32_eth.o(i.ETH_WakeUpFrameDetectionCmd), (36 bytes).
    Removing printf.o(i._sys_exit), (6 bytes).
    Removing printf.o(i.fgetc), (32 bytes).
    Removing usart1.o(i.usart1_FreeBuff), (76 bytes).
    Removing usart1.o(i.usart1_Receive), (84 bytes).
    Removing usart1.o(i.usart1_Send), (84 bytes).
    Removing delay.o(i.delay_s), (24 bytes).
    Removing stm32_config.o(i.SoftReset), (52 bytes).
    Removing os_core.o(i.OSSchedLock), (64 bytes).
    Removing os_core.o(i.OSSchedUnlock), (96 bytes).
    Removing os_core.o(i.OSVersion), (6 bytes).
    Removing os_core.o(i.OS_Dummy), (2 bytes).
    Removing os_core.o(i.OS_EventTaskRdy), (132 bytes).
    Removing os_core.o(i.OS_EventTaskRemove), (42 bytes).
    Removing os_core.o(i.OS_EventTaskWait), (124 bytes).
    Removing os_core.o(i.OS_EventWaitListInit), (28 bytes).
    Removing os_core.o(i.OS_MemCopy), (20 bytes).
    Removing os_core.o(i.OS_StrLen), (20 bytes).
    Removing os_flag.o(i.OSFlagAccept), (252 bytes).
    Removing os_flag.o(i.OSFlagCreate), (100 bytes).
    Removing os_flag.o(i.OSFlagDel), (228 bytes).
    Removing os_flag.o(i.OSFlagNameGet), (84 bytes).
    Removing os_flag.o(i.OSFlagNameSet), (72 bytes).
    Removing os_flag.o(i.OSFlagPend), (596 bytes).
    Removing os_flag.o(i.OSFlagPendGetFlagsRdy), (32 bytes).
    Removing os_flag.o(i.OSFlagPost), (312 bytes).
    Removing os_flag.o(i.OSFlagQuery), (48 bytes).
    Removing os_flag.o(i.OS_FlagBlock), (164 bytes).
    Removing os_flag.o(i.OS_FlagTaskRdy), (92 bytes).
    Removing os_flag.o(i.OS_FlagUnlink), (36 bytes).
    Removing os_mbox.o(i.OSMboxAccept), (38 bytes).
    Removing os_mbox.o(i.OSMboxCreate), (76 bytes).
    Removing os_mbox.o(i.OSMboxDel), (208 bytes).
    Removing os_mbox.o(i.OSMboxPend), (260 bytes).
    Removing os_mbox.o(i.OSMboxPendAbort), (128 bytes).
    Removing os_mbox.o(i.OSMboxPost), (80 bytes).
    Removing os_mbox.o(i.OSMboxPostOpt), (120 bytes).
    Removing os_mbox.o(i.OSMboxQuery), (76 bytes).
    Removing os_mutex.o(i.OSMutexAccept), (144 bytes).
    Removing os_mutex.o(i.OSMutexCreate), (148 bytes).
    Removing os_mutex.o(i.OSMutexDel), (280 bytes).
    Removing os_mutex.o(i.OSMutexPend), (568 bytes).
    Removing os_mutex.o(i.OSMutexPost), (200 bytes).
    Removing os_mutex.o(i.OSMutexQuery), (112 bytes).
    Removing os_mutex.o(i.OSMutex_RdyAtPrio), (132 bytes).
    Removing os_q.o(i.OSQAccept), (88 bytes).
    Removing os_q.o(i.OSQCreate), (152 bytes).
    Removing os_q.o(i.OSQDel), (248 bytes).
    Removing os_q.o(i.OSQFlush), (36 bytes).
    Removing os_q.o(i.OSQPend), (284 bytes).
    Removing os_q.o(i.OSQPendAbort), (128 bytes).
    Removing os_q.o(i.OSQPost), (114 bytes).
    Removing os_q.o(i.OSQPostFront), (116 bytes).
    Removing os_q.o(i.OSQPostOpt), (182 bytes).
    Removing os_q.o(i.OSQQuery), (98 bytes).
    Removing os_sem.o(i.OSSemAccept), (42 bytes).
    Removing os_sem.o(i.OSSemCreate), (76 bytes).
    Removing os_sem.o(i.OSSemDel), (208 bytes).
    Removing os_sem.o(i.OSSemPend), (236 bytes).
    Removing os_sem.o(i.OSSemPendAbort), (128 bytes).
    Removing os_sem.o(i.OSSemPost), (88 bytes).
    Removing os_sem.o(i.OSSemQuery), (76 bytes).
    Removing os_sem.o(i.OSSemSet), (66 bytes).
    Removing os_task.o(i.OSTaskChangePrio), (328 bytes).
    Removing os_task.o(i.OSTaskDel), (340 bytes).
    Removing os_task.o(i.OSTaskDelReq), (108 bytes).
    Removing os_task.o(i.OSTaskNameGet), (128 bytes).
    Removing os_task.o(i.OSTaskQuery), (92 bytes).
    Removing os_task.o(i.OSTaskRegGet), (68 bytes).
    Removing os_task.o(i.OSTaskRegSet), (72 bytes).
    Removing os_task.o(i.OSTaskResume), (172 bytes).
    Removing os_task.o(i.OS_TaskReturn), (24 bytes).
    Removing os_time.o(i.OSTimeDlyHMSM), (96 bytes).
    Removing os_time.o(i.OSTimeDlyResume), (180 bytes).
    Removing os_time.o(i.OSTimeGet), (28 bytes).
    Removing os_time.o(i.OSTimeSet), (28 bytes).
    Removing os_cpu_c.o(i.OSTaskDelHook), (2 bytes).
    Removing os_cpu_c.o(i.OSTaskReturnHook), (2 bytes).
    Removing os_cpu_c.o(.data), (4 bytes).
    Removing os_dbg.o(.constdata), (2 bytes).
    Removing init.o(i.lwip_init), (12 bytes).
    Removing mem.o(i.mem_calloc), (34 bytes).
    Removing netif.o(i.netif_find), (68 bytes).
    Removing netif.o(i.netif_remove), (84 bytes).
    Removing netif.o(i.netif_set_down), (24 bytes).
    Removing pbuf.o(i.pbuf_coalesce), (66 bytes).
    Removing pbuf.o(i.pbuf_dechain), (84 bytes).
    Removing pbuf.o(i.pbuf_take), (138 bytes).
    Removing tcp.o(i.tcp_fasttmr), (116 bytes).
    Removing tcp.o(i.tcp_slowtmr), (788 bytes).
    Removing tcp.o(i.tcp_tmr), (36 bytes).
    Removing tcp_out.o(i.tcp_keepalive), (92 bytes).
    Removing tcp_out.o(i.tcp_rexmit_rto), (58 bytes).
    Removing tcp_out.o(i.tcp_zero_window_probe), (102 bytes).
    Removing inet.o(i.inet_addr), (24 bytes).
    Removing inet.o(i.inet_aton), (336 bytes).
    Removing inet.o(i.inet_ntoa), (116 bytes).
    Removing inet.o(.bss), (16 bytes).
    Removing inet_chksum.o(i.inet_chksum_pseudo), (162 bytes).
    Removing ip.o(i.ip_current_header), (12 bytes).
    Removing ip.o(i.ip_current_netif), (12 bytes).
    Removing ip_frag.o(i.ip_reass_tmr), (52 bytes).
    Removing etharp.o(i.etharp_find_addr), (84 bytes).
    Removing etharp.o(i.etharp_tmr), (160 bytes).
    Removing core_cm3.o(.emb_text), (32 bytes).
    Removing misc.o(i.NVIC_SystemLPConfig), (32 bytes).
    Removing stm32f10x_fsmc.o(i.FSMC_ClearFlag), (64 bytes).
    Removing stm32f10x_fsmc.o(i.FSMC_ClearITPendingBit), (72 bytes).
    Removing stm32f10x_fsmc.o(i.FSMC_GetECC), (28 bytes).
    Removing stm32f10x_fsmc.o(i.FSMC_GetFlagStatus), (56 bytes).
    Removing stm32f10x_fsmc.o(i.FSMC_GetITStatus), (68 bytes).
    Removing stm32f10x_fsmc.o(i.FSMC_ITConfig), (128 bytes).
    Removing stm32f10x_fsmc.o(i.FSMC_NANDCmd), (92 bytes).
    Removing stm32f10x_fsmc.o(i.FSMC_NANDDeInit), (68 bytes).
    Removing stm32f10x_fsmc.o(i.FSMC_NANDECCCmd), (92 bytes).
    Removing stm32f10x_fsmc.o(i.FSMC_NANDInit), (136 bytes).
    Removing stm32f10x_fsmc.o(i.FSMC_NANDStructInit), (54 bytes).
    Removing stm32f10x_fsmc.o(i.FSMC_NORSRAMCmd), (52 bytes).
    Removing stm32f10x_fsmc.o(i.FSMC_NORSRAMDeInit), (54 bytes).
    Removing stm32f10x_fsmc.o(i.FSMC_NORSRAMInit), (230 bytes).
    Removing stm32f10x_fsmc.o(i.FSMC_NORSRAMStructInit), (114 bytes).
    Removing stm32f10x_fsmc.o(i.FSMC_PCCARDCmd), (48 bytes).
    Removing stm32f10x_fsmc.o(i.FSMC_PCCARDDeInit), (40 bytes).
    Removing stm32f10x_fsmc.o(i.FSMC_PCCARDInit), (132 bytes).
    Removing stm32f10x_fsmc.o(i.FSMC_PCCARDStructInit), (60 bytes).
    Removing stm32f10x_gpio.o(i.GPIO_AFIODeInit), (20 bytes).
    Removing stm32f10x_gpio.o(i.GPIO_DeInit), (200 bytes).
    Removing stm32f10x_gpio.o(i.GPIO_EXTILineConfig), (64 bytes).
    Removing stm32f10x_gpio.o(i.GPIO_EventOutputCmd), (12 bytes).
    Removing stm32f10x_gpio.o(i.GPIO_EventOutputConfig), (32 bytes).
    Removing stm32f10x_gpio.o(i.GPIO_PinLockConfig), (18 bytes).
    Removing stm32f10x_gpio.o(i.GPIO_ReadInputData), (8 bytes).
    Removing stm32f10x_gpio.o(i.GPIO_ReadInputDataBit), (18 bytes).
    Removing stm32f10x_gpio.o(i.GPIO_ReadOutputData), (8 bytes).
    Removing stm32f10x_gpio.o(i.GPIO_ReadOutputDataBit), (18 bytes).
    Removing stm32f10x_gpio.o(i.GPIO_ResetBits), (4 bytes).
    Removing stm32f10x_gpio.o(i.GPIO_SetBits), (4 bytes).
    Removing stm32f10x_gpio.o(i.GPIO_StructInit), (16 bytes).
    Removing stm32f10x_gpio.o(i.GPIO_Write), (4 bytes).
    Removing stm32f10x_gpio.o(i.GPIO_WriteBit), (10 bytes).
    Removing stm32f10x_rcc.o(i.RCC_ADCCLKConfig), (24 bytes).
    Removing stm32f10x_rcc.o(i.RCC_APB1PeriphResetCmd), (32 bytes).
    Removing stm32f10x_rcc.o(i.RCC_APB2PeriphResetCmd), (32 bytes).
    Removing stm32f10x_rcc.o(i.RCC_AdjustHSICalibrationValue), (24 bytes).
    Removing stm32f10x_rcc.o(i.RCC_BackupResetCmd), (12 bytes).
    Removing stm32f10x_rcc.o(i.RCC_ClearFlag), (20 bytes).
    Removing stm32f10x_rcc.o(i.RCC_ClearITPendingBit), (12 bytes).
    Removing stm32f10x_rcc.o(i.RCC_ClockSecuritySystemCmd), (12 bytes).
    Removing stm32f10x_rcc.o(i.RCC_DeInit), (92 bytes).
    Removing stm32f10x_rcc.o(i.RCC_GetITStatus), (24 bytes).
    Removing stm32f10x_rcc.o(i.RCC_GetSYSCLKSource), (16 bytes).
    Removing stm32f10x_rcc.o(i.RCC_HCLKConfig), (24 bytes).
    Removing stm32f10x_rcc.o(i.RCC_HSEConfig), (76 bytes).
    Removing stm32f10x_rcc.o(i.RCC_HSICmd), (12 bytes).
    Removing stm32f10x_rcc.o(i.RCC_I2S2CLKConfig), (12 bytes).
    Removing stm32f10x_rcc.o(i.RCC_I2S3CLKConfig), (12 bytes).
    Removing stm32f10x_rcc.o(i.RCC_ITConfig), (32 bytes).
    Removing stm32f10x_rcc.o(i.RCC_LSEConfig), (52 bytes).
    Removing stm32f10x_rcc.o(i.RCC_LSICmd), (12 bytes).
    Removing stm32f10x_rcc.o(i.RCC_OTGFSCLKConfig), (12 bytes).
    Removing stm32f10x_rcc.o(i.RCC_PCLK1Config), (24 bytes).
    Removing stm32f10x_rcc.o(i.RCC_PCLK2Config), (24 bytes).
    Removing stm32f10x_rcc.o(i.RCC_PLL2Cmd), (12 bytes).
    Removing stm32f10x_rcc.o(i.RCC_PLL2Config), (24 bytes).
    Removing stm32f10x_rcc.o(i.RCC_PLLCmd), (12 bytes).
    Removing stm32f10x_rcc.o(i.RCC_PLLConfig), (28 bytes).
    Removing stm32f10x_rcc.o(i.RCC_PREDIV1Config), (32 bytes).
    Removing stm32f10x_rcc.o(i.RCC_PREDIV2Config), (24 bytes).
    Removing stm32f10x_rcc.o(i.RCC_RTCCLKCmd), (12 bytes).
    Removing stm32f10x_rcc.o(i.RCC_RTCCLKConfig), (16 bytes).
    Removing stm32f10x_rcc.o(i.RCC_SYSCLKConfig), (24 bytes).
    Removing stm32f10x_rcc.o(i.RCC_WaitForHSEStartUp), (56 bytes).
    Removing stm32f10x_usart.o(i.USART_ClockInit), (34 bytes).
    Removing stm32f10x_usart.o(i.USART_ClockStructInit), (12 bytes).
    Removing stm32f10x_usart.o(i.USART_DMACmd), (18 bytes).
    Removing stm32f10x_usart.o(i.USART_DeInit), (156 bytes).
    Removing stm32f10x_usart.o(i.USART_HalfDuplexCmd), (24 bytes).
    Removing stm32f10x_usart.o(i.USART_IrDACmd), (24 bytes).
    Removing stm32f10x_usart.o(i.USART_IrDAConfig), (18 bytes).
    Removing stm32f10x_usart.o(i.USART_LINBreakDetectLengthConfig), (18 bytes).
    Removing stm32f10x_usart.o(i.USART_LINCmd), (24 bytes).
    Removing stm32f10x_usart.o(i.USART_OneBitMethodCmd), (24 bytes).
    Removing stm32f10x_usart.o(i.USART_OverSampling8Cmd), (22 bytes).
    Removing stm32f10x_usart.o(i.USART_ReceiverWakeUpCmd), (24 bytes).
    Removing stm32f10x_usart.o(i.USART_SendBreak), (10 bytes).
    Removing stm32f10x_usart.o(i.USART_SetAddress), (18 bytes).
    Removing stm32f10x_usart.o(i.USART_SetGuardTime), (16 bytes).
    Removing stm32f10x_usart.o(i.USART_SetPrescaler), (16 bytes).
    Removing stm32f10x_usart.o(i.USART_SmartCardCmd), (24 bytes).
    Removing stm32f10x_usart.o(i.USART_SmartCardNACKCmd), (24 bytes).
    Removing stm32f10x_usart.o(i.USART_StructInit), (24 bytes).
    Removing stm32f10x_usart.o(i.USART_WakeUpConfig), (18 bytes).
    Removing stm32f10x_spi.o(i.I2S_Cmd), (24 bytes).
    Removing stm32f10x_spi.o(i.I2S_Init), (304 bytes).
    Removing stm32f10x_spi.o(i.I2S_StructInit), (20 bytes).
    Removing stm32f10x_spi.o(i.SPI_BiDirectionalLineConfig), (28 bytes).
    Removing stm32f10x_spi.o(i.SPI_CalculateCRC), (24 bytes).
    Removing stm32f10x_spi.o(i.SPI_Cmd), (24 bytes).
    Removing stm32f10x_spi.o(i.SPI_DataSizeConfig), (18 bytes).
    Removing stm32f10x_spi.o(i.SPI_GetCRC), (16 bytes).
    Removing stm32f10x_spi.o(i.SPI_GetCRCPolynomial), (6 bytes).
    Removing stm32f10x_spi.o(i.SPI_I2S_ClearFlag), (6 bytes).
    Removing stm32f10x_spi.o(i.SPI_I2S_ClearITPendingBit), (20 bytes).
    Removing stm32f10x_spi.o(i.SPI_I2S_DMACmd), (18 bytes).
    Removing stm32f10x_spi.o(i.SPI_I2S_DeInit), (88 bytes).
    Removing stm32f10x_spi.o(i.SPI_I2S_GetFlagStatus), (18 bytes).
    Removing stm32f10x_spi.o(i.SPI_I2S_GetITStatus), (52 bytes).
    Removing stm32f10x_spi.o(i.SPI_I2S_ITConfig), (32 bytes).
    Removing stm32f10x_spi.o(i.SPI_I2S_ReceiveData), (6 bytes).
    Removing stm32f10x_spi.o(i.SPI_I2S_SendData), (4 bytes).
    Removing stm32f10x_spi.o(i.SPI_Init), (60 bytes).
    Removing stm32f10x_spi.o(i.SPI_NSSInternalSoftwareConfig), (30 bytes).
    Removing stm32f10x_spi.o(i.SPI_SSOutputCmd), (24 bytes).
    Removing stm32f10x_spi.o(i.SPI_StructInit), (24 bytes).
    Removing stm32f10x_spi.o(i.SPI_TransmitCRC), (10 bytes).
    Removing stm32f10x_adc.o(i.ADC_AnalogWatchdogCmd), (20 bytes).
    Removing stm32f10x_adc.o(i.ADC_AnalogWatchdogSingleChannelConfig), (16 bytes).
    Removing stm32f10x_adc.o(i.ADC_AnalogWatchdogThresholdsConfig), (6 bytes).
    Removing stm32f10x_adc.o(i.ADC_AutoInjectedConvCmd), (22 bytes).
    Removing stm32f10x_adc.o(i.ADC_ClearFlag), (6 bytes).
    Removing stm32f10x_adc.o(i.ADC_ClearITPendingBit), (10 bytes).
    Removing stm32f10x_adc.o(i.ADC_Cmd), (22 bytes).
    Removing stm32f10x_adc.o(i.ADC_DMACmd), (22 bytes).
    Removing stm32f10x_adc.o(i.ADC_DeInit), (92 bytes).
    Removing stm32f10x_adc.o(i.ADC_DiscModeChannelCountConfig), (24 bytes).
    Removing stm32f10x_adc.o(i.ADC_DiscModeCmd), (22 bytes).
    Removing stm32f10x_adc.o(i.ADC_ExternalTrigConvCmd), (22 bytes).
    Removing stm32f10x_adc.o(i.ADC_ExternalTrigInjectedConvCmd), (22 bytes).
    Removing stm32f10x_adc.o(i.ADC_ExternalTrigInjectedConvConfig), (16 bytes).
    Removing stm32f10x_adc.o(i.ADC_GetCalibrationStatus), (20 bytes).
    Removing stm32f10x_adc.o(i.ADC_GetConversionValue), (8 bytes).
    Removing stm32f10x_adc.o(i.ADC_GetDualModeConversionValue), (12 bytes).
    Removing stm32f10x_adc.o(i.ADC_GetFlagStatus), (18 bytes).
    Removing stm32f10x_adc.o(i.ADC_GetITStatus), (36 bytes).
    Removing stm32f10x_adc.o(i.ADC_GetInjectedConversionValue), (28 bytes).
    Removing stm32f10x_adc.o(i.ADC_GetResetCalibrationStatus), (20 bytes).
    Removing stm32f10x_adc.o(i.ADC_GetSoftwareStartConvStatus), (20 bytes).
    Removing stm32f10x_adc.o(i.ADC_GetSoftwareStartInjectedConvCmdStatus), (20 bytes).
    Removing stm32f10x_adc.o(i.ADC_ITConfig), (24 bytes).
    Removing stm32f10x_adc.o(i.ADC_Init), (80 bytes).
    Removing stm32f10x_adc.o(i.ADC_InjectedChannelConfig), (130 bytes).
    Removing stm32f10x_adc.o(i.ADC_InjectedDiscModeCmd), (22 bytes).
    Removing stm32f10x_adc.o(i.ADC_InjectedSequencerLengthConfig), (24 bytes).
    Removing stm32f10x_adc.o(i.ADC_RegularChannelConfig), (184 bytes).
    Removing stm32f10x_adc.o(i.ADC_ResetCalibration), (10 bytes).
    Removing stm32f10x_adc.o(i.ADC_SetInjectedOffset), (20 bytes).
    Removing stm32f10x_adc.o(i.ADC_SoftwareStartConvCmd), (22 bytes).
    Removing stm32f10x_adc.o(i.ADC_SoftwareStartInjectedConvCmd), (22 bytes).
    Removing stm32f10x_adc.o(i.ADC_StartCalibration), (10 bytes).
    Removing stm32f10x_adc.o(i.ADC_StructInit), (18 bytes).
    Removing stm32f10x_adc.o(i.ADC_TempSensorVrefintCmd), (36 bytes).
    Removing stm32f10x_exti.o(i.EXTI_ClearFlag), (12 bytes).
    Removing stm32f10x_exti.o(i.EXTI_ClearITPendingBit), (12 bytes).
    Removing stm32f10x_exti.o(i.EXTI_DeInit), (36 bytes).
    Removing stm32f10x_exti.o(i.EXTI_GenerateSWInterrupt), (16 bytes).
    Removing stm32f10x_exti.o(i.EXTI_GetFlagStatus), (24 bytes).
    Removing stm32f10x_exti.o(i.EXTI_GetITStatus), (40 bytes).
    Removing stm32f10x_exti.o(i.EXTI_Init), (148 bytes).
    Removing stm32f10x_exti.o(i.EXTI_StructInit), (16 bytes).
    Removing stm32f10x_tim.o(i.TI1_Config), (128 bytes).
    Removing stm32f10x_tim.o(i.TI2_Config), (152 bytes).
    Removing stm32f10x_tim.o(i.TI3_Config), (144 bytes).
    Removing stm32f10x_tim.o(i.TI4_Config), (152 bytes).
    Removing stm32f10x_tim.o(i.TIM_ARRPreloadConfig), (24 bytes).
    Removing stm32f10x_tim.o(i.TIM_BDTRConfig), (32 bytes).
    Removing stm32f10x_tim.o(i.TIM_BDTRStructInit), (18 bytes).
    Removing stm32f10x_tim.o(i.TIM_CCPreloadControl), (24 bytes).
    Removing stm32f10x_tim.o(i.TIM_CCxCmd), (30 bytes).
    Removing stm32f10x_tim.o(i.TIM_CCxNCmd), (30 bytes).
    Removing stm32f10x_tim.o(i.TIM_ClearFlag), (6 bytes).
    Removing stm32f10x_tim.o(i.TIM_ClearITPendingBit), (6 bytes).
    Removing stm32f10x_tim.o(i.TIM_ClearOC1Ref), (18 bytes).
    Removing stm32f10x_tim.o(i.TIM_ClearOC2Ref), (24 bytes).
    Removing stm32f10x_tim.o(i.TIM_ClearOC3Ref), (18 bytes).
    Removing stm32f10x_tim.o(i.TIM_ClearOC4Ref), (24 bytes).
    Removing stm32f10x_tim.o(i.TIM_Cmd), (24 bytes).
    Removing stm32f10x_tim.o(i.TIM_CounterModeConfig), (18 bytes).
    Removing stm32f10x_tim.o(i.TIM_CtrlPWMOutputs), (30 bytes).
    Removing stm32f10x_tim.o(i.TIM_DMACmd), (18 bytes).
    Removing stm32f10x_tim.o(i.TIM_DMAConfig), (10 bytes).
    Removing stm32f10x_tim.o(i.TIM_DeInit), (488 bytes).
    Removing stm32f10x_tim.o(i.TIM_ETRClockMode1Config), (54 bytes).
    Removing stm32f10x_tim.o(i.TIM_ETRClockMode2Config), (32 bytes).
    Removing stm32f10x_tim.o(i.TIM_ETRConfig), (28 bytes).
    Removing stm32f10x_tim.o(i.TIM_EncoderInterfaceConfig), (66 bytes).
    Removing stm32f10x_tim.o(i.TIM_ForcedOC1Config), (18 bytes).
    Removing stm32f10x_tim.o(i.TIM_ForcedOC2Config), (26 bytes).
    Removing stm32f10x_tim.o(i.TIM_ForcedOC3Config), (18 bytes).
    Removing stm32f10x_tim.o(i.TIM_ForcedOC4Config), (26 bytes).
    Removing stm32f10x_tim.o(i.TIM_GenerateEvent), (4 bytes).
    Removing stm32f10x_tim.o(i.TIM_GetCapture1), (6 bytes).
    Removing stm32f10x_tim.o(i.TIM_GetCapture2), (6 bytes).
    Removing stm32f10x_tim.o(i.TIM_GetCapture3), (6 bytes).
    Removing stm32f10x_tim.o(i.TIM_GetCapture4), (8 bytes).
    Removing stm32f10x_tim.o(i.TIM_GetCounter), (6 bytes).
    Removing stm32f10x_tim.o(i.TIM_GetFlagStatus), (18 bytes).
    Removing stm32f10x_tim.o(i.TIM_GetITStatus), (34 bytes).
    Removing stm32f10x_tim.o(i.TIM_GetPrescaler), (6 bytes).
    Removing stm32f10x_tim.o(i.TIM_ICInit), (172 bytes).
    Removing stm32f10x_tim.o(i.TIM_ICStructInit), (18 bytes).
    Removing stm32f10x_tim.o(i.TIM_ITConfig), (18 bytes).
    Removing stm32f10x_tim.o(i.TIM_ITRxExternalClockConfig), (24 bytes).
    Removing stm32f10x_tim.o(i.TIM_InternalClockConfig), (12 bytes).
    Removing stm32f10x_tim.o(i.TIM_OC1FastConfig), (18 bytes).
    Removing stm32f10x_tim.o(i.TIM_OC1Init), (152 bytes).
    Removing stm32f10x_tim.o(i.TIM_OC1NPolarityConfig), (18 bytes).
    Removing stm32f10x_tim.o(i.TIM_OC1PolarityConfig), (18 bytes).
    Removing stm32f10x_tim.o(i.TIM_OC1PreloadConfig), (18 bytes).
    Removing stm32f10x_tim.o(i.TIM_OC2FastConfig), (26 bytes).
    Removing stm32f10x_tim.o(i.TIM_OC2Init), (164 bytes).
    Removing stm32f10x_tim.o(i.TIM_OC2NPolarityConfig), (26 bytes).
    Removing stm32f10x_tim.o(i.TIM_OC2PolarityConfig), (26 bytes).
    Removing stm32f10x_tim.o(i.TIM_OC2PreloadConfig), (26 bytes).
    Removing stm32f10x_tim.o(i.TIM_OC3FastConfig), (18 bytes).
    Removing stm32f10x_tim.o(i.TIM_OC3Init), (160 bytes).
    Removing stm32f10x_tim.o(i.TIM_OC3NPolarityConfig), (26 bytes).
    Removing stm32f10x_tim.o(i.TIM_OC3PolarityConfig), (26 bytes).
    Removing stm32f10x_tim.o(i.TIM_OC3PreloadConfig), (18 bytes).
    Removing stm32f10x_tim.o(i.TIM_OC4FastConfig), (26 bytes).
    Removing stm32f10x_tim.o(i.TIM_OC4Init), (124 bytes).
    Removing stm32f10x_tim.o(i.TIM_OC4PolarityConfig), (26 bytes).
    Removing stm32f10x_tim.o(i.TIM_OC4PreloadConfig), (26 bytes).
    Removing stm32f10x_tim.o(i.TIM_OCStructInit), (20 bytes).
    Removing stm32f10x_tim.o(i.TIM_PWMIConfig), (124 bytes).
    Removing stm32f10x_tim.o(i.TIM_PrescalerConfig), (6 bytes).
    Removing stm32f10x_tim.o(i.TIM_SelectCCDMA), (24 bytes).
    Removing stm32f10x_tim.o(i.TIM_SelectCOM), (24 bytes).
    Removing stm32f10x_tim.o(i.TIM_SelectHallSensor), (24 bytes).
    Removing stm32f10x_tim.o(i.TIM_SelectInputTrigger), (18 bytes).
    Removing stm32f10x_tim.o(i.TIM_SelectMasterSlaveMode), (18 bytes).
    Removing stm32f10x_tim.o(i.TIM_SelectOCxM), (82 bytes).
    Removing stm32f10x_tim.o(i.TIM_SelectOnePulseMode), (18 bytes).
    Removing stm32f10x_tim.o(i.TIM_SelectOutputTrigger), (18 bytes).
    Removing stm32f10x_tim.o(i.TIM_SelectSlaveMode), (18 bytes).
    Removing stm32f10x_tim.o(i.TIM_SetAutoreload), (4 bytes).
    Removing stm32f10x_tim.o(i.TIM_SetClockDivision), (18 bytes).
    Removing stm32f10x_tim.o(i.TIM_SetCompare1), (4 bytes).
    Removing stm32f10x_tim.o(i.TIM_SetCompare2), (4 bytes).
    Removing stm32f10x_tim.o(i.TIM_SetCompare3), (4 bytes).
    Removing stm32f10x_tim.o(i.TIM_SetCompare4), (6 bytes).
    Removing stm32f10x_tim.o(i.TIM_SetCounter), (4 bytes).
    Removing stm32f10x_tim.o(i.TIM_SetIC1Prescaler), (18 bytes).
    Removing stm32f10x_tim.o(i.TIM_SetIC2Prescaler), (26 bytes).
    Removing stm32f10x_tim.o(i.TIM_SetIC3Prescaler), (18 bytes).
    Removing stm32f10x_tim.o(i.TIM_SetIC4Prescaler), (26 bytes).
    Removing stm32f10x_tim.o(i.TIM_TIxExternalClockConfig), (62 bytes).
    Removing stm32f10x_tim.o(i.TIM_TimeBaseInit), (164 bytes).
    Removing stm32f10x_tim.o(i.TIM_TimeBaseStructInit), (18 bytes).
    Removing stm32f10x_tim.o(i.TIM_UpdateDisableConfig), (24 bytes).
    Removing stm32f10x_tim.o(i.TIM_UpdateRequestConfig), (24 bytes).
    Removing stm32f10x_i2c.o(i.I2C_ARPCmd), (24 bytes).
    Removing stm32f10x_i2c.o(i.I2C_AcknowledgeConfig), (24 bytes).
    Removing stm32f10x_i2c.o(i.I2C_CalculatePEC), (24 bytes).
    Removing stm32f10x_i2c.o(i.I2C_CheckEvent), (42 bytes).
    Removing stm32f10x_i2c.o(i.I2C_ClearFlag), (12 bytes).
    Removing stm32f10x_i2c.o(i.I2C_ClearITPendingBit), (12 bytes).
    Removing stm32f10x_i2c.o(i.I2C_Cmd), (24 bytes).
    Removing stm32f10x_i2c.o(i.I2C_DMACmd), (24 bytes).
    Removing stm32f10x_i2c.o(i.I2C_DMALastTransferCmd), (24 bytes).
    Removing stm32f10x_i2c.o(i.I2C_DeInit), (56 bytes).
    Removing stm32f10x_i2c.o(i.I2C_DualAddressCmd), (24 bytes).
    Removing stm32f10x_i2c.o(i.I2C_FastModeDutyCycleConfig), (28 bytes).
    Removing stm32f10x_i2c.o(i.I2C_GeneralCallCmd), (24 bytes).
    Removing stm32f10x_i2c.o(i.I2C_GenerateSTART), (24 bytes).
    Removing stm32f10x_i2c.o(i.I2C_GenerateSTOP), (24 bytes).
    Removing stm32f10x_i2c.o(i.I2C_GetFlagStatus), (58 bytes).
    Removing stm32f10x_i2c.o(i.I2C_GetITStatus), (38 bytes).
    Removing stm32f10x_i2c.o(i.I2C_GetLastEvent), (26 bytes).
    Removing stm32f10x_i2c.o(i.I2C_GetPEC), (8 bytes).
    Removing stm32f10x_i2c.o(i.I2C_ITConfig), (18 bytes).
    Removing stm32f10x_i2c.o(i.I2C_Init), (236 bytes).
    Removing stm32f10x_i2c.o(i.I2C_NACKPositionConfig), (28 bytes).
    Removing stm32f10x_i2c.o(i.I2C_OwnAddress2Config), (22 bytes).
    Removing stm32f10x_i2c.o(i.I2C_PECPositionConfig), (28 bytes).
    Removing stm32f10x_i2c.o(i.I2C_ReadRegister), (22 bytes).
    Removing stm32f10x_i2c.o(i.I2C_ReceiveData), (8 bytes).
    Removing stm32f10x_i2c.o(i.I2C_SMBusAlertConfig), (28 bytes).
    Removing stm32f10x_i2c.o(i.I2C_Send7bitAddress), (18 bytes).
    Removing stm32f10x_i2c.o(i.I2C_SendData), (4 bytes).
    Removing stm32f10x_i2c.o(i.I2C_SoftwareResetCmd), (22 bytes).
    Removing stm32f10x_i2c.o(i.I2C_StretchClockCmd), (24 bytes).
    Removing stm32f10x_i2c.o(i.I2C_StructInit), (30 bytes).
    Removing stm32f10x_i2c.o(i.I2C_TransmitPEC), (24 bytes).
    Removing stm32f10x_iwdg.o(i.IWDG_Enable), (16 bytes).
    Removing stm32f10x_iwdg.o(i.IWDG_GetFlagStatus), (24 bytes).
    Removing stm32f10x_iwdg.o(i.IWDG_ReloadCounter), (16 bytes).
    Removing stm32f10x_iwdg.o(i.IWDG_SetPrescaler), (12 bytes).
    Removing stm32f10x_iwdg.o(i.IWDG_SetReload), (12 bytes).
    Removing stm32f10x_iwdg.o(i.IWDG_WriteAccessCmd), (12 bytes).
    Removing startup_stm32f10x_cl.o(HEAP), (512 bytes).
    Removing system_stm32f10x.o(i.SystemCoreClockUpdate), (256 bytes).
    Removing dadd.o(.text), (334 bytes).
    Removing dmul.o(.text), (228 bytes).
    Removing ddiv.o(.text), (222 bytes).
    Removing dfixul.o(.text), (48 bytes).
    Removing cdrcmple.o(.text), (48 bytes).
    Removing depilogue.o(.text), (186 bytes).

476 unused section(s) (total 28052 bytes) removed from the image.

==============================================================================

Image Symbol Table

    Local Symbols

    Symbol Name                              Value     Ov Type        Size  Object(Section)

    ../clib/../cmprslib/zerorunl2.c          0x00000000   Number         0  __dczerorl2.o ABSOLUTE
    ../clib/microlib/division.c              0x00000000   Number         0  uldiv.o ABSOLUTE
    ../clib/microlib/division.c              0x00000000   Number         0  uidiv.o ABSOLUTE
    ../clib/microlib/init/entry.s            0x00000000   Number         0  entry8b.o ABSOLUTE
    ../clib/microlib/init/entry.s            0x00000000   Number         0  entry2.o ABSOLUTE
    ../clib/microlib/init/entry.s            0x00000000   Number         0  entry10a.o ABSOLUTE
    ../clib/microlib/init/entry.s            0x00000000   Number         0  entry9b.o ABSOLUTE
    ../clib/microlib/init/entry.s            0x00000000   Number         0  entry7a.o ABSOLUTE
    ../clib/microlib/init/entry.s            0x00000000   Number         0  entry7b.o ABSOLUTE
    ../clib/microlib/init/entry.s            0x00000000   Number         0  entry9a.o ABSOLUTE
    ../clib/microlib/init/entry.s            0x00000000   Number         0  entry8a.o ABSOLUTE
    ../clib/microlib/init/entry.s            0x00000000   Number         0  entry10b.o ABSOLUTE
    ../clib/microlib/init/entry.s            0x00000000   Number         0  entry11a.o ABSOLUTE
    ../clib/microlib/init/entry.s            0x00000000   Number         0  entry5.o ABSOLUTE
    ../clib/microlib/init/entry.s            0x00000000   Number         0  entry.o ABSOLUTE
    ../clib/microlib/init/entry.s            0x00000000   Number         0  entry11b.o ABSOLUTE
    ../clib/microlib/longlong.c              0x00000000   Number         0  llushr.o ABSOLUTE
    ../clib/microlib/longlong.c              0x00000000   Number         0  llshl.o ABSOLUTE
    ../clib/microlib/longlong.c              0x00000000   Number         0  llsshr.o ABSOLUTE
    ../clib/microlib/printf/printf.c         0x00000000   Number         0  printf5.o ABSOLUTE
    ../clib/microlib/printf/printf.c         0x00000000   Number         0  printf7.o ABSOLUTE
    ../clib/microlib/printf/printf.c         0x00000000   Number         0  printf8.o ABSOLUTE
    ../clib/microlib/printf/printf.c         0x00000000   Number         0  printfa.o ABSOLUTE
    ../clib/microlib/printf/printf.c         0x00000000   Number         0  printf6.o ABSOLUTE
    ../clib/microlib/printf/printf.c         0x00000000   Number         0  printfb.o ABSOLUTE
    ../clib/microlib/printf/printf.c         0x00000000   Number         0  printf0.o ABSOLUTE
    ../clib/microlib/printf/printf.c         0x00000000   Number         0  printf1.o ABSOLUTE
    ../clib/microlib/printf/printf.c         0x00000000   Number         0  printf2.o ABSOLUTE
    ../clib/microlib/printf/printf.c         0x00000000   Number         0  printf3.o ABSOLUTE
    ../clib/microlib/printf/printf.c         0x00000000   Number         0  printf4.o ABSOLUTE
    ../clib/microlib/printf/stubs.s          0x00000000   Number         0  stubs.o ABSOLUTE
    ../clib/microlib/string/memcpy.c         0x00000000   Number         0  memcpyb.o ABSOLUTE
    ../clib/microlib/string/memcpy.c         0x00000000   Number         0  memcpya.o ABSOLUTE
    ../clib/microlib/string/memset.c         0x00000000   Number         0  memseta.o ABSOLUTE
    ../clib/microlib/stubs.s                 0x00000000   Number         0  iusefp.o ABSOLUTE
    ../fplib/microlib/fpadd.c                0x00000000   Number         0  dadd.o ABSOLUTE
    ../fplib/microlib/fpdiv.c                0x00000000   Number         0  ddiv.o ABSOLUTE
    ../fplib/microlib/fpepilogue.c           0x00000000   Number         0  depilogue.o ABSOLUTE
    ../fplib/microlib/fpfix.c                0x00000000   Number         0  dfixul.o ABSOLUTE
    ../fplib/microlib/fpmul.c                0x00000000   Number         0  dmul.o ABSOLUTE
    ..\USER\project\CORE\core_cm3.c          0x00000000   Number         0  core_cm3.o ABSOLUTE
    ..\USER\project\STM32F10x_FWLib\src\misc.c 0x00000000   Number         0  misc.o ABSOLUTE
    ..\USER\project\STM32F10x_FWLib\src\stm32f10x_adc.c 0x00000000   Number         0  stm32f10x_adc.o ABSOLUTE
    ..\USER\project\STM32F10x_FWLib\src\stm32f10x_exti.c 0x00000000   Number         0  stm32f10x_exti.o ABSOLUTE
    ..\USER\project\STM32F10x_FWLib\src\stm32f10x_fsmc.c 0x00000000   Number         0  stm32f10x_fsmc.o ABSOLUTE
    ..\USER\project\STM32F10x_FWLib\src\stm32f10x_gpio.c 0x00000000   Number         0  stm32f10x_gpio.o ABSOLUTE
    ..\USER\project\STM32F10x_FWLib\src\stm32f10x_i2c.c 0x00000000   Number         0  stm32f10x_i2c.o ABSOLUTE
    ..\USER\project\STM32F10x_FWLib\src\stm32f10x_iwdg.c 0x00000000   Number         0  stm32f10x_iwdg.o ABSOLUTE
    ..\USER\project\STM32F10x_FWLib\src\stm32f10x_rcc.c 0x00000000   Number         0  stm32f10x_rcc.o ABSOLUTE
    ..\USER\project\STM32F10x_FWLib\src\stm32f10x_spi.c 0x00000000   Number         0  stm32f10x_spi.o ABSOLUTE
    ..\USER\project\STM32F10x_FWLib\src\stm32f10x_tim.c 0x00000000   Number         0  stm32f10x_tim.o ABSOLUTE
    ..\USER\project\STM32F10x_FWLib\src\stm32f10x_usart.c 0x00000000   Number         0  stm32f10x_usart.o ABSOLUTE
    ..\USER\project\config\stm32_config.c    0x00000000   Number         0  stm32_config.o ABSOLUTE
    ..\USER\project\main\main.c              0x00000000   Number         0  main.o ABSOLUTE
    ..\USER\project\main\main_Cilent.c       0x00000000   Number         0  main_cilent.o ABSOLUTE
    ..\USER\project\main\main_Server.c       0x00000000   Number         0  main_server.o ABSOLUTE
    ..\USER\project\module\DP83848vv\STM32_ETH_Driver\src\stm32_eth.c 0x00000000   Number         0  stm32_eth.o ABSOLUTE
    ..\USER\project\module\DP83848vv\TCPclient.c 0x00000000   Number         0  tcpclient.o ABSOLUTE
    ..\USER\project\module\DP83848vv\TCPserver.c 0x00000000   Number         0  tcpserver.o ABSOLUTE
    ..\USER\project\module\DP83848vv\lwip-1.3.1\port\ethernetif.c 0x00000000   Number         0  ethernetif.o ABSOLUTE
    ..\USER\project\module\DP83848vv\lwip-1.3.1\src\api\api_lib.c 0x00000000   Number         0  api_lib.o ABSOLUTE
    ..\USER\project\module\DP83848vv\lwip-1.3.1\src\api\api_msg.c 0x00000000   Number         0  api_msg.o ABSOLUTE
    ..\USER\project\module\DP83848vv\lwip-1.3.1\src\api\err.c 0x00000000   Number         0  err.o ABSOLUTE
    ..\USER\project\module\DP83848vv\lwip-1.3.1\src\api\netbuf.c 0x00000000   Number         0  netbuf.o ABSOLUTE
    ..\USER\project\module\DP83848vv\lwip-1.3.1\src\api\netdb.c 0x00000000   Number         0  netdb.o ABSOLUTE
    ..\USER\project\module\DP83848vv\lwip-1.3.1\src\api\netifapi.c 0x00000000   Number         0  netifapi.o ABSOLUTE
    ..\USER\project\module\DP83848vv\lwip-1.3.1\src\api\tcpip.c 0x00000000   Number         0  tcpip.o ABSOLUTE
    ..\USER\project\module\DP83848vv\lwip-1.3.1\src\core\dhcp.c 0x00000000   Number         0  dhcp.o ABSOLUTE
    ..\USER\project\module\DP83848vv\lwip-1.3.1\src\core\init.c 0x00000000   Number         0  init.o ABSOLUTE
    ..\USER\project\module\DP83848vv\lwip-1.3.1\src\core\ipv4\autoip.c 0x00000000   Number         0  autoip.o ABSOLUTE
    ..\USER\project\module\DP83848vv\lwip-1.3.1\src\core\ipv4\icmp.c 0x00000000   Number         0  icmp.o ABSOLUTE
    ..\USER\project\module\DP83848vv\lwip-1.3.1\src\core\ipv4\igmp.c 0x00000000   Number         0  igmp.o ABSOLUTE
    ..\USER\project\module\DP83848vv\lwip-1.3.1\src\core\ipv4\inet.c 0x00000000   Number         0  inet.o ABSOLUTE
    ..\USER\project\module\DP83848vv\lwip-1.3.1\src\core\ipv4\inet_chksum.c 0x00000000   Number         0  inet_chksum.o ABSOLUTE
    ..\USER\project\module\DP83848vv\lwip-1.3.1\src\core\ipv4\ip.c 0x00000000   Number         0  ip.o ABSOLUTE
    ..\USER\project\module\DP83848vv\lwip-1.3.1\src\core\ipv4\ip_addr.c 0x00000000   Number         0  ip_addr.o ABSOLUTE
    ..\USER\project\module\DP83848vv\lwip-1.3.1\src\core\ipv4\ip_frag.c 0x00000000   Number         0  ip_frag.o ABSOLUTE
    ..\USER\project\module\DP83848vv\lwip-1.3.1\src\core\mem.c 0x00000000   Number         0  mem.o ABSOLUTE
    ..\USER\project\module\DP83848vv\lwip-1.3.1\src\core\memp.c 0x00000000   Number         0  memp.o ABSOLUTE
    ..\USER\project\module\DP83848vv\lwip-1.3.1\src\core\netif.c 0x00000000   Number         0  netif.o ABSOLUTE
    ..\USER\project\module\DP83848vv\lwip-1.3.1\src\core\pbuf.c 0x00000000   Number         0  pbuf.o ABSOLUTE
    ..\USER\project\module\DP83848vv\lwip-1.3.1\src\core\raw.c 0x00000000   Number         0  raw.o ABSOLUTE
    ..\USER\project\module\DP83848vv\lwip-1.3.1\src\core\stats.c 0x00000000   Number         0  stats.o ABSOLUTE
    ..\USER\project\module\DP83848vv\lwip-1.3.1\src\core\sys.c 0x00000000   Number         0  sys.o ABSOLUTE
    ..\USER\project\module\DP83848vv\lwip-1.3.1\src\core\tcp.c 0x00000000   Number         0  tcp.o ABSOLUTE
    ..\USER\project\module\DP83848vv\lwip-1.3.1\src\core\tcp_in.c 0x00000000   Number         0  tcp_in.o ABSOLUTE
    ..\USER\project\module\DP83848vv\lwip-1.3.1\src\core\tcp_out.c 0x00000000   Number         0  tcp_out.o ABSOLUTE
    ..\USER\project\module\DP83848vv\lwip-1.3.1\src\core\udp.c 0x00000000   Number         0  udp.o ABSOLUTE
    ..\USER\project\module\DP83848vv\lwip-1.3.1\src\netif\etharp.c 0x00000000   Number         0  etharp.o ABSOLUTE
    ..\USER\project\module\DP83848vv\netconf.c 0x00000000   Number         0  netconf.o ABSOLUTE
    ..\USER\project\module\DP83848vv\stm32f107.c 0x00000000   Number         0  stm32f107.o ABSOLUTE
    ..\USER\project\module\usart\printf.c    0x00000000   Number         0  printf.o ABSOLUTE
    ..\USER\project\module\usart\usart1.c    0x00000000   Number         0  usart1.o ABSOLUTE
    ..\USER\project\system\delay.c           0x00000000   Number         0  delay.o ABSOLUTE
    ..\USER\project\system\stm32f10x_it.c    0x00000000   Number         0  stm32f10x_it.o ABSOLUTE
    ..\USER\ucosii\CORE\os_core.c            0x00000000   Number         0  os_core.o ABSOLUTE
    ..\USER\ucosii\CORE\os_flag.c            0x00000000   Number         0  os_flag.o ABSOLUTE
    ..\USER\ucosii\CORE\os_mbox.c            0x00000000   Number         0  os_mbox.o ABSOLUTE
    ..\USER\ucosii\CORE\os_mem.c             0x00000000   Number         0  os_mem.o ABSOLUTE
    ..\USER\ucosii\CORE\os_mutex.c           0x00000000   Number         0  os_mutex.o ABSOLUTE
    ..\USER\ucosii\CORE\os_q.c               0x00000000   Number         0  os_q.o ABSOLUTE
    ..\USER\ucosii\CORE\os_sem.c             0x00000000   Number         0  os_sem.o ABSOLUTE
    ..\USER\ucosii\CORE\os_task.c            0x00000000   Number         0  os_task.o ABSOLUTE
    ..\USER\ucosii\CORE\os_time.c            0x00000000   Number         0  os_time.o ABSOLUTE
    ..\USER\ucosii\CORE\os_tmr.c             0x00000000   Number         0  os_tmr.o ABSOLUTE
    ..\USER\ucosii\PORT\os_cpu_a.asm         0x00000000   Number         0  os_cpu_a.o ABSOLUTE
    ..\USER\ucosii\PORT\os_cpu_c.c           0x00000000   Number         0  os_cpu_c.o ABSOLUTE
    ..\USER\ucosii\PORT\os_dbg.c             0x00000000   Number         0  os_dbg.o ABSOLUTE
    ..\\USER\\project\\CORE\\core_cm3.c      0x00000000   Number         0  core_cm3.o ABSOLUTE
    RTE\Device\STM32F107VC\startup_stm32f10x_cl.s 0x00000000   Number         0  startup_stm32f10x_cl.o ABSOLUTE
    RTE\Device\STM32F107VC\system_stm32f10x.c 0x00000000   Number         0  system_stm32f10x.o ABSOLUTE
    cdrcmple.s                               0x00000000   Number         0  cdrcmple.o ABSOLUTE
    dc.s                                     0x00000000   Number         0  dc.o ABSOLUTE
    handlers.s                               0x00000000   Number         0  handlers.o ABSOLUTE
    init.s                                   0x00000000   Number         0  init.o ABSOLUTE
    RESET                                    0x08000000   Section      336  startup_stm32f10x_cl.o(RESET)
    .ARM.Collect$$$$00000000                 0x08000150   Section        0  entry.o(.ARM.Collect$$$$00000000)
    .ARM.Collect$$$$00000001                 0x08000150   Section        4  entry2.o(.ARM.Collect$$$$00000001)
    .ARM.Collect$$$$00000004                 0x08000154   Section        4  entry5.o(.ARM.Collect$$$$00000004)
    .ARM.Collect$$$$00000008                 0x08000158   Section        0  entry7b.o(.ARM.Collect$$$$00000008)
    .ARM.Collect$$$$0000000A                 0x08000158   Section        0  entry8b.o(.ARM.Collect$$$$0000000A)
    .ARM.Collect$$$$0000000B                 0x08000158   Section        8  entry9a.o(.ARM.Collect$$$$0000000B)
    .ARM.Collect$$$$0000000D                 0x08000160   Section        0  entry10a.o(.ARM.Collect$$$$0000000D)
    .ARM.Collect$$$$0000000F                 0x08000160   Section        0  entry11a.o(.ARM.Collect$$$$0000000F)
    .ARM.Collect$$$$00002712                 0x08000160   Section        4  entry2.o(.ARM.Collect$$$$00002712)
    __lit__00000000                          0x08000160   Data           4  entry2.o(.ARM.Collect$$$$00002712)
    .text                                    0x08000164   Section      180  os_cpu_a.o(.text)
    .text                                    0x08000218   Section       36  startup_stm32f10x_cl.o(.text)
    .text                                    0x0800023c   Section        0  memcpya.o(.text)
    .text                                    0x08000260   Section        0  memseta.o(.text)
    .text                                    0x08000284   Section        0  uidiv.o(.text)
    .text                                    0x080002b0   Section       36  init.o(.text)
    .text                                    0x080002d4   Section        0  __dczerorl2.o(.text)
    i.BusFault_Handler                       0x0800032c   Section        0  stm32f10x_it.o(i.BusFault_Handler)
    i.DebugMon_Handler                       0x08000354   Section        0  stm32f10x_it.o(i.DebugMon_Handler)
    i.ETH_DMAClearITPendingBit               0x08000358   Section        0  stm32_eth.o(i.ETH_DMAClearITPendingBit)
    i.ETH_DMAITConfig                        0x08000364   Section        0  stm32_eth.o(i.ETH_DMAITConfig)
    i.ETH_DMAReceptionCmd                    0x08000384   Section        0  stm32_eth.o(i.ETH_DMAReceptionCmd)
    i.ETH_DMARxDescChainInit                 0x080003a8   Section        0  stm32_eth.o(i.ETH_DMARxDescChainInit)
    i.ETH_DMARxDescReceiveITConfig           0x080003fc   Section        0  stm32_eth.o(i.ETH_DMARxDescReceiveITConfig)
    i.ETH_DMATransmissionCmd                 0x08000414   Section        0  stm32_eth.o(i.ETH_DMATransmissionCmd)
    i.ETH_DMATxDescChainInit                 0x08000438   Section        0  stm32_eth.o(i.ETH_DMATxDescChainInit)
    i.ETH_DMATxDescChecksumInsertionConfig   0x08000488   Section        0  stm32_eth.o(i.ETH_DMATxDescChecksumInsertionConfig)
    i.ETH_DeInit                             0x08000490   Section        0  stm32_eth.o(i.ETH_DeInit)
    i.ETH_Delay                              0x080004a6   Section        0  stm32_eth.o(i.ETH_Delay)
    ETH_Delay                                0x080004a7   Thumb Code    28  stm32_eth.o(i.ETH_Delay)
    i.ETH_FlushTransmitFIFO                  0x080004c4   Section        0  stm32_eth.o(i.ETH_FlushTransmitFIFO)
    i.ETH_GetCurrentTxBuffer                 0x080004d8   Section        0  ethernetif.o(i.ETH_GetCurrentTxBuffer)
    i.ETH_GetDMARxDescFrameLength            0x080004e4   Section        0  stm32_eth.o(i.ETH_GetDMARxDescFrameLength)
    i.ETH_GetRxPktSize                       0x080004f0   Section        0  stm32_eth.o(i.ETH_GetRxPktSize)
    i.ETH_GetSoftwareResetStatus             0x08000538   Section        0  stm32_eth.o(i.ETH_GetSoftwareResetStatus)
    i.ETH_IRQHandler                         0x08000550   Section        0  stm32f10x_it.o(i.ETH_IRQHandler)
    i.ETH_Init                               0x08000578   Section        0  stm32_eth.o(i.ETH_Init)
    i.ETH_MACAddressConfig                   0x080007dc   Section        0  stm32_eth.o(i.ETH_MACAddressConfig)
    i.ETH_MACReceptionCmd                    0x08000810   Section        0  stm32_eth.o(i.ETH_MACReceptionCmd)
    i.ETH_MACTransmissionCmd                 0x08000834   Section        0  stm32_eth.o(i.ETH_MACTransmissionCmd)
    i.ETH_ReadPHYRegister                    0x08000858   Section        0  stm32_eth.o(i.ETH_ReadPHYRegister)
    i.ETH_RxPkt_ChainMode                    0x080008c4   Section        0  ethernetif.o(i.ETH_RxPkt_ChainMode)
    i.ETH_SoftwareReset                      0x08000960   Section        0  stm32_eth.o(i.ETH_SoftwareReset)
    i.ETH_Start                              0x08000974   Section        0  stm32_eth.o(i.ETH_Start)
    i.ETH_StructInit                         0x08000994   Section        0  stm32_eth.o(i.ETH_StructInit)
    i.ETH_TxPkt_ChainMode                    0x08000a38   Section        0  ethernetif.o(i.ETH_TxPkt_ChainMode)
    i.ETH_WritePHYRegister                   0x08000aa0   Section        0  stm32_eth.o(i.ETH_WritePHYRegister)
    i.Ethernet_Configuration                 0x08000b08   Section        0  stm32f107.o(i.Ethernet_Configuration)
    i.GPIO_Configuration                     0x08000bb8   Section        0  stm32f107.o(i.GPIO_Configuration)
    i.GPIO_ETH_MediaInterfaceConfig          0x08000c68   Section        0  stm32f10x_gpio.o(i.GPIO_ETH_MediaInterfaceConfig)
    i.GPIO_Init                              0x08000c74   Section        0  stm32f10x_gpio.o(i.GPIO_Init)
    i.GPIO_PinRemapConfig                    0x08000d8c   Section        0  stm32f10x_gpio.o(i.GPIO_PinRemapConfig)
    i.HardFault_Handler                      0x08000e1c   Section        0  stm32f10x_it.o(i.HardFault_Handler)
    i.LwIP_Init                              0x08000e44   Section        0  netconf.o(i.LwIP_Init)
    i.LwIP_Pkt_Handle                        0x08000ebc   Section        0  netconf.o(i.LwIP_Pkt_Handle)
    i.MemManage_Handler                      0x08000ecc   Section        0  stm32f10x_it.o(i.MemManage_Handler)
    i.NMI_Handler                            0x08000ef4   Section        0  stm32f10x_it.o(i.NMI_Handler)
    i.NVIC_Configuration                     0x08000ef6   Section        0  stm32f107.o(i.NVIC_Configuration)
    i.NVIC_Init                              0x08000f2c   Section        0  misc.o(i.NVIC_Init)
    i.NVIC_PriorityGroupConfig               0x08000f9c   Section        0  misc.o(i.NVIC_PriorityGroupConfig)
    i.NVIC_SetPriority                       0x08000fb0   Section        0  stm32f107.o(i.NVIC_SetPriority)
    NVIC_SetPriority                         0x08000fb1   Thumb Code    32  stm32f107.o(i.NVIC_SetPriority)
    i.NVIC_SetVectorTable                    0x08000fd8   Section        0  misc.o(i.NVIC_SetVectorTable)
    i.OSInit                                 0x08000fec   Section        0  os_core.o(i.OSInit)
    i.OSInitHookBegin                        0x08001018   Section        0  os_cpu_c.o(i.OSInitHookBegin)
    i.OSInitHookEnd                          0x0800101a   Section        0  os_cpu_c.o(i.OSInitHookEnd)
    i.OSIntEnter                             0x0800101c   Section        0  os_core.o(i.OSIntEnter)
    i.OSIntExit                              0x08001040   Section        0  os_core.o(i.OSIntExit)
    i.OSStart                                0x080010d0   Section        0  os_core.o(i.OSStart)
    i.OSStatInit                             0x08001118   Section        0  os_core.o(i.OSStatInit)
    i.OSTCBInitHook                          0x08001164   Section        0  os_cpu_c.o(i.OSTCBInitHook)
    i.OSTaskCreate                           0x08001168   Section        0  os_task.o(i.OSTaskCreate)
    i.OSTaskCreateExt                        0x08001208   Section        0  os_task.o(i.OSTaskCreateExt)
    i.OSTaskCreateHook                       0x080012c0   Section        0  os_cpu_c.o(i.OSTaskCreateHook)
    i.OSTaskIdleHook                         0x080012c2   Section        0  os_cpu_c.o(i.OSTaskIdleHook)
    i.OSTaskNameSet                          0x080012c4   Section        0  os_task.o(i.OSTaskNameSet)
    i.OSTaskStatHook                         0x08001334   Section        0  os_cpu_c.o(i.OSTaskStatHook)
    i.OSTaskStkChk                           0x08001338   Section        0  os_task.o(i.OSTaskStkChk)
    i.OSTaskStkInit                          0x080013c4   Section        0  os_cpu_c.o(i.OSTaskStkInit)
    i.OSTaskSuspend                          0x08001460   Section        0  os_task.o(i.OSTaskSuspend)
    i.OSTaskSwHook                           0x08001508   Section        0  os_cpu_c.o(i.OSTaskSwHook)
    i.OSTimeDly                              0x0800150c   Section        0  os_time.o(i.OSTimeDly)
    i.OSTimeTick                             0x08001584   Section        0  os_core.o(i.OSTimeTick)
    i.OSTimeTickHook                         0x08001670   Section        0  os_cpu_c.o(i.OSTimeTickHook)
    i.OS_FlagInit                            0x08001674   Section        0  os_flag.o(i.OS_FlagInit)
    i.OS_InitEventList                       0x080016cc   Section        0  os_core.o(i.OS_InitEventList)
    OS_InitEventList                         0x080016cd   Thumb Code    74  os_core.o(i.OS_InitEventList)
    i.OS_InitMisc                            0x08001720   Section        0  os_core.o(i.OS_InitMisc)
    OS_InitMisc                              0x08001721   Thumb Code    44  os_core.o(i.OS_InitMisc)
    i.OS_InitRdyList                         0x08001774   Section        0  os_core.o(i.OS_InitRdyList)
    OS_InitRdyList                           0x08001775   Thumb Code    44  os_core.o(i.OS_InitRdyList)
    i.OS_InitTCBList                         0x080017b8   Section        0  os_core.o(i.OS_InitTCBList)
    OS_InitTCBList                           0x080017b9   Thumb Code   106  os_core.o(i.OS_InitTCBList)
    i.OS_InitTaskIdle                        0x08001838   Section        0  os_core.o(i.OS_InitTaskIdle)
    OS_InitTaskIdle                          0x08001839   Thumb Code    50  os_core.o(i.OS_InitTaskIdle)
    i.OS_InitTaskStat                        0x08001888   Section        0  os_core.o(i.OS_InitTaskStat)
    OS_InitTaskStat                          0x08001889   Thumb Code    50  os_core.o(i.OS_InitTaskStat)
    i.OS_MemClr                              0x080018d8   Section        0  os_core.o(i.OS_MemClr)
    i.OS_QInit                               0x080018ec   Section        0  os_q.o(i.OS_QInit)
    i.OS_Sched                               0x0800193c   Section        0  os_core.o(i.OS_Sched)
    i.OS_SchedNew                            0x080019b0   Section        0  os_core.o(i.OS_SchedNew)
    OS_SchedNew                              0x080019b1   Thumb Code    26  os_core.o(i.OS_SchedNew)
    i.OS_TCBInit                             0x080019dc   Section        0  os_core.o(i.OS_TCBInit)
    i.OS_TaskIdle                            0x08001b10   Section        0  os_core.o(i.OS_TaskIdle)
    i.OS_TaskStat                            0x08001b38   Section        0  os_core.o(i.OS_TaskStat)
    i.OS_TaskStatStkChk                      0x08001bc0   Section        0  os_core.o(i.OS_TaskStatStkChk)
    i.OS_TaskStkClr                          0x08001bfc   Section        0  os_task.o(i.OS_TaskStkClr)
    i.RCC_AHBPeriphClockCmd                  0x08001c18   Section        0  stm32f10x_rcc.o(i.RCC_AHBPeriphClockCmd)
    i.RCC_AHBPeriphResetCmd                  0x08001c38   Section        0  stm32f10x_rcc.o(i.RCC_AHBPeriphResetCmd)
    i.RCC_APB1PeriphClockCmd                 0x08001c58   Section        0  stm32f10x_rcc.o(i.RCC_APB1PeriphClockCmd)
    i.RCC_APB2PeriphClockCmd                 0x08001c78   Section        0  stm32f10x_rcc.o(i.RCC_APB2PeriphClockCmd)
    i.RCC_GetClocksFreq                      0x08001c98   Section        0  stm32f10x_rcc.o(i.RCC_GetClocksFreq)
    i.RCC_GetFlagStatus                      0x08001e28   Section        0  stm32f10x_rcc.o(i.RCC_GetFlagStatus)
    i.RCC_MCOConfig                          0x08001e64   Section        0  stm32f10x_rcc.o(i.RCC_MCOConfig)
    i.RCC_PLL3Cmd                            0x08001e70   Section        0  stm32f10x_rcc.o(i.RCC_PLL3Cmd)
    i.RCC_PLL3Config                         0x08001e7c   Section        0  stm32f10x_rcc.o(i.RCC_PLL3Config)
    i.SVC_Handler                            0x08001e94   Section        0  stm32f10x_it.o(i.SVC_Handler)
    i.SetSysClock                            0x08001e96   Section        0  system_stm32f10x.o(i.SetSysClock)
    SetSysClock                              0x08001e97   Thumb Code     8  system_stm32f10x.o(i.SetSysClock)
    i.SetSysClockTo72                        0x08001ea0   Section        0  system_stm32f10x.o(i.SetSysClockTo72)
    SetSysClockTo72                          0x08001ea1   Thumb Code   264  system_stm32f10x.o(i.SetSysClockTo72)
    i.Set_MAC_Address                        0x08001fb8   Section        0  ethernetif.o(i.Set_MAC_Address)
    i.SysTick_CLKSourceConfig                0x08001fe4   Section        0  misc.o(i.SysTick_CLKSourceConfig)
    i.SysTick_Handler                        0x0800200c   Section        0  delay.o(i.SysTick_Handler)
    i.SystemInit                             0x0800201c   Section        0  system_stm32f10x.o(i.SystemInit)
    i.System_Setup                           0x08002088   Section        0  stm32f107.o(i.System_Setup)
    i.TCP_Client_Recv                        0x08002100   Section        0  tcpclient.o(i.TCP_Client_Recv)
    i.TCP_Client_Send                        0x08002140   Section        0  tcpclient.o(i.TCP_Client_Send)
    i.TCP_Server_Recv                        0x08002174   Section        0  tcpserver.o(i.TCP_Server_Recv)
    i.TCP_Server_Send                        0x080021b4   Section        0  tcpserver.o(i.TCP_Server_Send)
    i.USART1_IRQHandler                      0x080021e8   Section        0  usart1.o(i.USART1_IRQHandler)
    i.USART_ClearFlag                        0x08002254   Section        0  stm32f10x_usart.o(i.USART_ClearFlag)
    i.USART_ClearITPendingBit                0x08002266   Section        0  stm32f10x_usart.o(i.USART_ClearITPendingBit)
    i.USART_Cmd                              0x08002284   Section        0  stm32f10x_usart.o(i.USART_Cmd)
    i.USART_GetFlagStatus                    0x0800229c   Section        0  stm32f10x_usart.o(i.USART_GetFlagStatus)
    i.USART_GetITStatus                      0x080022b6   Section        0  stm32f10x_usart.o(i.USART_GetITStatus)
    i.USART_ITConfig                         0x0800230a   Section        0  stm32f10x_usart.o(i.USART_ITConfig)
    i.USART_Init                             0x08002354   Section        0  stm32f10x_usart.o(i.USART_Init)
    i.USART_ReceiveData                      0x0800242c   Section        0  stm32f10x_usart.o(i.USART_ReceiveData)
    i.USART_SendData                         0x08002436   Section        0  stm32f10x_usart.o(i.USART_SendData)
    i.UsageFault_Handler                     0x08002440   Section        0  stm32f10x_it.o(i.UsageFault_Handler)
    i.__0printf$3                            0x0800246c   Section        0  printf3.o(i.__0printf$3)
    i.__scatterload_copy                     0x0800248c   Section       14  handlers.o(i.__scatterload_copy)
    i.__scatterload_null                     0x0800249a   Section        2  handlers.o(i.__scatterload_null)
    i.__scatterload_zeroinit                 0x0800249c   Section       14  handlers.o(i.__scatterload_zeroinit)
    i._printf_core                           0x080024ac   Section        0  printf3.o(i._printf_core)
    _printf_core                             0x080024ad   Thumb Code   436  printf3.o(i._printf_core)
    i.delay_init                             0x08002664   Section        0  delay.o(i.delay_init)
    i.delay_ms                               0x080026c0   Section        0  delay.o(i.delay_ms)
    i.delay_us                               0x08002708   Section        0  delay.o(i.delay_us)
    i.etharp_arp_input                       0x08002754   Section        0  etharp.o(i.etharp_arp_input)
    i.etharp_ip_input                        0x08002886   Section        0  etharp.o(i.etharp_ip_input)
    i.etharp_output                          0x080028c0   Section        0  etharp.o(i.etharp_output)
    i.etharp_query                           0x08002984   Section        0  etharp.o(i.etharp_query)
    i.etharp_raw                             0x08002b3c   Section        0  etharp.o(i.etharp_raw)
    etharp_raw                               0x08002b3d   Thumb Code   202  etharp.o(i.etharp_raw)
    i.etharp_request                         0x08002c08   Section        0  etharp.o(i.etharp_request)
    i.etharp_send_ip                         0x08002c34   Section        0  etharp.o(i.etharp_send_ip)
    etharp_send_ip                           0x08002c35   Thumb Code    78  etharp.o(i.etharp_send_ip)
    i.ethernet_input                         0x08002c82   Section        0  etharp.o(i.ethernet_input)
    i.ethernetif_init                        0x08002cec   Section        0  ethernetif.o(i.ethernetif_init)
    i.ethernetif_input                       0x08002d38   Section        0  ethernetif.o(i.ethernetif_input)
    i.find_entry                             0x08002d64   Section        0  etharp.o(i.find_entry)
    find_entry                               0x08002d65   Thumb Code   506  etharp.o(i.find_entry)
    i.fputc                                  0x08002f68   Section        0  printf.o(i.fputc)
    i.free_etharp_q                          0x08002f8c   Section        0  etharp.o(i.free_etharp_q)
    free_etharp_q                            0x08002f8d   Thumb Code    64  etharp.o(i.free_etharp_q)
    i.htonl                                  0x08002fcc   Section        0  inet.o(i.htonl)
    i.htons                                  0x08002fe6   Section        0  inet.o(i.htons)
    i.icmp_dest_unreach                      0x08002ff2   Section        0  icmp.o(i.icmp_dest_unreach)
    i.icmp_input                             0x08003004   Section        0  icmp.o(i.icmp_input)
    i.icmp_send_response                     0x08003198   Section        0  icmp.o(i.icmp_send_response)
    icmp_send_response                       0x08003199   Thumb Code   118  icmp.o(i.icmp_send_response)
    i.icmp_time_exceeded                     0x0800320e   Section        0  icmp.o(i.icmp_time_exceeded)
    i.inet_chksum                            0x08003220   Section        0  inet_chksum.o(i.inet_chksum)
    i.inet_chksum_pbuf                       0x08003234   Section        0  inet_chksum.o(i.inet_chksum_pbuf)
    i.ip_addr_isbroadcast                    0x0800328a   Section        0  ip_addr.o(i.ip_addr_isbroadcast)
    i.ip_frag                                0x080032d8   Section        0  ip_frag.o(i.ip_frag)
    i.ip_input                               0x08003424   Section        0  ip.o(i.ip_input)
    i.ip_output                              0x080035a8   Section        0  ip.o(i.ip_output)
    i.ip_output_if                           0x080035dc   Section        0  ip.o(i.ip_output_if)
    i.ip_reass                               0x080036e0   Section        0  ip_frag.o(i.ip_reass)
    i.ip_reass_chain_frag_into_datagram_and_validate 0x08003878   Section        0  ip_frag.o(i.ip_reass_chain_frag_into_datagram_and_validate)
    ip_reass_chain_frag_into_datagram_and_validate 0x08003879   Thumb Code   418  ip_frag.o(i.ip_reass_chain_frag_into_datagram_and_validate)
    i.ip_reass_dequeue_datagram              0x08003a20   Section        0  ip_frag.o(i.ip_reass_dequeue_datagram)
    ip_reass_dequeue_datagram                0x08003a21   Thumb Code    46  ip_frag.o(i.ip_reass_dequeue_datagram)
    i.ip_reass_enqueue_new_datagram          0x08003a54   Section        0  ip_frag.o(i.ip_reass_enqueue_new_datagram)
    ip_reass_enqueue_new_datagram            0x08003a55   Thumb Code    80  ip_frag.o(i.ip_reass_enqueue_new_datagram)
    i.ip_reass_free_complete_datagram        0x08003aa8   Section        0  ip_frag.o(i.ip_reass_free_complete_datagram)
    ip_reass_free_complete_datagram          0x08003aa9   Thumb Code   166  ip_frag.o(i.ip_reass_free_complete_datagram)
    i.ip_reass_remove_oldest_datagram        0x08003b54   Section        0  ip_frag.o(i.ip_reass_remove_oldest_datagram)
    ip_reass_remove_oldest_datagram          0x08003b55   Thumb Code   118  ip_frag.o(i.ip_reass_remove_oldest_datagram)
    i.ip_route                               0x08003bd0   Section        0  ip.o(i.ip_route)
    i.low_level_init                         0x08003c20   Section        0  ethernetif.o(i.low_level_init)
    low_level_init                           0x08003c21   Thumb Code   142  ethernetif.o(i.low_level_init)
    i.low_level_input                        0x08003cc4   Section        0  ethernetif.o(i.low_level_input)
    low_level_input                          0x08003cc5   Thumb Code   110  ethernetif.o(i.low_level_input)
    i.low_level_output                       0x08003d38   Section        0  ethernetif.o(i.low_level_output)
    low_level_output                         0x08003d39   Thumb Code    52  ethernetif.o(i.low_level_output)
    i.lwip_standard_chksum                   0x08003d6c   Section        0  inet_chksum.o(i.lwip_standard_chksum)
    lwip_standard_chksum                     0x08003d6d   Thumb Code    74  inet_chksum.o(i.lwip_standard_chksum)
    i.main                                   0x08003db8   Section        0  main.o(i.main)
    i.main_Client_task                       0x08003dec   Section        0  main_cilent.o(i.main_Client_task)
    i.main_Server_task                       0x08003eec   Section        0  main_server.o(i.main_Server_task)
    i.mem_free                               0x08003f4c   Section        0  mem.o(i.mem_free)
    i.mem_init                               0x08003fc4   Section        0  mem.o(i.mem_init)
    i.mem_malloc                             0x08004028   Section        0  mem.o(i.mem_malloc)
    i.mem_realloc                            0x08004158   Section        0  mem.o(i.mem_realloc)
    i.memp_free                              0x080042a0   Section        0  memp.o(i.memp_free)
    i.memp_init                              0x080042cc   Section        0  memp.o(i.memp_init)
    i.memp_malloc                            0x08004330   Section        0  memp.o(i.memp_malloc)
    i.netif_add                              0x0800436c   Section        0  netif.o(i.netif_add)
    i.netif_is_up                            0x080043d4   Section        0  netif.o(i.netif_is_up)
    i.netif_set_addr                         0x080043e0   Section        0  netif.o(i.netif_set_addr)
    i.netif_set_default                      0x08004408   Section        0  netif.o(i.netif_set_default)
    i.netif_set_gw                           0x08004414   Section        0  netif.o(i.netif_set_gw)
    i.netif_set_ipaddr                       0x08004420   Section        0  netif.o(i.netif_set_ipaddr)
    i.netif_set_netmask                      0x08004498   Section        0  netif.o(i.netif_set_netmask)
    i.netif_set_up                           0x080044a4   Section        0  netif.o(i.netif_set_up)
    i.ntohl                                  0x080044d0   Section        0  inet.o(i.ntohl)
    i.ntohs                                  0x080044dc   Section        0  inet.o(i.ntohs)
    i.pbuf_alloc                             0x080044e8   Section        0  pbuf.o(i.pbuf_alloc)
    i.pbuf_cat                               0x080046fc   Section        0  pbuf.o(i.pbuf_cat)
    i.pbuf_chain                             0x0800474c   Section        0  pbuf.o(i.pbuf_chain)
    i.pbuf_clen                              0x08004762   Section        0  pbuf.o(i.pbuf_clen)
    i.pbuf_copy                              0x08004774   Section        0  pbuf.o(i.pbuf_copy)
    i.pbuf_copy_partial                      0x08004850   Section        0  pbuf.o(i.pbuf_copy_partial)
    i.pbuf_free                              0x080048ea   Section        0  pbuf.o(i.pbuf_free)
    i.pbuf_header                            0x08004982   Section        0  pbuf.o(i.pbuf_header)
    i.pbuf_realloc                           0x08004a0e   Section        0  pbuf.o(i.pbuf_realloc)
    i.pbuf_ref                               0x08004abe   Section        0  pbuf.o(i.pbuf_ref)
    i.plug_holes                             0x08004ac8   Section        0  mem.o(i.plug_holes)
    plug_holes                               0x08004ac9   Thumb Code   168  mem.o(i.plug_holes)
    i.start_task                             0x08004b7c   Section        0  main.o(i.start_task)
    i.tcp_abandon                            0x08004bf8   Section        0  tcp.o(i.tcp_abandon)
    i.tcp_accept                             0x08004c94   Section        0  tcp.o(i.tcp_accept)
    i.tcp_accept_null                        0x08004c98   Section        0  tcp.o(i.tcp_accept_null)
    tcp_accept_null                          0x08004c99   Thumb Code     8  tcp.o(i.tcp_accept_null)
    i.tcp_alloc                              0x08004ca0   Section        0  tcp.o(i.tcp_alloc)
    i.tcp_arg                                0x08004d54   Section        0  tcp.o(i.tcp_arg)
    i.tcp_bind                               0x08004d58   Section        0  tcp.o(i.tcp_bind)
    i.tcp_client_close                       0x08004e50   Section        0  tcpclient.o(i.tcp_client_close)
    i.tcp_client_error                       0x08004e88   Section        0  tcpclient.o(i.tcp_client_error)
    tcp_client_error                         0x08004e89   Thumb Code    48  tcpclient.o(i.tcp_client_error)
    i.tcp_client_sent                        0x08004ed8   Section        0  tcpclient.o(i.tcp_client_sent)
    tcp_client_sent                          0x08004ed9   Thumb Code    22  tcpclient.o(i.tcp_client_sent)
    i.tcp_close                              0x08004f08   Section        0  tcp.o(i.tcp_close)
    i.tcp_connect                            0x080050b8   Section        0  tcp.o(i.tcp_connect)
    i.tcp_echoclient_connect                 0x080051dc   Section        0  tcpclient.o(i.tcp_echoclient_connect)
    i.tcp_echoclient_connected               0x0800524c   Section        0  tcpclient.o(i.tcp_echoclient_connected)
    tcp_echoclient_connected                 0x0800524d   Thumb Code   124  tcpclient.o(i.tcp_echoclient_connected)
    i.tcp_echoclient_connection_close        0x080052e4   Section        0  tcpclient.o(i.tcp_echoclient_connection_close)
    tcp_echoclient_connection_close          0x080052e5   Thumb Code    64  tcpclient.o(i.tcp_echoclient_connection_close)
    i.tcp_echoclient_poll                    0x08005324   Section        0  tcpclient.o(i.tcp_echoclient_poll)
    tcp_echoclient_poll                      0x08005325   Thumb Code    84  tcpclient.o(i.tcp_echoclient_poll)
    i.tcp_echoclient_recv                    0x08005390   Section        0  tcpclient.o(i.tcp_echoclient_recv)
    tcp_echoclient_recv                      0x08005391   Thumb Code   188  tcpclient.o(i.tcp_echoclient_recv)
    i.tcp_echoserver_accept                  0x0800545c   Section        0  tcpserver.o(i.tcp_echoserver_accept)
    tcp_echoserver_accept                    0x0800545d   Thumb Code   120  tcpserver.o(i.tcp_echoserver_accept)
    i.tcp_echoserver_connection_close        0x080054fc   Section        0  tcpserver.o(i.tcp_echoserver_connection_close)
    tcp_echoserver_connection_close          0x080054fd   Thumb Code    64  tcpserver.o(i.tcp_echoserver_connection_close)
    i.tcp_echoserver_error                   0x0800553c   Section        0  tcpserver.o(i.tcp_echoserver_error)
    tcp_echoserver_error                     0x0800553d   Thumb Code    36  tcpserver.o(i.tcp_echoserver_error)
    i.tcp_echoserver_init                    0x08005564   Section        0  tcpserver.o(i.tcp_echoserver_init)
    i.tcp_echoserver_poll                    0x080055b0   Section        0  tcpserver.o(i.tcp_echoserver_poll)
    tcp_echoserver_poll                      0x080055b1   Thumb Code    72  tcpserver.o(i.tcp_echoserver_poll)
    i.tcp_echoserver_recv                    0x08005610   Section        0  tcpserver.o(i.tcp_echoserver_recv)
    tcp_echoserver_recv                      0x08005611   Thumb Code   298  tcpserver.o(i.tcp_echoserver_recv)
    i.tcp_echoserver_send                    0x08005760   Section        0  tcpserver.o(i.tcp_echoserver_send)
    tcp_echoserver_send                      0x08005761   Thumb Code    72  tcpserver.o(i.tcp_echoserver_send)
    i.tcp_echoserver_sent                    0x080057a8   Section        0  tcpserver.o(i.tcp_echoserver_sent)
    tcp_echoserver_sent                      0x080057a9   Thumb Code    46  tcpserver.o(i.tcp_echoserver_sent)
    i.tcp_eff_send_mss                       0x080057d6   Section        0  tcp.o(i.tcp_eff_send_mss)
    i.tcp_enqueue                            0x08005804   Section        0  tcp_out.o(i.tcp_enqueue)
    i.tcp_err                                0x08005c30   Section        0  tcp.o(i.tcp_err)
    i.tcp_input                              0x08005c38   Section        0  tcp_in.o(i.tcp_input)
    i.tcp_kill_prio                          0x080060e0   Section        0  tcp.o(i.tcp_kill_prio)
    tcp_kill_prio                            0x080060e1   Thumb Code    78  tcp.o(i.tcp_kill_prio)
    i.tcp_kill_timewait                      0x08006138   Section        0  tcp.o(i.tcp_kill_timewait)
    tcp_kill_timewait                        0x08006139   Thumb Code    52  tcp.o(i.tcp_kill_timewait)
    i.tcp_listen_input                       0x08006174   Section        0  tcp_in.o(i.tcp_listen_input)
    tcp_listen_input                         0x08006175   Thumb Code   306  tcp_in.o(i.tcp_listen_input)
    i.tcp_listen_with_backlog                0x080062c4   Section        0  tcp.o(i.tcp_listen_with_backlog)
    i.tcp_new                                0x080063b0   Section        0  tcp.o(i.tcp_new)
    i.tcp_new_port                           0x080063bc   Section        0  tcp.o(i.tcp_new_port)
    tcp_new_port                             0x080063bd   Thumb Code   104  tcp.o(i.tcp_new_port)
    i.tcp_next_iss                           0x08006434   Section        0  tcp.o(i.tcp_next_iss)
    i.tcp_output                             0x08006450   Section        0  tcp_out.o(i.tcp_output)
    i.tcp_output_segment                     0x080066b8   Section        0  tcp_out.o(i.tcp_output_segment)
    tcp_output_segment                       0x080066b9   Thumb Code   194  tcp_out.o(i.tcp_output_segment)
    i.tcp_output_set_header                  0x08006784   Section        0  tcp_out.o(i.tcp_output_set_header)
    tcp_output_set_header                    0x08006785   Thumb Code   132  tcp_out.o(i.tcp_output_set_header)
    i.tcp_parseopt                           0x08006808   Section        0  tcp_in.o(i.tcp_parseopt)
    tcp_parseopt                             0x08006809   Thumb Code   176  tcp_in.o(i.tcp_parseopt)
    i.tcp_pcb_purge                          0x080068bc   Section        0  tcp.o(i.tcp_pcb_purge)
    i.tcp_pcb_remove                         0x08006950   Section        0  tcp.o(i.tcp_pcb_remove)
    i.tcp_poll                               0x08006a00   Section        0  tcp.o(i.tcp_poll)
    i.tcp_process                            0x08006a0c   Section        0  tcp_in.o(i.tcp_process)
    tcp_process                              0x08006a0d   Thumb Code  1426  tcp_in.o(i.tcp_process)
    i.tcp_receive                            0x08006fb8   Section        0  tcp_in.o(i.tcp_receive)
    tcp_receive                              0x08006fb9   Thumb Code  1772  tcp_in.o(i.tcp_receive)
    i.tcp_recv                               0x080076b8   Section        0  tcp.o(i.tcp_recv)
    i.tcp_recv_null                          0x080076be   Section        0  tcp.o(i.tcp_recv_null)
    tcp_recv_null                            0x080076bf   Thumb Code    40  tcp.o(i.tcp_recv_null)
    i.tcp_recved                             0x080076e6   Section        0  tcp.o(i.tcp_recved)
    i.tcp_rexmit                             0x0800773a   Section        0  tcp_out.o(i.tcp_rexmit)
    i.tcp_rst                                0x08007790   Section        0  tcp_out.o(i.tcp_rst)
    i.tcp_seg_free                           0x0800783e   Section        0  tcp.o(i.tcp_seg_free)
    i.tcp_segs_free                          0x0800785e   Section        0  tcp.o(i.tcp_segs_free)
    i.tcp_send_ctrl                          0x0800787c   Section        0  tcp_out.o(i.tcp_send_ctrl)
    i.tcp_sent                               0x08007898   Section        0  tcp.o(i.tcp_sent)
    i.tcp_setprio                            0x0800789e   Section        0  tcp.o(i.tcp_setprio)
    i.tcp_timewait_input                     0x080078a4   Section        0  tcp_in.o(i.tcp_timewait_input)
    tcp_timewait_input                       0x080078a5   Thumb Code    72  tcp_in.o(i.tcp_timewait_input)
    i.tcp_update_rcv_ann_wnd                 0x080078f4   Section        0  tcp.o(i.tcp_update_rcv_ann_wnd)
    i.tcp_write                              0x0800792c   Section        0  tcp_out.o(i.tcp_write)
    i.update_arp_entry                       0x08007974   Section        0  etharp.o(i.update_arp_entry)
    update_arp_entry                         0x08007975   Thumb Code   244  etharp.o(i.update_arp_entry)
    i.usart1_Configuration                   0x08007a6c   Section        0  usart1.o(i.usart1_Configuration)
    .constdata                               0x08007b30   Section       76  tcpclient.o(.constdata)
    __FUNCTION__                             0x08007b30   Data          23  tcpclient.o(.constdata)
    __FUNCTION__                             0x08007b47   Data          16  tcpclient.o(.constdata)
    __FUNCTION__                             0x08007b57   Data          17  tcpclient.o(.constdata)
    __FUNCTION__                             0x08007b68   Data          20  tcpclient.o(.constdata)
    .constdata                               0x08007b7c   Section       62  tcpserver.o(.constdata)
    __FUNCTION__                             0x08007b7c   Data          22  tcpserver.o(.constdata)
    __FUNCTION__                             0x08007b92   Data          20  tcpserver.o(.constdata)
    __FUNCTION__                             0x08007ba6   Data          20  tcpserver.o(.constdata)
    .constdata                               0x08007bba   Section      256  os_core.o(.constdata)
    .constdata                               0x08007cba   Section       28  memp.o(.constdata)
    memp_sizes                               0x08007cba   Data          14  memp.o(.constdata)
    memp_num                                 0x08007cc8   Data          14  memp.o(.constdata)
    .constdata                               0x08007cd6   Section       30  tcp.o(.constdata)
    __FUNCTION__                             0x08007cea   Data          10  tcp.o(.constdata)
    .constdata                               0x08007cf4   Section        8  ip_addr.o(.constdata)
    .constdata                               0x08007cfc   Section       12  etharp.o(.constdata)
    .data                                    0x20000000   Section       16  stm32_eth.o(.data)
    .data                                    0x20000010   Section       24  tcpclient.o(.data)
    TcpClient_len                            0x20000010   Data           4  tcpclient.o(.data)
    .data                                    0x20000028   Section       12  tcpserver.o(.data)
    TcpServer_len                            0x20000028   Data           4  tcpserver.o(.data)
    tcp_echoserver_pcb                       0x2000002c   Data           4  tcpserver.o(.data)
    .data                                    0x20000034   Section        4  printf.o(.data)
    .data                                    0x20000038   Section        4  usart1.o(.data)
    RX_SIZ                                   0x20000038   Data           4  usart1.o(.data)
    .data                                    0x2000003c   Section        4  delay.o(.data)
    fac_us                                   0x2000003c   Data           1  delay.o(.data)
    fac_ms                                   0x2000003e   Data           2  delay.o(.data)
    .data                                    0x20000040   Section       72  os_core.o(.data)
    .data                                    0x20000088   Section       20  ethernetif.o(.data)
    .data                                    0x2000009c   Section       13  mem.o(.data)
    ram                                      0x2000009c   Data           4  mem.o(.data)
    ram_end                                  0x200000a0   Data           4  mem.o(.data)
    lfree                                    0x200000a4   Data           4  mem.o(.data)
    mem_sem                                  0x200000a8   Data           1  mem.o(.data)
    .data                                    0x200000ac   Section        9  netif.o(.data)
    netifnum                                 0x200000b4   Data           1  netif.o(.data)
    .data                                    0x200000b8   Section       32  tcp.o(.data)
    tcp_timer                                0x200000d0   Data           1  tcp.o(.data)
    port                                     0x200000d2   Data           2  tcp.o(.data)
    iss                                      0x200000d4   Data           4  tcp.o(.data)
    .data                                    0x200000d8   Section       32  tcp_in.o(.data)
    tcphdr                                   0x200000d8   Data           4  tcp_in.o(.data)
    iphdr                                    0x200000dc   Data           4  tcp_in.o(.data)
    seqno                                    0x200000e0   Data           4  tcp_in.o(.data)
    ackno                                    0x200000e4   Data           4  tcp_in.o(.data)
    flags                                    0x200000e8   Data           1  tcp_in.o(.data)
    tcplen                                   0x200000ea   Data           2  tcp_in.o(.data)
    recv_flags                               0x200000ec   Data           1  tcp_in.o(.data)
    recv_data                                0x200000f0   Data           4  tcp_in.o(.data)
    .data                                    0x200000f8   Section       10  ip.o(.data)
    current_netif                            0x200000f8   Data           4  ip.o(.data)
    current_header                           0x200000fc   Data           4  ip.o(.data)
    ip_id                                    0x20000100   Data           2  ip.o(.data)
    .data                                    0x20000104   Section        6  ip_frag.o(.data)
    reassdatagrams                           0x20000104   Data           4  ip_frag.o(.data)
    ip_reass_pbufcount                       0x20000108   Data           2  ip_frag.o(.data)
    .data                                    0x2000010a   Section        1  etharp.o(.data)
    etharp_cached_entry                      0x2000010a   Data           1  etharp.o(.data)
    .data                                    0x2000010b   Section       20  stm32f10x_rcc.o(.data)
    APBAHBPrescTable                         0x2000010b   Data          16  stm32f10x_rcc.o(.data)
    ADCPrescTable                            0x2000011b   Data           4  stm32f10x_rcc.o(.data)
    .data                                    0x20000120   Section       20  system_stm32f10x.o(.data)
    .bss                                     0x20000134   Section       48  netconf.o(.bss)
    .bss                                     0x20000164   Section      200  tcpclient.o(.bss)
    TcpClient_buff                           0x20000164   Data         200  tcpclient.o(.bss)
    .bss                                     0x2000022c   Section      200  tcpserver.o(.bss)
    TcpServer_buff                           0x2000022c   Data         200  tcpserver.o(.bss)
    .bss                                     0x200002f4   Section      200  usart1.o(.bss)
    RX_BUFF                                  0x200002f4   Data         200  usart1.o(.bss)
    .bss                                     0x200003bc   Section     8448  stm32_config.o(.bss)
    .bss                                     0x200024bc   Section     2604  os_core.o(.bss)
    .bss                                     0x20002ee8   Section     9216  ethernetif.o(.bss)
    .bss                                     0x200052e8   Section     1044  mem.o(.bss)
    ram_heap                                 0x200052e8   Data        1044  mem.o(.bss)
    .bss                                     0x200056fc   Section     2687  memp.o(.bss)
    memp_tab                                 0x200056fc   Data          28  memp.o(.bss)
    memp_memory                              0x20005718   Data        2659  memp.o(.bss)
    .bss                                     0x2000617c   Section       20  tcp_in.o(.bss)
    inseg                                    0x2000617c   Data          20  tcp_in.o(.bss)
    .bss                                     0x20006190   Section     1504  ip_frag.o(.bss)
    buf                                      0x20006190   Data        1504  ip_frag.o(.bss)
    .bss                                     0x20006770   Section      200  etharp.o(.bss)
    arp_table                                0x20006770   Data         200  etharp.o(.bss)
    STACK                                    0x20006838   Section     1024  startup_stm32f10x_cl.o(STACK)

    Global Symbols

    Symbol Name                              Value     Ov Type        Size  Object(Section)

    BuildAttributes$$THM_ISAv4$P$D$K$B$S$PE$A:L22UL41UL21$X:L11$S22US41US21$IEEE1$IW$USESV6$~STKCKD$USESV7$~SHL$OSPACE$ROPI$EBA8$MICROLIB$REQ8$PRES8$EABIv2 0x00000000   Number         0  anon$$obj.o ABSOLUTE
    __ARM_use_no_argv                        0x00000000   Number         0  main.o ABSOLUTE
    _printf_a                                0x00000000   Number         0  stubs.o ABSOLUTE
    _printf_c                                0x00000000   Number         0  stubs.o ABSOLUTE
    _printf_charcount                        0x00000000   Number         0  stubs.o ABSOLUTE
    _printf_d                                0x00000000   Number         0  stubs.o ABSOLUTE
    _printf_e                                0x00000000   Number         0  stubs.o ABSOLUTE
    _printf_f                                0x00000000   Number         0  stubs.o ABSOLUTE
    _printf_flags                            0x00000000   Number         0  stubs.o ABSOLUTE
    _printf_fp_dec                           0x00000000   Number         0  stubs.o ABSOLUTE
    _printf_fp_hex                           0x00000000   Number         0  stubs.o ABSOLUTE
    _printf_g                                0x00000000   Number         0  stubs.o ABSOLUTE
    _printf_i                                0x00000000   Number         0  stubs.o ABSOLUTE
    _printf_int_dec                          0x00000000   Number         0  stubs.o ABSOLUTE
    _printf_l                                0x00000000   Number         0  stubs.o ABSOLUTE
    _printf_lc                               0x00000000   Number         0  stubs.o ABSOLUTE
    _printf_ll                               0x00000000   Number         0  stubs.o ABSOLUTE
    _printf_lld                              0x00000000   Number         0  stubs.o ABSOLUTE
    _printf_lli                              0x00000000   Number         0  stubs.o ABSOLUTE
    _printf_llo                              0x00000000   Number         0  stubs.o ABSOLUTE
    _printf_llu                              0x00000000   Number         0  stubs.o ABSOLUTE
    _printf_llx                              0x00000000   Number         0  stubs.o ABSOLUTE
    _printf_longlong_dec                     0x00000000   Number         0  stubs.o ABSOLUTE
    _printf_longlong_hex                     0x00000000   Number         0  stubs.o ABSOLUTE
    _printf_longlong_oct                     0x00000000   Number         0  stubs.o ABSOLUTE
    _printf_ls                               0x00000000   Number         0  stubs.o ABSOLUTE
    _printf_mbtowc                           0x00000000   Number         0  stubs.o ABSOLUTE
    _printf_n                                0x00000000   Number         0  stubs.o ABSOLUTE
    _printf_o                                0x00000000   Number         0  stubs.o ABSOLUTE
    _printf_p                                0x00000000   Number         0  stubs.o ABSOLUTE
    _printf_percent                          0x00000000   Number         0  stubs.o ABSOLUTE
    _printf_pre_padding                      0x00000000   Number         0  stubs.o ABSOLUTE
    _printf_return_value                     0x00000000   Number         0  stubs.o ABSOLUTE
    _printf_s                                0x00000000   Number         0  stubs.o ABSOLUTE
    _printf_sizespec                         0x00000000   Number         0  stubs.o ABSOLUTE
    _printf_str                              0x00000000   Number         0  stubs.o ABSOLUTE
    _printf_truncate_signed                  0x00000000   Number         0  stubs.o ABSOLUTE
    _printf_truncate_unsigned                0x00000000   Number         0  stubs.o ABSOLUTE
    _printf_u                                0x00000000   Number         0  stubs.o ABSOLUTE
    _printf_wc                               0x00000000   Number         0  stubs.o ABSOLUTE
    _printf_wctomb                           0x00000000   Number         0  stubs.o ABSOLUTE
    _printf_widthprec                        0x00000000   Number         0  stubs.o ABSOLUTE
    _printf_x                                0x00000000   Number         0  stubs.o ABSOLUTE
    __cpp_initialize__aeabi_                  - Undefined Weak Reference
    __cxa_finalize                            - Undefined Weak Reference
    _clock_init                               - Undefined Weak Reference
    _microlib_exit                            - Undefined Weak Reference
    __Vectors_Size                           0x00000150   Number         0  startup_stm32f10x_cl.o ABSOLUTE
    __Vectors                                0x08000000   Data           4  startup_stm32f10x_cl.o(RESET)
    __Vectors_End                            0x08000150   Data           0  startup_stm32f10x_cl.o(RESET)
    __main                                   0x08000151   Thumb Code     0  entry.o(.ARM.Collect$$$$00000000)
    _main_stk                                0x08000151   Thumb Code     0  entry2.o(.ARM.Collect$$$$00000001)
    _main_scatterload                        0x08000155   Thumb Code     0  entry5.o(.ARM.Collect$$$$00000004)
    __main_after_scatterload                 0x08000159   Thumb Code     0  entry5.o(.ARM.Collect$$$$00000004)
    _main_clock                              0x08000159   Thumb Code     0  entry7b.o(.ARM.Collect$$$$00000008)
    _main_cpp_init                           0x08000159   Thumb Code     0  entry8b.o(.ARM.Collect$$$$0000000A)
    _main_init                               0x08000159   Thumb Code     0  entry9a.o(.ARM.Collect$$$$0000000B)
    __rt_final_cpp                           0x08000161   Thumb Code     0  entry10a.o(.ARM.Collect$$$$0000000D)
    __rt_final_exit                          0x08000161   Thumb Code     0  entry11a.o(.ARM.Collect$$$$0000000F)
    OS_CPU_SR_Save                           0x08000165   Thumb Code     0  os_cpu_a.o(.text)
    OS_CPU_SR_Restore                        0x0800016d   Thumb Code     0  os_cpu_a.o(.text)
    OSStartHighRdy                           0x08000173   Thumb Code     0  os_cpu_a.o(.text)
    OSCtxSw                                  0x08000195   Thumb Code     0  os_cpu_a.o(.text)
    OSIntCtxSw                               0x080001a3   Thumb Code     0  os_cpu_a.o(.text)
    PendSV_Handler                           0x080001b3   Thumb Code     0  os_cpu_a.o(.text)
    Reset_Handler                            0x08000219   Thumb Code     8  startup_stm32f10x_cl.o(.text)
    ADC1_2_IRQHandler                        0x08000233   Thumb Code     0  startup_stm32f10x_cl.o(.text)
    CAN1_RX0_IRQHandler                      0x08000233   Thumb Code     0  startup_stm32f10x_cl.o(.text)
    CAN1_RX1_IRQHandler                      0x08000233   Thumb Code     0  startup_stm32f10x_cl.o(.text)
    CAN1_SCE_IRQHandler                      0x08000233   Thumb Code     0  startup_stm32f10x_cl.o(.text)
    CAN1_TX_IRQHandler                       0x08000233   Thumb Code     0  startup_stm32f10x_cl.o(.text)
    CAN2_RX0_IRQHandler                      0x08000233   Thumb Code     0  startup_stm32f10x_cl.o(.text)
    CAN2_RX1_IRQHandler                      0x08000233   Thumb Code     0  startup_stm32f10x_cl.o(.text)
    CAN2_SCE_IRQHandler                      0x08000233   Thumb Code     0  startup_stm32f10x_cl.o(.text)
    CAN2_TX_IRQHandler                       0x08000233   Thumb Code     0  startup_stm32f10x_cl.o(.text)
    DMA1_Channel1_IRQHandler                 0x08000233   Thumb Code     0  startup_stm32f10x_cl.o(.text)
    DMA1_Channel2_IRQHandler                 0x08000233   Thumb Code     0  startup_stm32f10x_cl.o(.text)
    DMA1_Channel3_IRQHandler                 0x08000233   Thumb Code     0  startup_stm32f10x_cl.o(.text)
    DMA1_Channel4_IRQHandler                 0x08000233   Thumb Code     0  startup_stm32f10x_cl.o(.text)
    DMA1_Channel5_IRQHandler                 0x08000233   Thumb Code     0  startup_stm32f10x_cl.o(.text)
    DMA1_Channel6_IRQHandler                 0x08000233   Thumb Code     0  startup_stm32f10x_cl.o(.text)
    DMA1_Channel7_IRQHandler                 0x08000233   Thumb Code     0  startup_stm32f10x_cl.o(.text)
    DMA2_Channel1_IRQHandler                 0x08000233   Thumb Code     0  startup_stm32f10x_cl.o(.text)
    DMA2_Channel2_IRQHandler                 0x08000233   Thumb Code     0  startup_stm32f10x_cl.o(.text)
    DMA2_Channel3_IRQHandler                 0x08000233   Thumb Code     0  startup_stm32f10x_cl.o(.text)
    DMA2_Channel4_IRQHandler                 0x08000233   Thumb Code     0  startup_stm32f10x_cl.o(.text)
    DMA2_Channel5_IRQHandler                 0x08000233   Thumb Code     0  startup_stm32f10x_cl.o(.text)
    ETH_WKUP_IRQHandler                      0x08000233   Thumb Code     0  startup_stm32f10x_cl.o(.text)
    EXTI0_IRQHandler                         0x08000233   Thumb Code     0  startup_stm32f10x_cl.o(.text)
    EXTI15_10_IRQHandler                     0x08000233   Thumb Code     0  startup_stm32f10x_cl.o(.text)
    EXTI1_IRQHandler                         0x08000233   Thumb Code     0  startup_stm32f10x_cl.o(.text)
    EXTI2_IRQHandler                         0x08000233   Thumb Code     0  startup_stm32f10x_cl.o(.text)
    EXTI3_IRQHandler                         0x08000233   Thumb Code     0  startup_stm32f10x_cl.o(.text)
    EXTI4_IRQHandler                         0x08000233   Thumb Code     0  startup_stm32f10x_cl.o(.text)
    EXTI9_5_IRQHandler                       0x08000233   Thumb Code     0  startup_stm32f10x_cl.o(.text)
    FLASH_IRQHandler                         0x08000233   Thumb Code     0  startup_stm32f10x_cl.o(.text)
    I2C1_ER_IRQHandler                       0x08000233   Thumb Code     0  startup_stm32f10x_cl.o(.text)
    I2C1_EV_IRQHandler                       0x08000233   Thumb Code     0  startup_stm32f10x_cl.o(.text)
    I2C2_ER_IRQHandler                       0x08000233   Thumb Code     0  startup_stm32f10x_cl.o(.text)
    I2C2_EV_IRQHandler                       0x08000233   Thumb Code     0  startup_stm32f10x_cl.o(.text)
    OTG_FS_IRQHandler                        0x08000233   Thumb Code     0  startup_stm32f10x_cl.o(.text)
    OTG_FS_WKUP_IRQHandler                   0x08000233   Thumb Code     0  startup_stm32f10x_cl.o(.text)
    PVD_IRQHandler                           0x08000233   Thumb Code     0  startup_stm32f10x_cl.o(.text)
    RCC_IRQHandler                           0x08000233   Thumb Code     0  startup_stm32f10x_cl.o(.text)
    RTCAlarm_IRQHandler                      0x08000233   Thumb Code     0  startup_stm32f10x_cl.o(.text)
    RTC_IRQHandler                           0x08000233   Thumb Code     0  startup_stm32f10x_cl.o(.text)
    SPI1_IRQHandler                          0x08000233   Thumb Code     0  startup_stm32f10x_cl.o(.text)
    SPI2_IRQHandler                          0x08000233   Thumb Code     0  startup_stm32f10x_cl.o(.text)
    SPI3_IRQHandler                          0x08000233   Thumb Code     0  startup_stm32f10x_cl.o(.text)
    TAMPER_IRQHandler                        0x08000233   Thumb Code     0  startup_stm32f10x_cl.o(.text)
    TIM1_BRK_IRQHandler                      0x08000233   Thumb Code     0  startup_stm32f10x_cl.o(.text)
    TIM1_CC_IRQHandler                       0x08000233   Thumb Code     0  startup_stm32f10x_cl.o(.text)
    TIM1_TRG_COM_IRQHandler                  0x08000233   Thumb Code     0  startup_stm32f10x_cl.o(.text)
    TIM1_UP_IRQHandler                       0x08000233   Thumb Code     0  startup_stm32f10x_cl.o(.text)
    TIM2_IRQHandler                          0x08000233   Thumb Code     0  startup_stm32f10x_cl.o(.text)
    TIM3_IRQHandler                          0x08000233   Thumb Code     0  startup_stm32f10x_cl.o(.text)
    TIM4_IRQHandler                          0x08000233   Thumb Code     0  startup_stm32f10x_cl.o(.text)
    TIM5_IRQHandler                          0x08000233   Thumb Code     0  startup_stm32f10x_cl.o(.text)
    TIM6_IRQHandler                          0x08000233   Thumb Code     0  startup_stm32f10x_cl.o(.text)
    TIM7_IRQHandler                          0x08000233   Thumb Code     0  startup_stm32f10x_cl.o(.text)
    UART4_IRQHandler                         0x08000233   Thumb Code     0  startup_stm32f10x_cl.o(.text)
    UART5_IRQHandler                         0x08000233   Thumb Code     0  startup_stm32f10x_cl.o(.text)
    USART2_IRQHandler                        0x08000233   Thumb Code     0  startup_stm32f10x_cl.o(.text)
    USART3_IRQHandler                        0x08000233   Thumb Code     0  startup_stm32f10x_cl.o(.text)
    WWDG_IRQHandler                          0x08000233   Thumb Code     0  startup_stm32f10x_cl.o(.text)
    __aeabi_memcpy                           0x0800023d   Thumb Code    36  memcpya.o(.text)
    __aeabi_memcpy4                          0x0800023d   Thumb Code     0  memcpya.o(.text)
    __aeabi_memcpy8                          0x0800023d   Thumb Code     0  memcpya.o(.text)
    __aeabi_memset                           0x08000261   Thumb Code    14  memseta.o(.text)
    __aeabi_memset4                          0x08000261   Thumb Code     0  memseta.o(.text)
    __aeabi_memset8                          0x08000261   Thumb Code     0  memseta.o(.text)
    __aeabi_memclr                           0x0800026f   Thumb Code     4  memseta.o(.text)
    __aeabi_memclr4                          0x0800026f   Thumb Code     0  memseta.o(.text)
    __aeabi_memclr8                          0x0800026f   Thumb Code     0  memseta.o(.text)
    _memset$wrapper                          0x08000273   Thumb Code    18  memseta.o(.text)
    __aeabi_uidiv                            0x08000285   Thumb Code     0  uidiv.o(.text)
    __aeabi_uidivmod                         0x08000285   Thumb Code    44  uidiv.o(.text)
    __scatterload                            0x080002b1   Thumb Code    28  init.o(.text)
    __scatterload_rt2                        0x080002b1   Thumb Code     0  init.o(.text)
    __decompress                             0x080002d5   Thumb Code     0  __dczerorl2.o(.text)
    __decompress1                            0x080002d5   Thumb Code    86  __dczerorl2.o(.text)
    BusFault_Handler                         0x0800032d   Thumb Code    10  stm32f10x_it.o(i.BusFault_Handler)
    DebugMon_Handler                         0x08000355   Thumb Code     2  stm32f10x_it.o(i.DebugMon_Handler)
    ETH_DMAClearITPendingBit                 0x08000359   Thumb Code     6  stm32_eth.o(i.ETH_DMAClearITPendingBit)
    ETH_DMAITConfig                          0x08000365   Thumb Code    26  stm32_eth.o(i.ETH_DMAITConfig)
    ETH_DMAReceptionCmd                      0x08000385   Thumb Code    30  stm32_eth.o(i.ETH_DMAReceptionCmd)
    ETH_DMARxDescChainInit                   0x080003a9   Thumb Code    76  stm32_eth.o(i.ETH_DMARxDescChainInit)
    ETH_DMARxDescReceiveITConfig             0x080003fd   Thumb Code    22  stm32_eth.o(i.ETH_DMARxDescReceiveITConfig)
    ETH_DMATransmissionCmd                   0x08000415   Thumb Code    30  stm32_eth.o(i.ETH_DMATransmissionCmd)
    ETH_DMATxDescChainInit                   0x08000439   Thumb Code    70  stm32_eth.o(i.ETH_DMATxDescChainInit)
    ETH_DMATxDescChecksumInsertionConfig     0x08000489   Thumb Code     8  stm32_eth.o(i.ETH_DMATxDescChecksumInsertionConfig)
    ETH_DeInit                               0x08000491   Thumb Code    22  stm32_eth.o(i.ETH_DeInit)
    ETH_FlushTransmitFIFO                    0x080004c5   Thumb Code    14  stm32_eth.o(i.ETH_FlushTransmitFIFO)
    ETH_GetCurrentTxBuffer                   0x080004d9   Thumb Code     8  ethernetif.o(i.ETH_GetCurrentTxBuffer)
    ETH_GetDMARxDescFrameLength              0x080004e5   Thumb Code    10  stm32_eth.o(i.ETH_GetDMARxDescFrameLength)
    ETH_GetRxPktSize                         0x080004f1   Thumb Code    66  stm32_eth.o(i.ETH_GetRxPktSize)
    ETH_GetSoftwareResetStatus               0x08000539   Thumb Code    20  stm32_eth.o(i.ETH_GetSoftwareResetStatus)
    ETH_IRQHandler                           0x08000551   Thumb Code    40  stm32f10x_it.o(i.ETH_IRQHandler)
    ETH_Init                                 0x08000579   Thumb Code   576  stm32_eth.o(i.ETH_Init)
    ETH_MACAddressConfig                     0x080007dd   Thumb Code    46  stm32_eth.o(i.ETH_MACAddressConfig)
    ETH_MACReceptionCmd                      0x08000811   Thumb Code    30  stm32_eth.o(i.ETH_MACReceptionCmd)
    ETH_MACTransmissionCmd                   0x08000835   Thumb Code    30  stm32_eth.o(i.ETH_MACTransmissionCmd)
    ETH_ReadPHYRegister                      0x08000859   Thumb Code    98  stm32_eth.o(i.ETH_ReadPHYRegister)
    ETH_RxPkt_ChainMode                      0x080008c5   Thumb Code   148  ethernetif.o(i.ETH_RxPkt_ChainMode)
    ETH_SoftwareReset                        0x08000961   Thumb Code    14  stm32_eth.o(i.ETH_SoftwareReset)
    ETH_Start                                0x08000975   Thumb Code    32  stm32_eth.o(i.ETH_Start)
    ETH_StructInit                           0x08000995   Thumb Code   164  stm32_eth.o(i.ETH_StructInit)
    ETH_TxPkt_ChainMode                      0x08000a39   Thumb Code    94  ethernetif.o(i.ETH_TxPkt_ChainMode)
    ETH_WritePHYRegister                     0x08000aa1   Thumb Code    96  stm32_eth.o(i.ETH_WritePHYRegister)
    Ethernet_Configuration                   0x08000b09   Thumb Code   170  stm32f107.o(i.Ethernet_Configuration)
    GPIO_Configuration                       0x08000bb9   Thumb Code   164  stm32f107.o(i.GPIO_Configuration)
    GPIO_ETH_MediaInterfaceConfig            0x08000c69   Thumb Code     6  stm32f10x_gpio.o(i.GPIO_ETH_MediaInterfaceConfig)
    GPIO_Init                                0x08000c75   Thumb Code   278  stm32f10x_gpio.o(i.GPIO_Init)
    GPIO_PinRemapConfig                      0x08000d8d   Thumb Code   138  stm32f10x_gpio.o(i.GPIO_PinRemapConfig)
    HardFault_Handler                        0x08000e1d   Thumb Code    10  stm32f10x_it.o(i.HardFault_Handler)
    LwIP_Init                                0x08000e45   Thumb Code    94  netconf.o(i.LwIP_Init)
    LwIP_Pkt_Handle                          0x08000ebd   Thumb Code    10  netconf.o(i.LwIP_Pkt_Handle)
    MemManage_Handler                        0x08000ecd   Thumb Code    10  stm32f10x_it.o(i.MemManage_Handler)
    NMI_Handler                              0x08000ef5   Thumb Code     2  stm32f10x_it.o(i.NMI_Handler)
    NVIC_Configuration                       0x08000ef7   Thumb Code    52  stm32f107.o(i.NVIC_Configuration)
    NVIC_Init                                0x08000f2d   Thumb Code   100  misc.o(i.NVIC_Init)
    NVIC_PriorityGroupConfig                 0x08000f9d   Thumb Code    10  misc.o(i.NVIC_PriorityGroupConfig)
    NVIC_SetVectorTable                      0x08000fd9   Thumb Code    12  misc.o(i.NVIC_SetVectorTable)
    OSInit                                   0x08000fed   Thumb Code    44  os_core.o(i.OSInit)
    OSInitHookBegin                          0x08001019   Thumb Code     2  os_cpu_c.o(i.OSInitHookBegin)
    OSInitHookEnd                            0x0800101b   Thumb Code     2  os_cpu_c.o(i.OSInitHookEnd)
    OSIntEnter                               0x0800101d   Thumb Code    28  os_core.o(i.OSIntEnter)
    OSIntExit                                0x08001041   Thumb Code   112  os_core.o(i.OSIntExit)
    OSStart                                  0x080010d1   Thumb Code    48  os_core.o(i.OSStart)
    OSStatInit                               0x08001119   Thumb Code    62  os_core.o(i.OSStatInit)
    OSTCBInitHook                            0x08001165   Thumb Code     2  os_cpu_c.o(i.OSTCBInitHook)
    OSTaskCreate                             0x08001169   Thumb Code   148  os_task.o(i.OSTaskCreate)
    OSTaskCreateExt                          0x08001209   Thumb Code   170  os_task.o(i.OSTaskCreateExt)
    OSTaskCreateHook                         0x080012c1   Thumb Code     2  os_cpu_c.o(i.OSTaskCreateHook)
    OSTaskIdleHook                           0x080012c3   Thumb Code     2  os_cpu_c.o(i.OSTaskIdleHook)
    OSTaskNameSet                            0x080012c5   Thumb Code    98  os_task.o(i.OSTaskNameSet)
    OSTaskStatHook                           0x08001335   Thumb Code     2  os_cpu_c.o(i.OSTaskStatHook)
    OSTaskStkChk                             0x08001339   Thumb Code   132  os_task.o(i.OSTaskStkChk)
    OSTaskStkInit                            0x080013c5   Thumb Code   154  os_cpu_c.o(i.OSTaskStkInit)
    OSTaskSuspend                            0x08001461   Thumb Code   152  os_task.o(i.OSTaskSuspend)
    OSTaskSwHook                             0x08001509   Thumb Code     2  os_cpu_c.o(i.OSTaskSwHook)
    OSTimeDly                                0x0800150d   Thumb Code   100  os_time.o(i.OSTimeDly)
    OSTimeTick                               0x08001585   Thumb Code   210  os_core.o(i.OSTimeTick)
    OSTimeTickHook                           0x08001671   Thumb Code     2  os_cpu_c.o(i.OSTimeTickHook)
    OS_FlagInit                              0x08001675   Thumb Code    74  os_flag.o(i.OS_FlagInit)
    OS_MemClr                                0x080018d9   Thumb Code    18  os_core.o(i.OS_MemClr)
    OS_QInit                                 0x080018ed   Thumb Code    72  os_q.o(i.OS_QInit)
    OS_Sched                                 0x0800193d   Thumb Code    88  os_core.o(i.OS_Sched)
    OS_TCBInit                               0x080019dd   Thumb Code   278  os_core.o(i.OS_TCBInit)
    OS_TaskIdle                              0x08001b11   Thumb Code    34  os_core.o(i.OS_TaskIdle)
    OS_TaskStat                              0x08001b39   Thumb Code   116  os_core.o(i.OS_TaskStat)
    OS_TaskStatStkChk                        0x08001bc1   Thumb Code    54  os_core.o(i.OS_TaskStatStkChk)
    OS_TaskStkClr                            0x08001bfd   Thumb Code    26  os_task.o(i.OS_TaskStkClr)
    RCC_AHBPeriphClockCmd                    0x08001c19   Thumb Code    26  stm32f10x_rcc.o(i.RCC_AHBPeriphClockCmd)
    RCC_AHBPeriphResetCmd                    0x08001c39   Thumb Code    26  stm32f10x_rcc.o(i.RCC_AHBPeriphResetCmd)
    RCC_APB1PeriphClockCmd                   0x08001c59   Thumb Code    26  stm32f10x_rcc.o(i.RCC_APB1PeriphClockCmd)
    RCC_APB2PeriphClockCmd                   0x08001c79   Thumb Code    26  stm32f10x_rcc.o(i.RCC_APB2PeriphClockCmd)
    RCC_GetClocksFreq                        0x08001c99   Thumb Code   374  stm32f10x_rcc.o(i.RCC_GetClocksFreq)
    RCC_GetFlagStatus                        0x08001e29   Thumb Code    56  stm32f10x_rcc.o(i.RCC_GetFlagStatus)
    RCC_MCOConfig                            0x08001e65   Thumb Code     6  stm32f10x_rcc.o(i.RCC_MCOConfig)
    RCC_PLL3Cmd                              0x08001e71   Thumb Code     6  stm32f10x_rcc.o(i.RCC_PLL3Cmd)
    RCC_PLL3Config                           0x08001e7d   Thumb Code    18  stm32f10x_rcc.o(i.RCC_PLL3Config)
    SVC_Handler                              0x08001e95   Thumb Code     2  stm32f10x_it.o(i.SVC_Handler)
    Set_MAC_Address                          0x08001fb9   Thumb Code    40  ethernetif.o(i.Set_MAC_Address)
    SysTick_CLKSourceConfig                  0x08001fe5   Thumb Code    40  misc.o(i.SysTick_CLKSourceConfig)
    SysTick_Handler                          0x0800200d   Thumb Code    16  delay.o(i.SysTick_Handler)
    SystemInit                               0x0800201d   Thumb Code    92  system_stm32f10x.o(i.SystemInit)
    System_Setup                             0x08002089   Thumb Code   118  stm32f107.o(i.System_Setup)
    TCP_Client_Recv                          0x08002101   Thumb Code    56  tcpclient.o(i.TCP_Client_Recv)
    TCP_Client_Send                          0x08002141   Thumb Code    48  tcpclient.o(i.TCP_Client_Send)
    TCP_Server_Recv                          0x08002175   Thumb Code    56  tcpserver.o(i.TCP_Server_Recv)
    TCP_Server_Send                          0x080021b5   Thumb Code    48  tcpserver.o(i.TCP_Server_Send)
    USART1_IRQHandler                        0x080021e9   Thumb Code    94  usart1.o(i.USART1_IRQHandler)
    USART_ClearFlag                          0x08002255   Thumb Code    18  stm32f10x_usart.o(i.USART_ClearFlag)
    USART_ClearITPendingBit                  0x08002267   Thumb Code    30  stm32f10x_usart.o(i.USART_ClearITPendingBit)
    USART_Cmd                                0x08002285   Thumb Code    24  stm32f10x_usart.o(i.USART_Cmd)
    USART_GetFlagStatus                      0x0800229d   Thumb Code    26  stm32f10x_usart.o(i.USART_GetFlagStatus)
    USART_GetITStatus                        0x080022b7   Thumb Code    84  stm32f10x_usart.o(i.USART_GetITStatus)
    USART_ITConfig                           0x0800230b   Thumb Code    74  stm32f10x_usart.o(i.USART_ITConfig)
    USART_Init                               0x08002355   Thumb Code   210  stm32f10x_usart.o(i.USART_Init)
    USART_ReceiveData                        0x0800242d   Thumb Code    10  stm32f10x_usart.o(i.USART_ReceiveData)
    USART_SendData                           0x08002437   Thumb Code     8  stm32f10x_usart.o(i.USART_SendData)
    UsageFault_Handler                       0x08002441   Thumb Code    10  stm32f10x_it.o(i.UsageFault_Handler)
    __0printf$3                              0x0800246d   Thumb Code    22  printf3.o(i.__0printf$3)
    __1printf$3                              0x0800246d   Thumb Code     0  printf3.o(i.__0printf$3)
    __2printf                                0x0800246d   Thumb Code     0  printf3.o(i.__0printf$3)
    __scatterload_copy                       0x0800248d   Thumb Code    14  handlers.o(i.__scatterload_copy)
    __scatterload_null                       0x0800249b   Thumb Code     2  handlers.o(i.__scatterload_null)
    __scatterload_zeroinit                   0x0800249d   Thumb Code    14  handlers.o(i.__scatterload_zeroinit)
    delay_init                               0x08002665   Thumb Code    76  delay.o(i.delay_init)
    delay_ms                                 0x080026c1   Thumb Code    62  delay.o(i.delay_ms)
    delay_us                                 0x08002709   Thumb Code    70  delay.o(i.delay_us)
    etharp_arp_input                         0x08002755   Thumb Code   306  etharp.o(i.etharp_arp_input)
    etharp_ip_input                          0x08002887   Thumb Code    58  etharp.o(i.etharp_ip_input)
    etharp_output                            0x080028c1   Thumb Code   190  etharp.o(i.etharp_output)
    etharp_query                             0x08002985   Thumb Code   436  etharp.o(i.etharp_query)
    etharp_request                           0x08002c09   Thumb Code    36  etharp.o(i.etharp_request)
    ethernet_input                           0x08002c83   Thumb Code   106  etharp.o(i.ethernet_input)
    ethernetif_init                          0x08002ced   Thumb Code    68  ethernetif.o(i.ethernetif_init)
    ethernetif_input                         0x08002d39   Thumb Code    44  ethernetif.o(i.ethernetif_input)
    fputc                                    0x08002f69   Thumb Code    32  printf.o(i.fputc)
    htonl                                    0x08002fcd   Thumb Code    26  inet.o(i.htonl)
    htons                                    0x08002fe7   Thumb Code    12  inet.o(i.htons)
    icmp_dest_unreach                        0x08002ff3   Thumb Code    18  icmp.o(i.icmp_dest_unreach)
    icmp_input                               0x08003005   Thumb Code   404  icmp.o(i.icmp_input)
    icmp_time_exceeded                       0x0800320f   Thumb Code    18  icmp.o(i.icmp_time_exceeded)
    inet_chksum                              0x08003221   Thumb Code    20  inet_chksum.o(i.inet_chksum)
    inet_chksum_pbuf                         0x08003235   Thumb Code    86  inet_chksum.o(i.inet_chksum_pbuf)
    ip_addr_isbroadcast                      0x0800328b   Thumb Code    78  ip_addr.o(i.ip_addr_isbroadcast)
    ip_frag                                  0x080032d9   Thumb Code   326  ip_frag.o(i.ip_frag)
    ip_input                                 0x08003425   Thumb Code   374  ip.o(i.ip_input)
    ip_output                                0x080035a9   Thumb Code    52  ip.o(i.ip_output)
    ip_output_if                             0x080035dd   Thumb Code   256  ip.o(i.ip_output_if)
    ip_reass                                 0x080036e1   Thumb Code   400  ip_frag.o(i.ip_reass)
    ip_route                                 0x08003bd1   Thumb Code    70  ip.o(i.ip_route)
    main                                     0x08003db9   Thumb Code    44  main.o(i.main)
    main_Client_task                         0x08003ded   Thumb Code   156  main_cilent.o(i.main_Client_task)
    main_Server_task                         0x08003eed   Thumb Code    62  main_server.o(i.main_Server_task)
    mem_free                                 0x08003f4d   Thumb Code   106  mem.o(i.mem_free)
    mem_init                                 0x08003fc5   Thumb Code    78  mem.o(i.mem_init)
    mem_malloc                               0x08004029   Thumb Code   290  mem.o(i.mem_malloc)
    mem_realloc                              0x08004159   Thumb Code   316  mem.o(i.mem_realloc)
    memp_free                                0x080042a1   Thumb Code    38  memp.o(i.memp_free)
    memp_init                                0x080042cd   Thumb Code    82  memp.o(i.memp_init)
    memp_malloc                              0x08004331   Thumb Code    54  memp.o(i.memp_malloc)
    netif_add                                0x0800436d   Thumb Code    96  netif.o(i.netif_add)
    netif_is_up                              0x080043d5   Thumb Code    12  netif.o(i.netif_is_up)
    netif_set_addr                           0x080043e1   Thumb Code    40  netif.o(i.netif_set_addr)
    netif_set_default                        0x08004409   Thumb Code     6  netif.o(i.netif_set_default)
    netif_set_gw                             0x08004415   Thumb Code    12  netif.o(i.netif_set_gw)
    netif_set_ipaddr                         0x08004421   Thumb Code   110  netif.o(i.netif_set_ipaddr)
    netif_set_netmask                        0x08004499   Thumb Code    12  netif.o(i.netif_set_netmask)
    netif_set_up                             0x080044a5   Thumb Code    44  netif.o(i.netif_set_up)
    ntohl                                    0x080044d1   Thumb Code    12  inet.o(i.ntohl)
    ntohs                                    0x080044dd   Thumb Code    12  inet.o(i.ntohs)
    pbuf_alloc                               0x080044e9   Thumb Code   532  pbuf.o(i.pbuf_alloc)
    pbuf_cat                                 0x080046fd   Thumb Code    80  pbuf.o(i.pbuf_cat)
    pbuf_chain                               0x0800474d   Thumb Code    22  pbuf.o(i.pbuf_chain)
    pbuf_clen                                0x08004763   Thumb Code    18  pbuf.o(i.pbuf_clen)
    pbuf_copy                                0x08004775   Thumb Code   220  pbuf.o(i.pbuf_copy)
    pbuf_copy_partial                        0x08004851   Thumb Code   154  pbuf.o(i.pbuf_copy_partial)
    pbuf_free                                0x080048eb   Thumb Code   152  pbuf.o(i.pbuf_free)
    pbuf_header                              0x08004983   Thumb Code   140  pbuf.o(i.pbuf_header)
    pbuf_realloc                             0x08004a0f   Thumb Code   176  pbuf.o(i.pbuf_realloc)
    pbuf_ref                                 0x08004abf   Thumb Code    10  pbuf.o(i.pbuf_ref)
    start_task                               0x08004b7d   Thumb Code    84  main.o(i.start_task)
    tcp_abandon                              0x08004bf9   Thumb Code   148  tcp.o(i.tcp_abandon)
    tcp_accept                               0x08004c95   Thumb Code     4  tcp.o(i.tcp_accept)
    tcp_alloc                                0x08004ca1   Thumb Code   166  tcp.o(i.tcp_alloc)
    tcp_arg                                  0x08004d55   Thumb Code     4  tcp.o(i.tcp_arg)
    tcp_bind                                 0x08004d59   Thumb Code   232  tcp.o(i.tcp_bind)
    tcp_client_close                         0x08004e51   Thumb Code    44  tcpclient.o(i.tcp_client_close)
    tcp_close                                0x08004f09   Thumb Code   390  tcp.o(i.tcp_close)
    tcp_connect                              0x080050b9   Thumb Code   278  tcp.o(i.tcp_connect)
    tcp_echoclient_connect                   0x080051dd   Thumb Code    74  tcpclient.o(i.tcp_echoclient_connect)
    tcp_echoserver_init                      0x08005565   Thumb Code    62  tcpserver.o(i.tcp_echoserver_init)
    tcp_eff_send_mss                         0x080057d7   Thumb Code    46  tcp.o(i.tcp_eff_send_mss)
    tcp_enqueue                              0x08005805   Thumb Code  1068  tcp_out.o(i.tcp_enqueue)
    tcp_err                                  0x08005c31   Thumb Code     6  tcp.o(i.tcp_err)
    tcp_input                                0x08005c39   Thumb Code  1166  tcp_in.o(i.tcp_input)
    tcp_listen_with_backlog                  0x080062c5   Thumb Code   220  tcp.o(i.tcp_listen_with_backlog)
    tcp_new                                  0x080063b1   Thumb Code    10  tcp.o(i.tcp_new)
    tcp_next_iss                             0x08006435   Thumb Code    20  tcp.o(i.tcp_next_iss)
    tcp_output                               0x08006451   Thumb Code   610  tcp_out.o(i.tcp_output)
    tcp_pcb_purge                            0x080068bd   Thumb Code   142  tcp.o(i.tcp_pcb_purge)
    tcp_pcb_remove                           0x08006951   Thumb Code   170  tcp.o(i.tcp_pcb_remove)
    tcp_poll                                 0x08006a01   Thumb Code    10  tcp.o(i.tcp_poll)
    tcp_recv                                 0x080076b9   Thumb Code     6  tcp.o(i.tcp_recv)
    tcp_recved                               0x080076e7   Thumb Code    84  tcp.o(i.tcp_recved)
    tcp_rexmit                               0x0800773b   Thumb Code    86  tcp_out.o(i.tcp_rexmit)
    tcp_rst                                  0x08007791   Thumb Code   174  tcp_out.o(i.tcp_rst)
    tcp_seg_free                             0x0800783f   Thumb Code    32  tcp.o(i.tcp_seg_free)
    tcp_segs_free                            0x0800785f   Thumb Code    30  tcp.o(i.tcp_segs_free)
    tcp_send_ctrl                            0x0800787d   Thumb Code    28  tcp_out.o(i.tcp_send_ctrl)
    tcp_sent                                 0x08007899   Thumb Code     6  tcp.o(i.tcp_sent)
    tcp_setprio                              0x0800789f   Thumb Code     4  tcp.o(i.tcp_setprio)
    tcp_update_rcv_ann_wnd                   0x080078f5   Thumb Code    56  tcp.o(i.tcp_update_rcv_ann_wnd)
    tcp_write                                0x0800792d   Thumb Code    72  tcp_out.o(i.tcp_write)
    usart1_Configuration                     0x08007a6d   Thumb Code   182  usart1.o(i.usart1_Configuration)
    OSUnMapTbl                               0x08007bba   Data         256  os_core.o(.constdata)
    tcp_backoff                              0x08007cd6   Data          13  tcp.o(.constdata)
    tcp_persist_backoff                      0x08007ce3   Data           7  tcp.o(.constdata)
    ip_addr_any                              0x08007cf4   Data           4  ip_addr.o(.constdata)
    ip_addr_broadcast                        0x08007cf8   Data           4  ip_addr.o(.constdata)
    ethbroadcast                             0x08007cfc   Data           6  etharp.o(.constdata)
    ethzero                                  0x08007d02   Data           6  etharp.o(.constdata)
    Region$$Table$$Base                      0x08007d08   Number         0  anon$$obj.o(Region$$Table)
    Region$$Table$$Limit                     0x08007d28   Number         0  anon$$obj.o(Region$$Table)
    DMATxDescToSet                           0x20000000   Data           4  stm32_eth.o(.data)
    DMARxDescToGet                           0x20000004   Data           4  stm32_eth.o(.data)
    DMAPTPTxDescToSet                        0x20000008   Data           4  stm32_eth.o(.data)
    DMAPTPRxDescToGet                        0x2000000c   Data           4  stm32_eth.o(.data)
    TcpClient_Link                           0x20000014   Data           1  tcpclient.o(.data)
    message_count                            0x20000018   Data           4  tcpclient.o(.data)
    echoclient_pcb                           0x2000001c   Data           4  tcpclient.o(.data)
    Socket_Client                            0x20000020   Data           4  tcpclient.o(.data)
    rjes                                     0x20000024   Data           4  tcpclient.o(.data)
    Socket_Server                            0x20000030   Data           4  tcpserver.o(.data)
    __stdout                                 0x20000034   Data           4  printf.o(.data)
    OSCtxSwCtr                               0x20000040   Data           4  os_core.o(.data)
    OSEventFreeList                          0x20000044   Data           4  os_core.o(.data)
    OSFlagFreeList                           0x20000048   Data           4  os_core.o(.data)
    OSCPUUsage                               0x2000004c   Data           1  os_core.o(.data)
    OSIdleCtrMax                             0x20000050   Data           4  os_core.o(.data)
    OSIdleCtrRun                             0x20000054   Data           4  os_core.o(.data)
    OSStatRdy                                0x20000058   Data           1  os_core.o(.data)
    OSIntNesting                             0x20000059   Data           1  os_core.o(.data)
    OSLockNesting                            0x2000005a   Data           1  os_core.o(.data)
    OSPrioCur                                0x2000005b   Data           1  os_core.o(.data)
    OSPrioHighRdy                            0x2000005c   Data           1  os_core.o(.data)
    OSRdyGrp                                 0x2000005d   Data           1  os_core.o(.data)
    OSRdyTbl                                 0x2000005e   Data           8  os_core.o(.data)
    OSRunning                                0x20000066   Data           1  os_core.o(.data)
    OSTaskCtr                                0x20000067   Data           1  os_core.o(.data)
    OSIdleCtr                                0x20000068   Data           4  os_core.o(.data)
    OSTCBCur                                 0x2000006c   Data           4  os_core.o(.data)
    OSTCBFreeList                            0x20000070   Data           4  os_core.o(.data)
    OSTCBHighRdy                             0x20000074   Data           4  os_core.o(.data)
    OSTCBList                                0x20000078   Data           4  os_core.o(.data)
    OSTickStepState                          0x2000007c   Data           1  os_core.o(.data)
    OSQFreeList                              0x20000080   Data           4  os_core.o(.data)
    OSTime                                   0x20000084   Data           4  os_core.o(.data)
    tcp_end_time                             0x20000088   Data           4  ethernetif.o(.data)
    arp_end_time                             0x2000008c   Data           4  ethernetif.o(.data)
    MACaddr                                  0x20000090   Data           6  ethernetif.o(.data)
    DMATxDesc                                0x20000098   Data           4  ethernetif.o(.data)
    netif_list                               0x200000ac   Data           4  netif.o(.data)
    netif_default                            0x200000b0   Data           4  netif.o(.data)
    tcp_ticks                                0x200000b8   Data           4  tcp.o(.data)
    tcp_bound_pcbs                           0x200000bc   Data           4  tcp.o(.data)
    tcp_listen_pcbs                          0x200000c0   Data           4  tcp.o(.data)
    tcp_active_pcbs                          0x200000c4   Data           4  tcp.o(.data)
    tcp_tw_pcbs                              0x200000c8   Data           4  tcp.o(.data)
    tcp_tmp_pcb                              0x200000cc   Data           4  tcp.o(.data)
    tcp_input_pcb                            0x200000f4   Data           4  tcp_in.o(.data)
    SystemCoreClock                          0x20000120   Data           4  system_stm32f10x.o(.data)
    AHBPrescTable                            0x20000124   Data          16  system_stm32f10x.o(.data)
    netif                                    0x20000134   Data          48  netconf.o(.bss)
    START_TASK_STK                           0x200003bc   Data         256  stm32_config.o(.bss)
    LED1_TASK_STK                            0x200004bc   Data        4096  stm32_config.o(.bss)
    LED2_TASK_STK                            0x200014bc   Data        4096  stm32_config.o(.bss)
    OSEventTbl                               0x200024bc   Data         200  os_core.o(.bss)
    OSFlagTbl                                0x20002584   Data          80  os_core.o(.bss)
    OSTaskStatStk                            0x200025d4   Data         512  os_core.o(.bss)
    OSTaskIdleStk                            0x200027d4   Data         512  os_core.o(.bss)
    OSTCBPrioTbl                             0x200029d4   Data         256  os_core.o(.bss)
    OSTCBTbl                                 0x20002ad4   Data         924  os_core.o(.bss)
    OSQTbl                                   0x20002e70   Data         120  os_core.o(.bss)
    DMARxDscrTab                             0x20002ee8   Data          64  ethernetif.o(.bss)
    DMATxDscrTab                             0x20002f28   Data          32  ethernetif.o(.bss)
    Rx_Buff                                  0x20002f48   Data        6080  ethernetif.o(.bss)
    Tx_Buff                                  0x20004708   Data        3040  ethernetif.o(.bss)
    __initial_sp                             0x20006c38   Data           0  startup_stm32f10x_cl.o(STACK)



==============================================================================

Memory Map of the image

  Image Entry point : 0x08000151

  Load Region LR_IROM1 (Base: 0x08000000, Size: 0x00007e5c, Max: 0x00040000, ABSOLUTE, COMPRESSED[0x00007d4c])

    Execution Region ER_IROM1 (Base: 0x08000000, Size: 0x00007d28, Max: 0x00040000, ABSOLUTE)

    Base Addr    Size         Type   Attr      Idx    E Section Name        Object

    0x08000000   0x00000150   Data   RO         5028    RESET               startup_stm32f10x_cl.o
    0x08000150   0x00000000   Code   RO         5067  * .ARM.Collect$$$$00000000  mc_w.l(entry.o)
    0x08000150   0x00000004   Code   RO         5337    .ARM.Collect$$$$00000001  mc_w.l(entry2.o)
    0x08000154   0x00000004   Code   RO         5340    .ARM.Collect$$$$00000004  mc_w.l(entry5.o)
    0x08000158   0x00000000   Code   RO         5342    .ARM.Collect$$$$00000008  mc_w.l(entry7b.o)
    0x08000158   0x00000000   Code   RO         5344    .ARM.Collect$$$$0000000A  mc_w.l(entry8b.o)
    0x08000158   0x00000008   Code   RO         5345    .ARM.Collect$$$$0000000B  mc_w.l(entry9a.o)
    0x08000160   0x00000000   Code   RO         5347    .ARM.Collect$$$$0000000D  mc_w.l(entry10a.o)
    0x08000160   0x00000000   Code   RO         5349    .ARM.Collect$$$$0000000F  mc_w.l(entry11a.o)
    0x08000160   0x00000004   Code   RO         5338    .ARM.Collect$$$$00002712  mc_w.l(entry2.o)
    0x08000164   0x000000b4   Code   RO         1967    .text               os_cpu_a.o
    0x08000218   0x00000024   Code   RO         5029    .text               startup_stm32f10x_cl.o
    0x0800023c   0x00000024   Code   RO         5070    .text               mc_w.l(memcpya.o)
    0x08000260   0x00000024   Code   RO         5072    .text               mc_w.l(memseta.o)
    0x08000284   0x0000002c   Code   RO         5351    .text               mc_w.l(uidiv.o)
    0x080002b0   0x00000024   Code   RO         5366    .text               mc_w.l(init.o)
    0x080002d4   0x00000056   Code   RO         5384    .text               mc_w.l(__dczerorl2.o)
    0x0800032a   0x00000002   PAD
    0x0800032c   0x00000028   Code   RO         1162    i.BusFault_Handler  stm32f10x_it.o
    0x08000354   0x00000002   Code   RO         1163    i.DebugMon_Handler  stm32f10x_it.o
    0x08000356   0x00000002   PAD
    0x08000358   0x0000000c   Code   RO          264    i.ETH_DMAClearITPendingBit  stm32_eth.o
    0x08000364   0x00000020   Code   RO          265    i.ETH_DMAITConfig   stm32_eth.o
    0x08000384   0x00000024   Code   RO          268    i.ETH_DMAReceptionCmd  stm32_eth.o
    0x080003a8   0x00000054   Code   RO          269    i.ETH_DMARxDescChainInit  stm32_eth.o
    0x080003fc   0x00000016   Code   RO          271    i.ETH_DMARxDescReceiveITConfig  stm32_eth.o
    0x08000412   0x00000002   PAD
    0x08000414   0x00000024   Code   RO          274    i.ETH_DMATransmissionCmd  stm32_eth.o
    0x08000438   0x00000050   Code   RO          277    i.ETH_DMATxDescChainInit  stm32_eth.o
    0x08000488   0x00000008   Code   RO          278    i.ETH_DMATxDescChecksumInsertionConfig  stm32_eth.o
    0x08000490   0x00000016   Code   RO          286    i.ETH_DeInit        stm32_eth.o
    0x080004a6   0x0000001c   Code   RO          287    i.ETH_Delay         stm32_eth.o
    0x080004c2   0x00000002   PAD
    0x080004c4   0x00000014   Code   RO          292    i.ETH_FlushTransmitFIFO  stm32_eth.o
    0x080004d8   0x0000000c   Code   RO         1971    i.ETH_GetCurrentTxBuffer  ethernetif.o
    0x080004e4   0x0000000a   Code   RO          303    i.ETH_GetDMARxDescFrameLength  stm32_eth.o
    0x080004ee   0x00000002   PAD
    0x080004f0   0x00000048   Code   RO          318    i.ETH_GetRxPktSize  stm32_eth.o
    0x08000538   0x00000018   Code   RO          319    i.ETH_GetSoftwareResetStatus  stm32_eth.o
    0x08000550   0x00000028   Code   RO         1164    i.ETH_IRQHandler    stm32f10x_it.o
    0x08000578   0x00000264   Code   RO          326    i.ETH_Init          stm32_eth.o
    0x080007dc   0x00000034   Code   RO          329    i.ETH_MACAddressConfig  stm32_eth.o
    0x08000810   0x00000024   Code   RO          334    i.ETH_MACReceptionCmd  stm32_eth.o
    0x08000834   0x00000024   Code   RO          335    i.ETH_MACTransmissionCmd  stm32_eth.o
    0x08000858   0x0000006c   Code   RO          346    i.ETH_ReadPHYRegister  stm32_eth.o
    0x080008c4   0x0000009c   Code   RO         1972    i.ETH_RxPkt_ChainMode  ethernetif.o
    0x08000960   0x00000014   Code   RO          357    i.ETH_SoftwareReset  stm32_eth.o
    0x08000974   0x00000020   Code   RO          358    i.ETH_Start         stm32_eth.o
    0x08000994   0x000000a4   Code   RO          359    i.ETH_StructInit    stm32_eth.o
    0x08000a38   0x00000068   Code   RO         1973    i.ETH_TxPkt_ChainMode  ethernetif.o
    0x08000aa0   0x00000068   Code   RO          361    i.ETH_WritePHYRegister  stm32_eth.o
    0x08000b08   0x000000b0   Code   RO          873    i.Ethernet_Configuration  stm32f107.o
    0x08000bb8   0x000000b0   Code   RO          874    i.GPIO_Configuration  stm32f107.o
    0x08000c68   0x0000000c   Code   RO         3257    i.GPIO_ETH_MediaInterfaceConfig  stm32f10x_gpio.o
    0x08000c74   0x00000116   Code   RO         3261    i.GPIO_Init         stm32f10x_gpio.o
    0x08000d8a   0x00000002   PAD
    0x08000d8c   0x00000090   Code   RO         3263    i.GPIO_PinRemapConfig  stm32f10x_gpio.o
    0x08000e1c   0x00000028   Code   RO         1165    i.HardFault_Handler  stm32f10x_it.o
    0x08000e44   0x00000078   Code   RO          171    i.LwIP_Init         netconf.o
    0x08000ebc   0x00000010   Code   RO          173    i.LwIP_Pkt_Handle   netconf.o
    0x08000ecc   0x00000028   Code   RO         1166    i.MemManage_Handler  stm32f10x_it.o
    0x08000ef4   0x00000002   Code   RO         1167    i.NMI_Handler       stm32f10x_it.o
    0x08000ef6   0x00000034   Code   RO          875    i.NVIC_Configuration  stm32f107.o
    0x08000f2a   0x00000002   PAD
    0x08000f2c   0x00000070   Code   RO         3096    i.NVIC_Init         misc.o
    0x08000f9c   0x00000014   Code   RO         3097    i.NVIC_PriorityGroupConfig  misc.o
    0x08000fb0   0x00000028   Code   RO          876    i.NVIC_SetPriority  stm32f107.o
    0x08000fd8   0x00000014   Code   RO         3098    i.NVIC_SetVectorTable  misc.o
    0x08000fec   0x0000002c   Code   RO         1242    i.OSInit            os_core.o
    0x08001018   0x00000002   Code   RO         1876    i.OSInitHookBegin   os_cpu_c.o
    0x0800101a   0x00000002   Code   RO         1877    i.OSInitHookEnd     os_cpu_c.o
    0x0800101c   0x00000024   Code   RO         1243    i.OSIntEnter        os_core.o
    0x08001040   0x00000090   Code   RO         1244    i.OSIntExit         os_core.o
    0x080010d0   0x00000048   Code   RO         1247    i.OSStart           os_core.o
    0x08001118   0x0000004c   Code   RO         1248    i.OSStatInit        os_core.o
    0x08001164   0x00000002   Code   RO         1878    i.OSTCBInitHook     os_cpu_c.o
    0x08001166   0x00000002   PAD
    0x08001168   0x000000a0   Code   RO         1739    i.OSTaskCreate      os_task.o
    0x08001208   0x000000b8   Code   RO         1740    i.OSTaskCreateExt   os_task.o
    0x080012c0   0x00000002   Code   RO         1879    i.OSTaskCreateHook  os_cpu_c.o
    0x080012c2   0x00000002   Code   RO         1881    i.OSTaskIdleHook    os_cpu_c.o
    0x080012c4   0x00000070   Code   RO         1744    i.OSTaskNameSet     os_task.o
    0x08001334   0x00000002   Code   RO         1883    i.OSTaskStatHook    os_cpu_c.o
    0x08001336   0x00000002   PAD
    0x08001338   0x0000008c   Code   RO         1749    i.OSTaskStkChk      os_task.o
    0x080013c4   0x0000009a   Code   RO         1884    i.OSTaskStkInit     os_cpu_c.o
    0x0800145e   0x00000002   PAD
    0x08001460   0x000000a8   Code   RO         1750    i.OSTaskSuspend     os_task.o
    0x08001508   0x00000002   Code   RO         1885    i.OSTaskSwHook      os_cpu_c.o
    0x0800150a   0x00000002   PAD
    0x0800150c   0x00000078   Code   RO         1834    i.OSTimeDly         os_time.o
    0x08001584   0x000000ec   Code   RO         1249    i.OSTimeTick        os_core.o
    0x08001670   0x00000002   Code   RO         1886    i.OSTimeTickHook    os_cpu_c.o
    0x08001672   0x00000002   PAD
    0x08001674   0x00000058   Code   RO         1433    i.OS_FlagInit       os_flag.o
    0x080016cc   0x00000054   Code   RO         1256    i.OS_InitEventList  os_core.o
    0x08001720   0x00000054   Code   RO         1257    i.OS_InitMisc       os_core.o
    0x08001774   0x00000044   Code   RO         1258    i.OS_InitRdyList    os_core.o
    0x080017b8   0x00000080   Code   RO         1259    i.OS_InitTCBList    os_core.o
    0x08001838   0x00000050   Code   RO         1260    i.OS_InitTaskIdle   os_core.o
    0x08001888   0x00000050   Code   RO         1261    i.OS_InitTaskStat   os_core.o
    0x080018d8   0x00000012   Code   RO         1262    i.OS_MemClr         os_core.o
    0x080018ea   0x00000002   PAD
    0x080018ec   0x00000050   Code   RO         1622    i.OS_QInit          os_q.o
    0x0800193c   0x00000074   Code   RO         1264    i.OS_Sched          os_core.o
    0x080019b0   0x0000002c   Code   RO         1265    i.OS_SchedNew       os_core.o
    0x080019dc   0x00000134   Code   RO         1267    i.OS_TCBInit        os_core.o
    0x08001b10   0x00000028   Code   RO         1268    i.OS_TaskIdle       os_core.o
    0x08001b38   0x00000088   Code   RO         1269    i.OS_TaskStat       os_core.o
    0x08001bc0   0x0000003c   Code   RO         1270    i.OS_TaskStatStkChk  os_core.o
    0x08001bfc   0x0000001a   Code   RO         1752    i.OS_TaskStkClr     os_task.o
    0x08001c16   0x00000002   PAD
    0x08001c18   0x00000020   Code   RO         3370    i.RCC_AHBPeriphClockCmd  stm32f10x_rcc.o
    0x08001c38   0x00000020   Code   RO         3371    i.RCC_AHBPeriphResetCmd  stm32f10x_rcc.o
    0x08001c58   0x00000020   Code   RO         3372    i.RCC_APB1PeriphClockCmd  stm32f10x_rcc.o
    0x08001c78   0x00000020   Code   RO         3374    i.RCC_APB2PeriphClockCmd  stm32f10x_rcc.o
    0x08001c98   0x00000190   Code   RO         3382    i.RCC_GetClocksFreq  stm32f10x_rcc.o
    0x08001e28   0x0000003c   Code   RO         3383    i.RCC_GetFlagStatus  stm32f10x_rcc.o
    0x08001e64   0x0000000c   Code   RO         3394    i.RCC_MCOConfig     stm32f10x_rcc.o
    0x08001e70   0x0000000c   Code   RO         3400    i.RCC_PLL3Cmd       stm32f10x_rcc.o
    0x08001e7c   0x00000018   Code   RO         3401    i.RCC_PLL3Config    stm32f10x_rcc.o
    0x08001e94   0x00000002   Code   RO         1168    i.SVC_Handler       stm32f10x_it.o
    0x08001e96   0x00000008   Code   RO         5033    i.SetSysClock       system_stm32f10x.o
    0x08001e9e   0x00000002   PAD
    0x08001ea0   0x00000118   Code   RO         5034    i.SetSysClockTo72   system_stm32f10x.o
    0x08001fb8   0x0000002c   Code   RO         1974    i.Set_MAC_Address   ethernetif.o
    0x08001fe4   0x00000028   Code   RO         3100    i.SysTick_CLKSourceConfig  misc.o
    0x0800200c   0x00000010   Code   RO         1124    i.SysTick_Handler   delay.o
    0x0800201c   0x0000006c   Code   RO         5036    i.SystemInit        system_stm32f10x.o
    0x08002088   0x00000076   Code   RO          877    i.System_Setup      stm32f107.o
    0x080020fe   0x00000002   PAD
    0x08002100   0x00000040   Code   RO          912    i.TCP_Client_Recv   tcpclient.o
    0x08002140   0x00000034   Code   RO          913    i.TCP_Client_Send   tcpclient.o
    0x08002174   0x00000040   Code   RO          987    i.TCP_Server_Recv   tcpserver.o
    0x080021b4   0x00000034   Code   RO          988    i.TCP_Server_Send   tcpserver.o
    0x080021e8   0x0000006c   Code   RO         1082    i.USART1_IRQHandler  usart1.o
    0x08002254   0x00000012   Code   RO         3623    i.USART_ClearFlag   stm32f10x_usart.o
    0x08002266   0x0000001e   Code   RO         3624    i.USART_ClearITPendingBit  stm32f10x_usart.o
    0x08002284   0x00000018   Code   RO         3627    i.USART_Cmd         stm32f10x_usart.o
    0x0800229c   0x0000001a   Code   RO         3630    i.USART_GetFlagStatus  stm32f10x_usart.o
    0x080022b6   0x00000054   Code   RO         3631    i.USART_GetITStatus  stm32f10x_usart.o
    0x0800230a   0x0000004a   Code   RO         3633    i.USART_ITConfig    stm32f10x_usart.o
    0x08002354   0x000000d8   Code   RO         3634    i.USART_Init        stm32f10x_usart.o
    0x0800242c   0x0000000a   Code   RO         3641    i.USART_ReceiveData  stm32f10x_usart.o
    0x08002436   0x00000008   Code   RO         3644    i.USART_SendData    stm32f10x_usart.o
    0x0800243e   0x00000002   PAD
    0x08002440   0x0000002c   Code   RO         1169    i.UsageFault_Handler  stm32f10x_it.o
    0x0800246c   0x00000020   Code   RO         5165    i.__0printf$3       mc_w.l(printf3.o)
    0x0800248c   0x0000000e   Code   RO         5378    i.__scatterload_copy  mc_w.l(handlers.o)
    0x0800249a   0x00000002   Code   RO         5379    i.__scatterload_null  mc_w.l(handlers.o)
    0x0800249c   0x0000000e   Code   RO         5380    i.__scatterload_zeroinit  mc_w.l(handlers.o)
    0x080024aa   0x00000002   PAD
    0x080024ac   0x000001b8   Code   RO         5172    i._printf_core      mc_w.l(printf3.o)
    0x08002664   0x0000005c   Code   RO         1125    i.delay_init        delay.o
    0x080026c0   0x00000048   Code   RO         1126    i.delay_ms          delay.o
    0x08002708   0x0000004c   Code   RO         1128    i.delay_us          delay.o
    0x08002754   0x00000132   Code   RO         2999    i.etharp_arp_input  etharp.o
    0x08002886   0x0000003a   Code   RO         3001    i.etharp_ip_input   etharp.o
    0x080028c0   0x000000c4   Code   RO         3002    i.etharp_output     etharp.o
    0x08002984   0x000001b8   Code   RO         3003    i.etharp_query      etharp.o
    0x08002b3c   0x000000ca   Code   RO         3004    i.etharp_raw        etharp.o
    0x08002c06   0x00000002   PAD
    0x08002c08   0x0000002c   Code   RO         3005    i.etharp_request    etharp.o
    0x08002c34   0x0000004e   Code   RO         3006    i.etharp_send_ip    etharp.o
    0x08002c82   0x0000006a   Code   RO         3008    i.ethernet_input    etharp.o
    0x08002cec   0x0000004c   Code   RO         1975    i.ethernetif_init   ethernetif.o
    0x08002d38   0x0000002c   Code   RO         1976    i.ethernetif_input  ethernetif.o
    0x08002d64   0x00000204   Code   RO         3009    i.find_entry        etharp.o
    0x08002f68   0x00000024   Code   RO         1053    i.fputc             printf.o
    0x08002f8c   0x00000040   Code   RO         3010    i.free_etharp_q     etharp.o
    0x08002fcc   0x0000001a   Code   RO         2796    i.htonl             inet.o
    0x08002fe6   0x0000000c   Code   RO         2797    i.htons             inet.o
    0x08002ff2   0x00000012   Code   RO         2761    i.icmp_dest_unreach  icmp.o
    0x08003004   0x00000194   Code   RO         2762    i.icmp_input        icmp.o
    0x08003198   0x00000076   Code   RO         2763    i.icmp_send_response  icmp.o
    0x0800320e   0x00000012   Code   RO         2764    i.icmp_time_exceeded  icmp.o
    0x08003220   0x00000014   Code   RO         2845    i.inet_chksum       inet_chksum.o
    0x08003234   0x00000056   Code   RO         2846    i.inet_chksum_pbuf  inet_chksum.o
    0x0800328a   0x0000004e   Code   RO         2925    i.ip_addr_isbroadcast  ip_addr.o
    0x080032d8   0x0000014c   Code   RO         2947    i.ip_frag           ip_frag.o
    0x08003424   0x00000184   Code   RO         2883    i.ip_input          ip.o
    0x080035a8   0x00000034   Code   RO         2884    i.ip_output         ip.o
    0x080035dc   0x00000104   Code   RO         2885    i.ip_output_if      ip.o
    0x080036e0   0x00000198   Code   RO         2948    i.ip_reass          ip_frag.o
    0x08003878   0x000001a8   Code   RO         2949    i.ip_reass_chain_frag_into_datagram_and_validate  ip_frag.o
    0x08003a20   0x00000034   Code   RO         2950    i.ip_reass_dequeue_datagram  ip_frag.o
    0x08003a54   0x00000054   Code   RO         2951    i.ip_reass_enqueue_new_datagram  ip_frag.o
    0x08003aa8   0x000000ac   Code   RO         2952    i.ip_reass_free_complete_datagram  ip_frag.o
    0x08003b54   0x0000007c   Code   RO         2953    i.ip_reass_remove_oldest_datagram  ip_frag.o
    0x08003bd0   0x00000050   Code   RO         2886    i.ip_route          ip.o
    0x08003c20   0x000000a4   Code   RO         1977    i.low_level_init    ethernetif.o
    0x08003cc4   0x00000074   Code   RO         1978    i.low_level_input   ethernetif.o
    0x08003d38   0x00000034   Code   RO         1979    i.low_level_output  ethernetif.o
    0x08003d6c   0x0000004a   Code   RO         2848    i.lwip_standard_chksum  inet_chksum.o
    0x08003db6   0x00000002   PAD
    0x08003db8   0x00000034   Code   RO            1    i.main              main.o
    0x08003dec   0x00000100   Code   RO          158    i.main_Client_task  main_cilent.o
    0x08003eec   0x00000060   Code   RO          146    i.main_Server_task  main_server.o
    0x08003f4c   0x00000078   Code   RO         2167    i.mem_free          mem.o
    0x08003fc4   0x00000064   Code   RO         2168    i.mem_init          mem.o
    0x08004028   0x00000130   Code   RO         2169    i.mem_malloc        mem.o
    0x08004158   0x00000148   Code   RO         2170    i.mem_realloc       mem.o
    0x080042a0   0x0000002c   Code   RO         2210    i.memp_free         memp.o
    0x080042cc   0x00000064   Code   RO         2211    i.memp_init         memp.o
    0x08004330   0x0000003c   Code   RO         2212    i.memp_malloc       memp.o
    0x0800436c   0x00000068   Code   RO         2252    i.netif_add         netif.o
    0x080043d4   0x0000000c   Code   RO         2254    i.netif_is_up       netif.o
    0x080043e0   0x00000028   Code   RO         2256    i.netif_set_addr    netif.o
    0x08004408   0x0000000c   Code   RO         2257    i.netif_set_default  netif.o
    0x08004414   0x0000000c   Code   RO         2259    i.netif_set_gw      netif.o
    0x08004420   0x00000078   Code   RO         2260    i.netif_set_ipaddr  netif.o
    0x08004498   0x0000000c   Code   RO         2261    i.netif_set_netmask  netif.o
    0x080044a4   0x0000002c   Code   RO         2262    i.netif_set_up      netif.o
    0x080044d0   0x0000000c   Code   RO         2801    i.ntohl             inet.o
    0x080044dc   0x0000000c   Code   RO         2802    i.ntohs             inet.o
    0x080044e8   0x00000214   Code   RO         2330    i.pbuf_alloc        pbuf.o
    0x080046fc   0x00000050   Code   RO         2331    i.pbuf_cat          pbuf.o
    0x0800474c   0x00000016   Code   RO         2332    i.pbuf_chain        pbuf.o
    0x08004762   0x00000012   Code   RO         2333    i.pbuf_clen         pbuf.o
    0x08004774   0x000000dc   Code   RO         2335    i.pbuf_copy         pbuf.o
    0x08004850   0x0000009a   Code   RO         2336    i.pbuf_copy_partial  pbuf.o
    0x080048ea   0x00000098   Code   RO         2338    i.pbuf_free         pbuf.o
    0x08004982   0x0000008c   Code   RO         2339    i.pbuf_header       pbuf.o
    0x08004a0e   0x000000b0   Code   RO         2340    i.pbuf_realloc      pbuf.o
    0x08004abe   0x0000000a   Code   RO         2341    i.pbuf_ref          pbuf.o
    0x08004ac8   0x000000b4   Code   RO         2171    i.plug_holes        mem.o
    0x08004b7c   0x0000007c   Code   RO            2    i.start_task        main.o
    0x08004bf8   0x0000009c   Code   RO         2435    i.tcp_abandon       tcp.o
    0x08004c94   0x00000004   Code   RO         2436    i.tcp_accept        tcp.o
    0x08004c98   0x00000008   Code   RO         2437    i.tcp_accept_null   tcp.o
    0x08004ca0   0x000000b4   Code   RO         2438    i.tcp_alloc         tcp.o
    0x08004d54   0x00000004   Code   RO         2439    i.tcp_arg           tcp.o
    0x08004d58   0x000000f8   Code   RO         2440    i.tcp_bind          tcp.o
    0x08004e50   0x00000038   Code   RO          914    i.tcp_client_close  tcpclient.o
    0x08004e88   0x00000050   Code   RO          915    i.tcp_client_error  tcpclient.o
    0x08004ed8   0x00000030   Code   RO          916    i.tcp_client_sent   tcpclient.o
    0x08004f08   0x000001b0   Code   RO         2441    i.tcp_close         tcp.o
    0x080050b8   0x00000124   Code   RO         2442    i.tcp_connect       tcp.o
    0x080051dc   0x00000070   Code   RO          917    i.tcp_echoclient_connect  tcpclient.o
    0x0800524c   0x00000098   Code   RO          918    i.tcp_echoclient_connected  tcpclient.o
    0x080052e4   0x00000040   Code   RO          919    i.tcp_echoclient_connection_close  tcpclient.o
    0x08005324   0x0000006c   Code   RO          920    i.tcp_echoclient_poll  tcpclient.o
    0x08005390   0x000000cc   Code   RO          921    i.tcp_echoclient_recv  tcpclient.o
    0x0800545c   0x000000a0   Code   RO          989    i.tcp_echoserver_accept  tcpserver.o
    0x080054fc   0x00000040   Code   RO          990    i.tcp_echoserver_connection_close  tcpserver.o
    0x0800553c   0x00000028   Code   RO          991    i.tcp_echoserver_error  tcpserver.o
    0x08005564   0x0000004c   Code   RO          992    i.tcp_echoserver_init  tcpserver.o
    0x080055b0   0x00000060   Code   RO          993    i.tcp_echoserver_poll  tcpserver.o
    0x08005610   0x00000150   Code   RO          994    i.tcp_echoserver_recv  tcpserver.o
    0x08005760   0x00000048   Code   RO          995    i.tcp_echoserver_send  tcpserver.o
    0x080057a8   0x0000002e   Code   RO          996    i.tcp_echoserver_sent  tcpserver.o
    0x080057d6   0x0000002e   Code   RO         2443    i.tcp_eff_send_mss  tcp.o
    0x08005804   0x0000042c   Code   RO         2679    i.tcp_enqueue       tcp_out.o
    0x08005c30   0x00000006   Code   RO         2444    i.tcp_err           tcp.o
    0x08005c36   0x00000002   PAD
    0x08005c38   0x000004a8   Code   RO         2631    i.tcp_input         tcp_in.o
    0x080060e0   0x00000058   Code   RO         2446    i.tcp_kill_prio     tcp.o
    0x08006138   0x0000003c   Code   RO         2447    i.tcp_kill_timewait  tcp.o
    0x08006174   0x00000150   Code   RO         2632    i.tcp_listen_input  tcp_in.o
    0x080062c4   0x000000ec   Code   RO         2448    i.tcp_listen_with_backlog  tcp.o
    0x080063b0   0x0000000a   Code   RO         2449    i.tcp_new           tcp.o
    0x080063ba   0x00000002   PAD
    0x080063bc   0x00000078   Code   RO         2450    i.tcp_new_port      tcp.o
    0x08006434   0x0000001c   Code   RO         2451    i.tcp_next_iss      tcp.o
    0x08006450   0x00000268   Code   RO         2681    i.tcp_output        tcp_out.o
    0x080066b8   0x000000cc   Code   RO         2682    i.tcp_output_segment  tcp_out.o
    0x08006784   0x00000084   Code   RO         2683    i.tcp_output_set_header  tcp_out.o
    0x08006808   0x000000b4   Code   RO         2633    i.tcp_parseopt      tcp_in.o
    0x080068bc   0x00000094   Code   RO         2452    i.tcp_pcb_purge     tcp.o
    0x08006950   0x000000b0   Code   RO         2453    i.tcp_pcb_remove    tcp.o
    0x08006a00   0x0000000a   Code   RO         2454    i.tcp_poll          tcp.o
    0x08006a0a   0x00000002   PAD
    0x08006a0c   0x000005ac   Code   RO         2634    i.tcp_process       tcp_in.o
    0x08006fb8   0x00000700   Code   RO         2635    i.tcp_receive       tcp_in.o
    0x080076b8   0x00000006   Code   RO         2455    i.tcp_recv          tcp.o
    0x080076be   0x00000028   Code   RO         2456    i.tcp_recv_null     tcp.o
    0x080076e6   0x00000054   Code   RO         2457    i.tcp_recved        tcp.o
    0x0800773a   0x00000056   Code   RO         2684    i.tcp_rexmit        tcp_out.o
    0x08007790   0x000000ae   Code   RO         2686    i.tcp_rst           tcp_out.o
    0x0800783e   0x00000020   Code   RO         2458    i.tcp_seg_free      tcp.o
    0x0800785e   0x0000001e   Code   RO         2459    i.tcp_segs_free     tcp.o
    0x0800787c   0x0000001c   Code   RO         2687    i.tcp_send_ctrl     tcp_out.o
    0x08007898   0x00000006   Code   RO         2460    i.tcp_sent          tcp.o
    0x0800789e   0x00000004   Code   RO         2461    i.tcp_setprio       tcp.o
    0x080078a2   0x00000002   PAD
    0x080078a4   0x00000050   Code   RO         2636    i.tcp_timewait_input  tcp_in.o
    0x080078f4   0x00000038   Code   RO         2464    i.tcp_update_rcv_ann_wnd  tcp.o
    0x0800792c   0x00000048   Code   RO         2688    i.tcp_write         tcp_out.o
    0x08007974   0x000000f8   Code   RO         3011    i.update_arp_entry  etharp.o
    0x08007a6c   0x000000c4   Code   RO         1083    i.usart1_Configuration  usart1.o
    0x08007b30   0x0000004c   Data   RO          923    .constdata          tcpclient.o
    0x08007b7c   0x0000003e   Data   RO          998    .constdata          tcpserver.o
    0x08007bba   0x00000100   Data   RO         1272    .constdata          os_core.o
    0x08007cba   0x0000001c   Data   RO         2214    .constdata          memp.o
    0x08007cd6   0x0000001e   Data   RO         2465    .constdata          tcp.o
    0x08007cf4   0x00000008   Data   RO         2926    .constdata          ip_addr.o
    0x08007cfc   0x0000000c   Data   RO         3013    .constdata          etharp.o
    0x08007d08   0x00000020   Data   RO         5376    Region$$Table       anon$$obj.o


    Execution Region RW_IRAM1 (Base: 0x20000000, Size: 0x00006c38, Max: 0x00010000, ABSOLUTE, COMPRESSED[0x00000024])

    Base Addr    Size         Type   Attr      Idx    E Section Name        Object

    0x20000000   0x00000010   Data   RW          362    .data               stm32_eth.o
    0x20000010   0x00000018   Data   RW          924    .data               tcpclient.o
    0x20000028   0x0000000c   Data   RW          999    .data               tcpserver.o
    0x20000034   0x00000004   Data   RW         1054    .data               printf.o
    0x20000038   0x00000004   Data   RW         1088    .data               usart1.o
    0x2000003c   0x00000004   Data   RW         1129    .data               delay.o
    0x20000040   0x00000048   Data   RW         1273    .data               os_core.o
    0x20000088   0x00000014   Data   RW         1981    .data               ethernetif.o
    0x2000009c   0x0000000d   Data   RW         2173    .data               mem.o
    0x200000a9   0x00000003   PAD
    0x200000ac   0x00000009   Data   RW         2263    .data               netif.o
    0x200000b5   0x00000003   PAD
    0x200000b8   0x00000020   Data   RW         2466    .data               tcp.o
    0x200000d8   0x00000020   Data   RW         2638    .data               tcp_in.o
    0x200000f8   0x0000000a   Data   RW         2887    .data               ip.o
    0x20000102   0x00000002   PAD
    0x20000104   0x00000006   Data   RW         2956    .data               ip_frag.o
    0x2000010a   0x00000001   Data   RW         3014    .data               etharp.o
    0x2000010b   0x00000014   Data   RW         3410    .data               stm32f10x_rcc.o
    0x2000011f   0x00000001   PAD
    0x20000120   0x00000014   Data   RW         5037    .data               system_stm32f10x.o
    0x20000134   0x00000030   Zero   RW          174    .bss                netconf.o
    0x20000164   0x000000c8   Zero   RW          922    .bss                tcpclient.o
    0x2000022c   0x000000c8   Zero   RW          997    .bss                tcpserver.o
    0x200002f4   0x000000c8   Zero   RW         1087    .bss                usart1.o
    0x200003bc   0x00002100   Zero   RW         1220    .bss                stm32_config.o
    0x200024bc   0x00000a2c   Zero   RW         1271    .bss                os_core.o
    0x20002ee8   0x00002400   Zero   RW         1980    .bss                ethernetif.o
    0x200052e8   0x00000414   Zero   RW         2172    .bss                mem.o
    0x200056fc   0x00000a7f   Zero   RW         2213    .bss                memp.o
    0x2000617b   0x00000001   PAD
    0x2000617c   0x00000014   Zero   RW         2637    .bss                tcp_in.o
    0x20006190   0x000005e0   Zero   RW         2955    .bss                ip_frag.o
    0x20006770   0x000000c8   Zero   RW         3012    .bss                etharp.o
    0x20006838   0x00000400   Zero   RW         5026    STACK               startup_stm32f10x_cl.o


==============================================================================

Image component sizes


      Code (inc. data)   RO Data    RW Data    ZI Data      Debug   Object Name

       256         32          0          4          0       2433   delay.o
      2258         32         12          1        200      13145   etharp.o
       768         62          0         20       9216      20142   ethernetif.o
       558          0          0          0          0       4070   icmp.o
        62          0          0          0          0       2344   inet.o
       180          0          0          0          0       5841   inet_chksum.o
         0          0          0          0          0       8458   init.o
       780         28          0         10          0       5085   ip.o
        78          0          8          0          0       5773   ip_addr.o
      1596         42          0          6       1504       8517   ip_frag.o
       176         48          0          0          0     296209   main.o
       256        100          0          0          0        707   main_cilent.o
        96         34          0          0          0        611   main_server.o
      1032         74          0         13       1044       5353   mem.o
       204         30         28          0       2687       4118   memp.o
       192         30          0          0          0       2767   misc.o
       136         32          0          0         48      16461   netconf.o
       356         24          0          9          0       7723   netif.o
      1854        368        256         72       2604      18954   os_core.o
       180         36          0          0          0        368   os_cpu_a.o
       170          0          0          0          0      12987   os_cpu_c.o
        88         14          0          0          0        606   os_flag.o
        80          8          0          0          0        575   os_q.o
       790         64          0          0          0       5528   os_task.o
       120         20          0          0          0        644   os_time.o
      1504          0          0          0          0       8405   pbuf.o
        36          4          0          4          0       2510   printf.o
        36          8        336          0       1024        816   startup_stm32f10x_cl.o
         0          0          0          0       8448        725   stm32_config.o
      1650        136          0         16          0      49150   stm32_eth.o
       562         26          0          0          0      18317   stm32f107.o
       434         12          0          0          0       3494   stm32f10x_gpio.o
       210        124          0          0          0       3828   stm32f10x_it.o
       636         72          0         20          0       8941   stm32f10x_rcc.o
       490          6          0          0          0       7713   stm32f10x_usart.o
       396         32          0         20          0       2377   system_stm32f10x.o
      2510        172         30         32          0      28006   tcp.o
      5032        248          0         32         20      15532   tcp_in.o
      2380         16          0          0          0       8902   tcp_out.o
       940        188         76         24        200       8353   tcpclient.o
      1006        132         62         12        200       8358   tcpserver.o
       304         28          0          4        200       2263   usart1.o

    ----------------------------------------------------------------------
     30436       2282        840        308      27396     627109   Object Totals
         0          0         32          0          0          0   (incl. Generated)
        44          0          0          9          1          0   (incl. Padding)

    ----------------------------------------------------------------------

      Code (inc. data)   RO Data    RW Data    ZI Data      Debug   Library Member Name

        86          0          0          0          0          0   __dczerorl2.o
         0          0          0          0          0          0   entry.o
         0          0          0          0          0          0   entry10a.o
         0          0          0          0          0          0   entry11a.o
         8          4          0          0          0          0   entry2.o
         4          0          0          0          0          0   entry5.o
         0          0          0          0          0          0   entry7b.o
         0          0          0          0          0          0   entry8b.o
         8          4          0          0          0          0   entry9a.o
        30          0          0          0          0          0   handlers.o
        36          8          0          0          0         68   init.o
        36          0          0          0          0         68   memcpya.o
        36          0          0          0          0        108   memseta.o
       472         14          0          0          0        184   printf3.o
        44          0          0          0          0         80   uidiv.o

    ----------------------------------------------------------------------
       764         30          0          0          0        508   Library Totals
         4          0          0          0          0          0   (incl. Padding)

    ----------------------------------------------------------------------

      Code (inc. data)   RO Data    RW Data    ZI Data      Debug   Library Name

       760         30          0          0          0        508   mc_w.l

    ----------------------------------------------------------------------
       764         30          0          0          0        508   Library Totals

    ----------------------------------------------------------------------

==============================================================================


      Code (inc. data)   RO Data    RW Data    ZI Data      Debug   

     31200       2312        840        308      27396     615213   Grand Totals
     31200       2312        840         36      27396     615213   ELF Image Totals (compressed)
     31200       2312        840         36          0          0   ROM Totals

==============================================================================

    Total RO  Size (Code + RO Data)                32040 (  31.29kB)
    Total RW  Size (RW Data + ZI Data)             27704 (  27.05kB)
    Total ROM Size (Code + RO Data + RW Data)      32076 (  31.32kB)

==============================================================================

